:100000000C94A60E0C943F5D0C94D70E0C94D70E56
:100010000C94D70E0C9430650C94E0A20C94D70E7F
:100020000C94D70E0C94D70E0C94D70E0C94D70EBC
:100030000C94D70E0C94D70E0C94D70E0C94D70EAC
:100040000C94D70E0C94D2410C94B4640C94D70E3B
:100050000C94D70E0C94D70E0C94D70E0C94305BE6
:100060000C94D70E0C94A5920C947C920C94D70E01
:100070000C94D70E0C94D70E0C94D70E0C94D70E6C
:100080000C94EF6E0C94D70E0C94D70E0C94D70EE4
:100090000C9453920C942A920C94D70E0C94D70E75
:1000A0000C94D70E0C94D70E0C94D70E0C94D70E3C
:1000B0000C94D70E0C94AF8A0C94D70E0C94D70ED8
:1000C0000C94D70E0C94D70E0C94D70E0C9401926E
:1000D0000C94D8910C94D70E0C94AF910C948691FB
:1000E0000C94D70EC01BC31BCA1BCD1BD01BD31B2C
:1000F000DA1BE11BE41BEB1BF21BF91BA821D62129
:100100000D2244221F2356238423B22379247924E9
:1001100079247924792479247924792479247924F7
:1001200079247924792479247924792479247924E7
:1001300079247924792479247924792479247924D7
:100140007924792479247B22B222EA22E0230E2426
:10015000462477267D26832689268F2695269B266C
:10016000A126A726AD26B326B926CB26D126D7268B
:10017000EF26F526FB26012707270D27132719272A
:100180001F2725272B27312737273D274927552785
:100190005B27612767277F2785278B27912797274D
:1001A0009D278D2893289928AB28B128B728C928DE
:1001B000CF28D528DB28E128E7281129172941294C
:1001C00047294D2953296B29712977297D29122A1D
:1001D000122A122A122A122A122A122A122A9329BF
:1001E00097299B29A129A529A929AD29B129B52993
:1001F000B929BF29DD29E329E9296D27A327A927E3
:10020000AF27B527BB27C12759295F29652983292E
:1002100089298F29EF29F529FB29ED28F328C727FC
:10022000CD27D327D927DF27E5279F28BD284F27AC
:10023000BF26C52673277927012A072A0D2A4327B7
:100240001D29232929292F2935293B29EB27F12786
:10025000F727FD27032809280F2815281B28212800
:1002600027282D28332839283F2845284B2851286E
:100270005D28632869286F2875287B2881288728AE
:10028000D129CB29C529D729A528C328DD26E326CE
:10029000E926F9285728FF2805290B2976315331FB
:1002A0002C319331EA31B231E131D0319B327E329F
:1002B0005732EB32B832B832DA32C332813981394F
:1002C000903981399D39B639D139EC3989528D52FD
:1002D0009152955299529D52A152A552A952AD5296
:1002E000B152DD52E152E852F552025315532853F0
:1002F00041535A5378538E53B456B756A656AA56FE
:10030000B056EE56BB56BF56C556C956CD56D356F7
:10031000D756DB56EE56E156E556E956CA58CF5841
:10032000D458DE58E8586159F258FA5802590C5915
:10033000165920592F593959615943594D5957590F
:10034000CB7FFF7F348054808980F18001812B82B4
:1003500075817F81B381E881F6812B82BD80DE8A41
:10036000E78AEF8A038B158B278B328BE3A5FAA5DF
:1003700011A628A63FA66DA684A69BA6B2A6D1A6C6
:10038000E9A600A71FA735A756A605A84CCDB2D44D
:100390004EB93836A9020C50B9918688083CA6AAF5
:1003A000AA2ABE000000803F3400330032004E6FA6
:1003B0006E650053746F70706564004E657574727D
:1003C000616C205475726E004D6F76696E672052B5
:1003D000657665727365004D6F76696E6720466F4E
:1003E0007277617264004272616B696E670054419A
:1003F0004E4B20524553544F52454400250048650A
:10040000616C7468204C6576656C3A2000564548EE
:1004100049434C452052455041495220434F4D508D
:100420004C4554450054414E4B2044455354524F83
:100430005945440025004865616C7468204C657618
:10044000656C3A2000290056454849434C452052E6
:1004500045504149522053544152544544202800AC
:10046000524550414952204F5045524154494F4EF8
:100470002043414E43454C4C45440029004D4143E7
:1004800048494E452047554E2048495421202800D0
:10049000524550414952204F5045524154494F4EC8
:1004A0002043414E43454C4C454400290043414EB6
:1004B0004E4F4E20484954212028005475727265D1
:1004C0007420726F746174696F6E206973206E6F2F
:1004D00074206F66207479706520536572766F2E74
:1004E000204E6F20736574757020617661696C6150
:1004F000626C652E004E6F207374656572696E675D
:1005000020736572766F2061737369676E65642C02
:100510002072652D636865636B2076656869636C1E
:100520006520747970652E0054757272657420654B
:100530006C65766174696F6E206973206E6F7420CC
:100540006F66207479706520536572766F2E204E29
:100550006F20736574757020617661696C61626C7F
:10056000652E00546F70204C65667400546F7020C7
:1005700043656E74657200546F70205269676874C9
:10058000004D6964646C65204C656674004D696457
:10059000646C652043656E746572004D6964646CBB
:1005A0006520526967687400426F74746F6D204CE7
:1005B00065667400426F74746F6D2043656E746578
:1005C0007200426F74746F6D2052696768740046E0
:1005D00049524D574152452056455253494F4E3A84
:1005E00020006942757300534275730050504D00EE
:1005F0004E6F6E6520446574656374656400417A6E
:10060000696D7574682020202000456C65766174E2
:10061000696F6E2020005475726E202020202020EB
:1006200020005468726F74746C652020200053742D
:1006300069636B202020202020204D696E2020201F
:100640002043656E7465722020204D617820202043
:10065000204465616462616E642020526576657233
:1006600073656400524144494F20494E464F202D46
:1006700020004E4F542044455445435445440049BE
:10068000474E4F52454400416E616C6F67004469AC
:10069000676974616C00417578204368616E2E2033
:1006A00020204D696E20202020204D6178202020C0
:1006B000202054797065004368616E6E656C73200C
:1006C0007574696C697A65643A20004368616E6E7E
:1006D000656C732064657465637465643A200020FA
:1006E0002844697361626C656429002028456E6145
:1006F000626C656429004D656368616E6963616C55
:10070000207265636F696C00416972736F66740073
:100710004D656368616E6963616C204261727265E8
:100720006C3A200020284D31290020284D32290024
:10073000202842290042617272656C20456C657602
:100740006174696F6E3A20200020284D3029002006
:10075000284D312900202841290054757272657492
:1007600020526F746174696F6E3A2020200020411E
:100770006D70732900202843757272656E74204C69
:10078000696D69743A20004472697665204D6F7412
:100790006F72733A202020202020004D4F544F527A
:1007A00020545950455300496E646570656E646508
:1007B0006E7420547265616420436F6E74726F6C46
:1007C0000054616E6B202854616D69796120444D3D
:1007D00044290054616E6B2028444B4C4D204765E2
:1007E0006172626F7829004361720048616C6674BF
:1007F0007261636B0054616E6B00554E4B4E4F57E8
:100800004E00596573004E6F002900252C20446569
:1008100063656C65726174696F6E20666163746F85
:1008200072200020284B69636B6261636B207370D8
:100830006565642000547261636B205265636F6963
:100840006C20456E61626C65643A202020004E2F5A
:100850004120666F722076656869636C65207479E3
:100860007065005475726E204D6F64653A202020CB
:10087000202020202020202020202000250053742C
:10088000656572696E672050637420746F2074729E
:10089000656164733A20004E2F4120666F722076A6
:1008A000656869636C6520747970650059657320AB
:1008B0002854616D69796129002500202D20004EA2
:1008C00065757472616C205475726E20416C6C6F2A
:1008D0007765643A202020002073656300547261BC
:1008E0006E736D697373696F6E2044656C61793ADC
:1008F0002020202020002073656300456E67696E0C
:10090000652050617573652054696D653A2020201B
:1009100020202000207365630053686966742054AA
:10092000696D653A202020202020202020202020D2
:1009300020004175746F6D61746963004D616E755F
:10094000616C005472616E736D697373696F6E20B0
:10095000547970653A202020202020002500596518
:1009600073202D2000526576657273652053706583
:100970006564204C696D697465643A202000250027
:10098000596573202D2000466F7277617264205381
:1009900070656564204C696D697465643A20200057
:1009A000206D73290025207468726F74746C652043
:1009B000666F7220002028004D6F746F72204E7594
:1009C00064676520456E61626C65643A2020202072
:1009D0000029004E6F6E65004E6F6E65002C205032
:1009E00072657365743A20002900202841646A7595
:1009F0007374656420746F200020284C6576656CE4
:100A00003A2000446563656C2052616D7020456E2C
:100A100061626C65643A20202020200029004E6F1E
:100A20006E65004E6F6E65002C20507265736574A4
:100A30003A20002900202841646A75737465642097
:100A4000746F200020284C6576656C3A2000416365
:100A500063656C2052616D7020456E61626C6564E7
:100A60003A2020202020004163746976652044727A
:100A70006976696E672050726F66696C653A20000E
:100A800056656869636C6520547970653A2020204A
:100A90002020202020202020004452495645205369
:100AA000455454494E4753002073656300526563B3
:100AB0006F696C2064656C61793A202020202020C9
:100AC0002020202020202020202020202000250061
:100AD000596573202D200042617272656C20456C4F
:100AE00065766174696F6E205370656564204C692A
:100AF0006D697465643A20002500596573202D20C6
:100B00000054757272657420526F746174696F6EEF
:100B1000205370656564204C696D697465643A2082
:100B200020005455525245542053455454494E4781
:100B30005300556E6B6E6F776E0045787065726905
:100B40006D656E74616C00536570617261746520CF
:100B50004865617420262046616E00436F6D6269AE
:100B60006E6564204865617420262046616E00250C
:100B70000044697361626C656400536D6F6B65203E
:100B80007768656E2064657374726F7965643A2066
:100B90000046616E206D61782073706565643A204F
:100BA000202020202020200046616E206661737482
:100BB0002069646C652073706565643A2020004686
:100BC000616E2069646C652073706565643A2020ED
:100BD000202020202000202863757272656E746CBE
:100BE000792064697361626C6564290020736563B0
:100BF0006F6E6473004E2F41005072652D68656101
:100C0000742064656C61793A202020202020200027
:100C1000536D6F6B657220547970653A20202020E7
:100C200020202020202000536D6F6B6572206F758F
:100C30007470757420636F6E74726F6C6C65642071
:100C40006D616E75616C6C7900534D4F4B45520070
:100C5000556E6B6E6F776E004865617679004D65F5
:100C60006469756D004C6967687400437573746FCF
:100C70006D00556E6B6E6F776E004E6F6E65004F38
:100C800070656E2050616E7A65720054616D69798D
:100C90006120537065630020736563207265636F24
:100CA000766572792900207365632072656C6F61C7
:100CB000642C2000204D4720686974732C2000208C
:100CC00063616E6E6F6E20686974732C200028005B
:100CD00057656967687420436C6173733A202020FC
:100CE00020200044616D6167652050726F66696CF9
:100CF000653A202020005965732028004163636510
:100D00007074204D472044616D6167653A20005939
:100D1000657320280053656E64204D47204952209A
:100D2000436F64653A2020004E2F41005265706188
:100D3000697265642062793A202020202020004ECC
:100D40002F41004869742050726F746F636F6C207C
:100D5000323A20202000290020285465616D2000AF
:100D6000466972652050726F746F636F6C3A202011
:100D7000202000466972652050726F746F636F6C3B
:100D80003A2020202000497320526570616972204A
:100D900054616E6B3F202020004952202620546170
:100DA0006E6B20426174746C696E67204469736174
:100DB000626C656400424154544C4520494E464F94
:100DC00000554E4B4E4F574E0042656E6564696E3E
:100DD0006920544253204D6963726F004265696512
:100DE000722055534D2D52432D3200546169676571
:100DF0006E20536F756E642043617264004F70659E
:100E00006E2050616E7A657220536F756E64204358
:100E10006172640042656E6564696E692054425374
:100E2000204D696E6900536F756E64206361726452
:100E30003A2000534F554E44204341524400556ED2
:100E40006B6E6F776E0042617272656C20456C65E7
:100E5000766174696F6E20436F6D6D616E640054CE
:100E6000757272657420526F746174696F6E20437D
:100E70006F6D6D616E64005374656572696E672095
:100E8000436F6D6D616E640056656869636C6520C3
:100E9000537065656400456E67696E6520537065C3
:100EA0006564005468726F74746C6520436F6D6D77
:100EB000616E64005370656564206465637265618A
:100EC0007365732062656C6F77200053706565648D
:100ED00020696E637265617365732061626F766508
:100EE00020005475726E2053746F70706564004CEE
:100EF000656674205475726E2053746172746564F3
:100F0000005269676874205475726E205374617260
:100F10007465640056656869636C652053746F700E
:100F2000706564004D6F76696E67205265766572F4
:100F30007365004D6F76696E6720466F72776172D8
:100F40006400456E67696E652053746F7000456E6E
:100F500067696E652053746172740043616E6E6FD1
:100F60006E2052656C6F61646564005665686963E4
:100F70006C652044657374726F7965640043616EBB
:100F80006E6F6E20486974004272616B6573204118
:100F900070706C696564005661726961626C6500AD
:100FA000290020286F662000506F7320004175785B
:100FB000204368616E6E656C2000566172696162E3
:100FC0006C65004F6E004F66660042004100457838
:100FD0007465726E616C20496E707574200007082C
:100FE00009090B0C0C0B0C0C5475727265742053B0
:100FF0007469636B202D200046756E6374696F6E93
:10100000202300202D3E200020736563005475725C
:10101000726574206D6F76656D656E742064656CA5
:1010200061793A2020004E6F6E6500596573005457
:10103000757272657420737469636B2066756E6374
:1010400074696F6E733A200046554E4354494F4EB3
:101050002054524947474552530076206375746FB8
:10106000666629002028004C564320456E61626C5C
:1010700065643A202020202020007600566F6C7492
:101080006167653A20202020202020202020005960
:101090006573004E6F004261747465727920446517
:1010A0007465637465643A20004241545445525952
:1010B0000053657269616C20332054782042617559
:1010C000643A2020004175782053657269616C2074
:1010D000426175643A202020004D6F746F72205376
:1010E000657269616C20426175643A200055534213
:1010F0002053657269616C20426175643A2020203A
:10110000004241554420524154455300212000469D
:101110004143544F525920524553455421200020F9
:101120002D2053746F70005573657220536F756E68
:1011300064200041202D200042202D2000536F7597
:101140006E642042616E6B2000506C61792F537485
:101150006F7000506C61792052616E646F6D005049
:101160006C61792050726576696F757300506C619F
:1011700079204E6578740020287769746820495278
:101180002900466972652043616E6E6F6E00466984
:10119000726520526570616972205369676E616C77
:1011A00000416972736F6674202D204D616E756108
:1011B0006C2054726967676572004D656368616E83
:1011C0006963616C205265636F696C202D204D61ED
:1011D0006E75616C20547269676765720053657241
:1011E000766F205265636F696C202D204D616E759E
:1011F000616C20547269676765720048696768208E
:10120000496E74656E7369747920466C61736820E9
:10121000556E6974202D204D616E75616C2054727D
:101220006967676572004D47205374617274004DA1
:10123000472053746F70004952204E4F5420656E02
:1012400061626C6564202D206E6F2049522070729F
:101250006F746F636F6C732073656C656374656422
:101260002E00556E61626C6520746F20656E616240
:101270006C6520495200495220656E61626C65645C
:101280000049522064697361626C6564004175783D
:10129000204F757470757420466C617368656400C6
:1012A000417578204F757470757420496E7665723B
:1012B000736520466C61736865640053746F7020B9
:1012C000417578204F757470757420426C696E6B2F
:1012D000696E670053746F70205265766F6C766923
:1012E0006E6720417578204C696768740053746F8D
:1012F0007020416C6C205573657220536F756E645D
:101300007300494F20506F72742041202D2050757A
:101310006C73656400494F20506F72742041202D1A
:1013200020537461727420426C696E6B696E670041
:10133000494F20506F72742041204F75747075743E
:10134000202D204F6E00494F20506F727420412095
:101350004F7574707574202D204F666600494F20BC
:10136000506F72742042204F7574707574202D2058
:101370004F6E00494F20506F72742042204F757499
:10138000707574202D204F6666004C5643204578BA
:101390006974202D20566F6C7461676520526573E7
:1013A000746F726564007629004C5643207468722D
:1013B0006573686F6C642072656163686564212081
:1013C00028004C696768742031204F6E004C6967B3
:1013D00068742031204F6666004C6967687420325B
:1013E000204F6E004C696768742032204F6666009B
:1013F000326E64204D472053746F7000326E64204B
:101400004D472053746172740052756E6E696E6739
:10141000204C6967687473204F6E0052756E6E6958
:101420006E67204C6967687473204F66660041756B
:1014300078204F7574707574204F6E004175782058
:101440004F7574707574204F66660053746F70200A
:101450005265766F6C76696E6720417578204C69AD
:101460006768740053746F7020417578204F7574ED
:1014700070757420426C696E6B696E670041757897
:10148000204F7574707574205072657365742044B4
:10149000696D00537461727420417578204F7574C2
:1014A00070757420426C696E6B696E670000002174
:1014B00000240027002A002D003000330001010025
:1014C00000040107010A0100002200250028002B6A
:1014D000002E003100340002010000050108010B5C
:1014E00001494F20506F72742042202D2050756C9E
:1014F00073656400494F20506F72742042202D2084
:10150000537461727420426C696E6B696E6700552A
:101510007365722046756E6374696F6E2031005575
:101520007365722046756E6374696F6E2032004673
:101530006F72776172642047656172004E657574E1
:1015400072616C20476561720052657665727365E1
:1015500020476561720053657420416363656C20A8
:1015600052616D70204C6576656C3A20005365744D
:1015700020446563656C2052616D70204C65766512
:101580006C3A2000416E616C6F6720557365722064
:1015900046756E6374696F6E2031202D2000416E98
:1015A000616C6F6720557365722046756E63746950
:1015B0006F6E2032202D20002D00202D20002000D5
:1015C000545255450046414C53450025005761692A
:1015D00074696E6720666F7220726164696F2E2E67
:1015E0002E200054616967656E2056322F563300F5
:1015F000536F6E790052435441204D616368696EA8
:10160000652047756E00436C61726B204D616368A5
:10161000696E652047756E005243544120526570D3
:1016200061697200494255205265706169720043D8
:101630006C61726B20526570616972004F70656EEB
:1016400050616E7A657200567354616E6B00464F3E
:10165000560054616967656E2056310048656E67B3
:10166000204C6F6E670054616D69796120312F33B2
:10167000350054616D69796120322D53686F7400B3
:1016800054616D69796100556E6B6E6F776E003ACB
:10169000200042697420004761703A200052616462
:1016A000696F205265616479202D2000526576654E
:1016B000727365643A2020004D61782050756C7318
:1016C000653A20004D696E2050756C73653A2000B4
:1016D000456E642056616C75657300456E642052DA
:1016E00065636F696C20536572766F2053657475FE
:1016F0007000456E6420526F746174696F6E205380
:101700006572766F20536574757000456E64205362
:1017100074656572696E6720536572766F205365D4
:1017200074757000456E64205374656572696E67E8
:1017300020536572766F20536574757000456E6432
:1017400020456C65766174696F6E20536572766FA3
:1017500020536574757000536572766F20756E2D19
:10176000726576657273656400536572766F207278
:10177000657665727365640052657665727365643B
:101780003A2020004D61782050756C73653A200036
:101790004D696E2050756C73653A20005374617208
:1017A000742056616C75657300494E56414C49442E
:1017B00020534552564F2E204E4F205345545550DE
:1017C0002E005365747570205265636F696C2053E9
:1017D0006572766F0053657475702054757272650A
:1017E0007420526F746174696F6E2050616E205363
:1017F0006572766F005365747570205374656572F9
:10180000696E6720536572766F20284F7574707506
:1018100074203229005365747570205374656572A5
:10182000696E6720536572766F20284F75747075E6
:101830007420342900536574757020547572726574
:101840007420456C65766174696F6E20536572769D
:101850006F00416972736F6674202D20456E61625E
:101860006C6564004D656368616E6963616C2052EC
:1018700065636F696C202D20456E61626C65640044
:10188000416972736F6674202D2044697361626CC4
:101890006564004D656368616E6963616C205265C3
:1018A000636F696C202D2044697361626C6564000C
:1018B000436F6D6D73206368616E67656420746F3C
:1018C0002055534200436F6D6D73206368616E67EE
:1018D000656420746F2053657269616C2031004427
:1018E000726976696E672050726F66696C652073E5
:1018F000657420746F202300250053706565642093
:101900007265647563656420746F2000537065654B
:101910006420726573746F726564005475726E2012
:10192000456E67696E65204F6E00207365636F6E4C
:1019300064732061676F202D20736D6F6B6572205B
:101940007072656865617420736B6970706564009E
:10195000456E67696E65206C6173742073746F7077
:101960007065642000207365636F6E647300536D4F
:101970006F6B6572207072652D6865617420737479
:101980006172746564202D20656E67696E652077CD
:10199000696C6C207475726E206F6E20696E200009
:1019A0004D616E75616C207472616E736D697373D5
:1019B000696F6E202D2070757420696E206E6575BC
:1019C0007472616C2067656172206265666F726512
:1019D000207374617274696E6720656E67696E65E5
:1019E0002100456E67696E65204175746F205368EC
:1019F0007574646F776E00456E6761676520547219
:101A0000616E736D697373696F6E00446973656E9F
:101A100067616765205472616E736D697373696F76
:101A20006E00536574205475726E204D6F64653A74
:101A3000203100536574205475726E204D6F6465BB
:101A40003A203200536574205475726E204D6F64D5
:101A5000653A203300456E61626C65204E65757491
:101A600072616C205475726E730044697361626CAC
:101A700065204E65757472616C205475726E7300CA
:101A8000401F7017D007A00FA00FDC05D007C409B6
:101A900010278813983A102758026C0258026C02DB
:101AA00058026C0258026C0258026C0258026C0216
:101AB00058026C0258026C025802B0366C023A02AC
:101AC0006C023A026C023A026C02B036384A5C127E
:101AD0001C255C125C121C255C12BC7FC7F2C0780E
:101AE00087A5B7C5A00F8813B80B401FB80BB80B5C
:101AF0007017401F556E6B6E6F776E004F6E626F82
:101B0000617264204D6F746F7220447269766572E1
:101B10007320432026204400446574616368656433
:101B20002F4E41005265636F696C20536572766F6A
:101B30000050616E20536572766F00536572766F48
:101B40002F455343004F6E626F617264204D6F7476
:101B50006F7220447269766572004F70656E205016
:101B6000616E7A65722053636F7574205365726974
:101B7000616C20455343005361626572746F6F74EA
:101B8000682053657269616C00506F6C6F6C7520D2
:101B900053657269616C00536572766F2031005332
:101BA0006572766F203200536572766F2033005372
:101BB0006572766F203400536572766F203500535E
:101BC0006572766F203600536572766F203700534A
:101BD0006572766F2038000000200023002600295F
:101BE000002C002F00320000010000030106010953
:101BF0000105050505070508080808020202020A92
:101C00000A0808040404040101010101010101039F
:101C100003030303030303040707070C0C0C0C0C5A
:101C20000C0C0C0202020206060606060606060B4D
:101C30000B0B0B0B0B0B0B010210202008081020C4
:101C40004010204080020102010804020101020448
:101C50000810204080804020100804020180040207
:101C6000018040201008040201080402010102045E
:101C70000810204080010204081020408000000A63
:101C80000B02090C0D0E0807030401000000000000
:101C90000000000000000000000000000000000044
:101CA0000000000000000000001211100000000001
:101CB0000000000000000000000000000000000024
:101CC000000000536D6F6B657220656E61626C651C
:101CD0006400536D6F6B65722064697361626C653B
:101CE000640053657420766F6C756D653A20002032
:101CF0002D20537461727420526570656174696E31
:101D000067004865617420416D743A200048656140
:101D1000743A200053616D652061732066616E0026
:101D20005374617274205265766F6C76696E6720A9
:101D3000417578204C6967687400524144494F20CE
:101D40004641494C53414645000072BB11241FBE19
:101D5000CFEFD1E2DEBFCDBF00E00CBF17E0A0E0C7
:101D6000B2E0E0EDFEEB01E00BBF02C007900D9288
:101D7000AC32B107D9F725E1ACE2B7E001C01D9262
:101D8000A435B207E1F71EE0C6EADEE000E006C0D7
:101D900021970109802FFE010E94A0CBC53AD107EF
:101DA00080E00807A9F70E948BA80C94F3CD0C944F
:101DB00000002F923F924F925F926F927F928F928C
:101DC0009F92AF92BF92CF92DF92EF92FF920F93CA
:101DD0001F93CF93DF93CDB7DEB7E6970FB6F89496
:101DE000DEBF0FBECDBF80918E1490918F140E94E4
:101DF0005A900E94BC616FEC75E080918E149091B6
:101E00008F140E9452916DE876E0CE0101960E94F7
:101E1000DA8F80918E1490918F14DC01ED91FC91FA
:101E20004D815E8169817A810280F381E02D19956F
:101E300065E976E080918E1490918F140E94519103
:101E40002AE041EE51E060E070E080918E149091C4
:101E50008F140E94129060ED76E080918E14909124
:101E60008F140E945D90CE0101960E947E8F0E9489
:101E7000C9A080918E1490918F14DC01ED91FC919A
:101E80000680F781E02D199580918E1490918F1422
:101E90000E945A900E94BC6164E676E080918E14A4
:101EA00090918F140E945291E091620CE4300CF0FA
:101EB000E0E080EF95E09A8389838CEE95E09C8347
:101EC0008B8387EE95E09E838D8382EE95E09887E5
:101ED0008F83EE0FFF0B21E030E02C0F3D1FE20F50
:101EE000F31F6081718180918E1490918F140E94F4
:101EF00076910E94BC616EE276E080918E149091A2
:101F00008F140E9476910E94BC6162E276E080911B
:101F10008E1490918F140E945291E091C511F0910E
:101F2000C61181819281883E934014F40E94AC6175
:101F3000E091C511F091C6116181728180918E147A
:101F400090918F140E94038484E00E9405A8E09180
:101F5000C511F091C6116581768180918E149091A2
:101F60008F140E94038485E00E9405A8E091C511AA
:101F7000F091C6116381748180918E1490918F14B9
:101F80000E94038484E00E9405A8E091C511F091AD
:101F9000C611678180918E1490918F140E94518296
:101FA00088E00E9405A8E091C511F091C6118085D6
:101FB0000E94926166E176E080918E1490918F1478
:101FC0000E945291E091CF11F091D01181819281C4
:101FD000883E934014F40E94AC61E091CF11F091DF
:101FE000D0116181728180918E1490918F140E9422
:101FF000038484E00E9405A8E091CF11F091D011F4
:102000006581768180918E1490918F140E94038453
:1020100085E00E9405A8E091CF11F091D011638175
:10202000748180918E1490918F140E94038484E0B7
:102030000E9405A8E091CF11F091D01167818091A5
:102040008E1490918F140E94518288E00E9405A8FE
:10205000E091CF11F091D01180850E9492616AE0E9
:1020600076E080918E1490918F140E945291E091AD
:10207000D911F091DA1181819281883E934014F454
:102080000E94AC61E091D911F091DA116181728105
:1020900080918E1490918F140E94038484E00E949A
:1020A00005A8E091D911F091DA11658176818091CE
:1020B0008E1490918F140E94038485E00E9405A8DD
:1020C000E091D911F091DA116381748180918E14BD
:1020D00090918F140E94038484E00E9405A8E091EF
:1020E000D911F091DA11678180918E1490918F143B
:1020F0000E94518288E00E9405A8E091D911F091D8
:10210000DA1180850E9492616EEF75E080918E14E5
:1021100090918F140E945291E091E311F091E4119B
:1021200081819281883E934014F40E94AC61E091D9
:10213000E311F091E4116181728180918E1490918C
:102140008F140E94038484E00E9405A8E091E311AB
:10215000F091E4116581768180918E1490918F14B5
:102160000E94038485E00E9405A8E091E311F091AC
:10217000E4116381748180918E1490918F140E9478
:10218000038484E00E9405A8E091E311F091E4113A
:10219000678180918E1490918F140E94518288E003
:1021A0000E9405A8E091E311F091E41180850E945E
:1021B000926180918E1490918F140E945A900E9487
:1021C0007D50C82E66E976E080918E1490918F1430
:1021D0000E9476910E94BC6109E611E1E12CF12C8C
:1021E000D12C5701BFEFAB1ABB0AB50180918E14F9
:1021F00090918F140E940384E9E0EE16F10410F42C
:102200008BE001C08AE00E9405A8D8012C91809142
:102210008E1490918F142223C9F11596ED91FC91A3
:102220001697618172810E940384D8011596ED9101
:10223000FC91169781819281883E934014F40E940C
:10224000AC6184E00E9405A8D8011596ED91FC913F
:1022500016976381748180918E1490918F140E94DF
:10226000038484E00E9405A8D8011596ED91FC91A5
:102270001697278180918E1490918F14222319F044
:102280006EE876E00BC067E876E008C0EC14FD0469
:102290001CF46FE776E002C062E776E00E94769178
:1022A000095F1F4F7501BCE0AB16B10409F099CF6F
:1022B0000E94BC616BEC76E080918E1490918F143B
:1022C0000E9452910E947D50682F80918E149091AF
:1022D0008F140E943A8267EB76E080918E14909181
:1022E0008F140E94529160915F0C7091600C8091EC
:1022F0008E1490918F140E9439840E94C9A08091FD
:102300008E1490918F14DC01ED91FC910680F78181
:10231000E02D199580918E1490918F140E945A90FF
:102320000E94BC616BE977E080918E1490918F14CC
:102330000E9476910E94BC6167E877E080918E14DC
:1023400090918F140E9452918091C4130E941C8915
:10235000BC0180918E1490918F140E9452918091B3
:10236000C4138A30C1F465E777E080918E149091B0
:102370008F140E9452916091821480918E149091DA
:102380008F140E9451826EE677E080918E149091B6
:102390008F140E94529180918E1490918F140E94FC
:1023A0005A906AE577E080918E1490918F140E9484
:1023B00052918091C5130E941C89BC0180918E149A
:1023C00090918F140E9452912091C51380918E1488
:1023D00090918F142B303CF4293054F4283069F458
:1023E00069E477E007C02B3041F465E577E002C08F
:1023F0006FE477E00E94769102C00E945A9065E3F4
:1024000077E080918E1490918F140E945291809168
:10241000C6130E941C89BC0180918E1490918F1468
:102420000E9452912091C61380918E1490918F1426
:102430002B303CF4293054F4283069F464E277E01E
:1024400007C02B3041F460E377E002C06AE277E036
:102450000E94769102C00E945A9060E177E08091DC
:102460008E1490918F140E9452912091D8138091D4
:102470008E1490918F14222319F068E077E002C047
:1024800066EF76E00E9452912091E40F80918E14C5
:1024900090918F14222319F06BEE76E002C06FED5D
:1024A00076E00E94529180918E1490918F140E9438
:1024B0005A900E94C9A080918E1490918F14DC01D3
:1024C000ED91FC910680F781E02D19958091000235
:1024D000823011F00C94F41CF090FF130091021460
:1024E00010E080918E1490918F140E945A900E9457
:1024F000BC6169E97AE080918E1490918F140E94FA
:1025000076910E94BC6160E87AE080918E1490918F
:102510008F140E945291E0910F14E7300CF0E0E02C
:102520008AEF97E09A83898385EF97E09C838B837A
:102530008BEE97E09E838D8387EE97E098878F835D
:1025400083ED97E09A87898781EC97E09C878B875A
:1025500087EA97E09E878D87EE0FFF0B21E030E042
:102560002C0F3D1FE20FF31F6081718180918E144B
:1025700090918F140E94769167E67AE080918E1494
:1025800090918F140E9452916091000280918E145C
:1025900090918F140E943A826EE47AE080918E14BA
:1025A00090918F140E9452918F2D0E947D61FF2087
:1025B00009F44BC064E47AE080918E1490918F14FA
:1025C0000E94529180918E1490918F14112339F0B2
:1025D0006091FA130E9451829091FA1306C06091A3
:1025E00000140E945182909100148091101598134C
:1025F0000C94FB1C68E27AE080918E1490918F1409
:102600000E94529180918E1490918F14112339F071
:102610006091FB1361110CC063E27AE006C0609127
:102620000114611105C06EE17AE00E94529105C06B
:10263000062E000C770B0E9403846CE17AE08091F7
:102640008E1490918F140E94529180918E149091CB
:102650008F140E945A9063E07AE080918E149091DA
:102660008F140E945291802F0E947D61002309F4F3
:102670004BC069EF79E080918E1490918F140E9485
:10268000529180918E1490918F14112339F06091A2
:10269000FD130E9451829091FD1306C060910314B6
:1026A0000E945182909103148091121598130C94FA
:1026B000151D6DED79E080918E1490918F140E941C
:1026C000529180918E1490918F14112339F0609162
:1026D000FE1361110CC068ED79E006C0609104142E
:1026E000611105C063ED79E00E94529105C0062E8C
:1026F000000C770B0E94038461ED79E080918E14C9
:1027000090918F140E94529180918E1490918F1409
:102710000E945A9068EB79E080918E1490918F140A
:102720000E94529180911814811103C00E948B6104
:1027300035C062E078E080918E1490918F140E94F1
:10274000529165EB79E080918E1490918F140E94E4
:1027500052916091181480918E1490918F140E9460
:10276000518265EA79E080918E1490918F140E94D5
:1027700052914091191450911A1460E070E02AE0CF
:1027800080918E1490918F140E94129060EA79E0EB
:1027900080918E1490918F140E94769167E879E071
:1027A00080918E1490918F140E94529180911014F8
:1027B0008436C8F460E879E080918E1490918F148B
:1027C0000E9452916091101480918E1490918F14F8
:1027D0000E9451826EE779E080918E1490918F145F
:1027E0000E94769103C080E00E948B6165E679E0EB
:1027F00080918E1490918F140E94529180911114A7
:102800008436C8F46EE579E080918E1490918F142F
:102810000E9452916091111480918E1490918F14A6
:102820000E9451826CE579E080918E1490918F1412
:102830000E94769103C080E00E948B6163E479E09E
:1028400080918E1490918F140E9452912091C10713
:1028500080918E1490918F14222319F06CE379E00B
:1028600002C062E379E00E94769169E179E08091AB
:102870008E1490918F140E94529160910614709161
:102880000714072E000C880B990B0E9441C820E00A
:1028900030E04AE754E40E9446CAAB01BC0121E0A3
:1028A00080918E1490918F140E94749064E179E06D
:1028B00080918E1490918F140E9476916BEF78E046
:1028C00080918E1490918F140E94529160910814FF
:1028D00070910914072E000C880B990B0E9441C8B7
:1028E00020E030E04AE754E40E9446CAAB01BC0154
:1028F00021E080918E1490918F140E94749066EF65
:1029000078E080918E1490918F140E9476916DEDF5
:1029100078E080918E1490918F140E945291609172
:102920000A1470910B14072E000C880B990B0E944F
:1029300041C820E030E04AE754E40E9446CAAB01B7
:10294000BC0121E080918E1490918F140E947490AC
:1029500068ED78E080918E1490918F140E947691AA
:102960006FEB78E080918E1490918F140E945291B9
:1029700090910F14913011F09430F9F480910C146F
:102980000E947D6180910C14882329F16BEB78E023
:1029900080918E1490918F140E94529160910D1429
:1029A00080918E1490918F140E94518269EB78E08F
:1029B00080918E1490918F140CC020918E143091C0
:1029C0008F14953019F46CEA78E002C067E978E07A
:1029D000C9010E94529180918E1490918F140E948F
:1029E0005A9080910F148230C1F46EE778E08091A4
:1029F0008E1490918F140E945291609112148091C4
:102A00008E1490918F140E9451826CE778E080912F
:102A10008E1490918F140E94769163E678E08091F5
:102A20008E1490918F140E94529190910F142FEF59
:102A3000290F80918E1490918F14223028F4609188
:102A40002C070E943A8204C06EE478E00E947691DE
:102A500065E378E080918E1490918F140E945291DA
:102A600080911C140E947D6180911C14882341F187
:102A700063E278E080918E1490918F140E945291BD
:102A800060911D1480918E1490918F140E94518238
:102A90006BE078E080918E1490918F140E94529197
:102AA00060911E1480918E1490918F140E94518217
:102AB00069E078E080918E1490918F140E94529179
:102AC00080918E1490918F140E945A900E94C9A0F8
:102AD00080918E1490918F14DC01ED91FC91068011
:102AE000F781E02D199580918E1490918F140E949A
:102AF0005A900E94BC6162E27BE080918E149091BA
:102B00008F140E9476910E94BC6161E07BE080910D
:102B10008E1490918F140E9452918091CD1384361F
:102B2000C8F46AEF7AE080918E1490918F140E941D
:102B300052916091CD1380918E1490918F140E94C8
:102B4000518268EF7AE080918E1490918F140E94E8
:102B5000769103C080E00E948B6167ED7AE08091FE
:102B60008E1490918F140E9452918091CC138436D0
:102B7000C8F460ED7AE080918E1490918F140E94D9
:102B800052916091CC1380918E1490918F140E9479
:102B900051826EEC7AE080918E1490918F140E9495
:102BA000769103C080E00E948B616DEA7AE08091AB
:102BB0008E1490918F140E9452916091DA1370914B
:102BC000DB131616170614F500918E1410918F144E
:102BD000072E000C880B990B0E9441C820E030E0C2
:102BE0004AE754E40E9446CAAB01BC0122E0C80196
:102BF0000E947490C8010E945A9068EA7AE080911D
:102C00008E1490918F140E94769103C080E00E94F0
:102C10008B610E94C9A080918E1490918F14DC0169
:102C2000ED91FC910680F781E02D199580918E142D
:102C300090918F140E945A900E94BC6169E47CE0DC
:102C400080918E1490918F140E9476910E94BC61A5
:102C50002091E71380918E1490918F14FE0131968C
:102C60006F01211103C067E27CE0C7C160E17CE035
:102C70000E945291E091F013E3300CF0E3E08BE519
:102C80009BE09A83898387E49BE09C838B838AE320
:102C90009BE09E838D8382E39BE098878F83EE0F7A
:102CA000FF0BEC0DFD1D6081718180918E14909160
:102CB0008F140E947691FF24F3948091F013811178
:102CC00001C0F12C69EF7BE080918E1490918F14FC
:102CD0000E9452916091F11380918E1490918F1403
:102CE000611105C065EF7BE00E9476911AC00E94D9
:102CF00051826CEE7BE080918E1490918F140E9433
:102D0000529180910E08811108C066ED7BE08091A0
:102D10008E1490918F140E94529181EF99E00E943D
:102D20005A906091E8137091E913072E000C880BFC
:102D3000990B0E9441C820E030E04FE753E40E9425
:102D400046CA20E030E048EC52E40E94A0C820E0EF
:102D500030E040E05FE30E94E2C90E94AECAE62E86
:102D6000262F372F8901A090F213B090F3136FEB49
:102D70007BE080918E1490918F140E9452918E2D41
:102D80000E946E61043611053CF40E94AC610A3069
:102D9000110514F40E94AC6183E00E9405A8FF2095
:102DA00001F10E946BA8B501BB0C880B990B0E9426
:102DB00041C820E030E04FE753E40E9446CA20E0DB
:102DC00030E048EC52E40E94A0C820E030E040E04F
:102DD0005FE30E94E2C90E94AECA862F0E946E6124
:102DE00004C00E9463A80E945BA80E94A661609133
:102DF000EA137091EB13072E000C880B990B0E94BD
:102E000041C820E030E04FE753E40E9446CA20E08A
:102E100030E048EC52E40E94A0C820E030E040E0FE
:102E20005FE30E94E2C90E94AECAE62E262F372F2A
:102E30008901A090F413B090F51368EA7BE08091CB
:102E40008E1490918F140E9452918E2D0E946E616B
:102E5000043611053CF40E94AC610A30110514F4EB
:102E60000E94AC6183E00E9405A8FF2001F10E944E
:102E70006BA8B501BB0C880B990B0E9441C820E0E0
:102E800030E04FE753E40E9446CA20E030E048ECCF
:102E900052E40E94A0C820E030E040E05FE30E94DE
:102EA000E2C90E94AECA862F0E946E6104C00E94D1
:102EB00063A80E945BA80E94A6616091EC137091C8
:102EC000ED13072E000C880B990B0E9441C820E0DF
:102ED00030E04FE753E40E9446CA20E030E048EC7F
:102EE00052E40E94A0C820E030E040E05FE30E948E
:102EF000E2C90E94AECAE62E262F372F8901A09084
:102F0000F613B090F71361E97BE080918E149091F5
:102F10008F140E9452918E2D0E946E61043611050D
:102F20003CF40E94AC610A30110514F40E94AC61BB
:102F300083E00E9405A8FF2001F10E946BA8B50163
:102F4000BB0C880B990B0E9441C820E030E04FE792
:102F500053E40E9446CA20E030E048EC52E40E946C
:102F6000A0C820E030E040E05FE30E94E2C90E9498
:102F7000AECA862F0E946E6104C00E9463A80E94A0
:102F80005BA80E94A6616AE77BE080918E14909115
:102F90008F140E9452916091EE137091EF13009183
:102FA0008E1410918F146115710521F461E77BE097
:102FB000C80123C0072E000C880B990B0E9441C842
:102FC00020E030E04FE753E40E9446CA20E030E0C2
:102FD00048EC52E40E94A0C820E030E040E05FE30B
:102FE0000E94E2C90E94AECAC8010E9403846FE633
:102FF0007BE080918E1490918F140E9476910E94B4
:10300000C9A080918E1490918F14DC01ED91FC91F8
:103010000680F781E02D199580918E1490918F1480
:103020000E945A900E94BC6165EB7DE080918E14F5
:1030300090918F140E9476910E94BC6120914C0760
:1030400080918E1490918F14222309F4B7C166E801
:103050007DE00E9452910E94A2660E948B610E94B4
:10306000A26620918E1430918F14882389F063E733
:103070007DE0C9010E94529180914F070E945F6AD2
:10308000BC0180918E1490918F140E9476914BC058
:1030900060E67DE0C9010E94529180914C070E9438
:1030A0005F6ABC0180918E1490918F140E9452919E
:1030B00080914D07882389F168E57DE080918E1429
:1030C00090918F140E945291E0914D07E4300CF0E2
:1030D000E0E08EEA93E09A8389838CEA93E09C8314
:1030E0008B838AEA93E09E838D8388EA93E09887B6
:1030F0008F83EE0FFF0BEC0DFD1D608171818091C0
:103100008E1490918F140E94529166E57DE080911B
:103110008E1490918F140E94529180918E149091F0
:103120008F140E945A9063E47DE080918E149091F8
:103130008F140E94529180914E0700918E1410912D
:103140008F14882321F00E945F6ABC0102C06FE3E4
:103150007DE0C8010E9476916CE27DE080918E1442
:1031600090918F140E94529180914F0700918E147C
:1031700010918F14882321F00E945F6ABC0102C065
:1031800068E27DE0C8010E94769165E17DE0809172
:103190008E1490918F140E94529180915107882330
:1031A000E1F06FE07DE080918E1490918F140E9489
:1031B0005291809150070E945F6ABC0180918E14E9
:1031C00090918F140E94529160ED76E080918E1460
:1031D00090918F140E945D9003C080E00E948B61EB
:1031E0006CEF7CE080918E1490918F140E9452912C
:1031F000809152078823E1F066EF7CE080918E1485
:1032000090918F140E945291809150070E945F6AA2
:10321000BC0180918E1490918F140E94529160EDA8
:1032200076E080918E1490918F140E945D9003C07F
:1032300080E00E948B6163EE7CE080918E1490911F
:103240008F140E945291E0915307E3300CF0E3E0B9
:103250008BE89CE09A8389838FE79CE09C838B8337
:103260008AE79CE09E838D8382E79CE098878F832A
:10327000EE0FFF0BEC0DFD1D6081718180918E14AE
:1032800090918F140E94769160ED7CE080918E1475
:1032900090918F140E945291E0914507E4300CF018
:1032A000E4E08BE69CE09A83898385E69CE09C833E
:1032B0008B838EE59CE09E838D8388E59CE09887D8
:1032C0008F8380E59CE09A878987EE0FFF0BEC0DDA
:1032D000FD1D6081718180918E1490918F140E94E8
:1032E00076916EEC7CE080918E1490918F140E9408
:1032F000529160914A0780918E1490918F140E9490
:1033000051826FEB7CE080918E1490918F140E941B
:10331000529180914507811110C060914B078091B7
:103320008E1490918F140E94518264EB7CE0809106
:103330008E1490918F140E94529160914607709163
:103340004707072E000C880B990B0E9441C820E00C
:1033500030E04AE754E40E9446CAAB01BC0121E0D8
:1033600080918E1490918F140E94749066EA7CE094
:1033700080918E1490918F140E9452916091480711
:1033800070914907072E000C880B990B0E9441C8C9
:1033900020E030E04AE754E40E9446CAAB01BC0199
:1033A00021E080918E1490918F140E94749067E9AF
:1033B0007CE080918E1490918F1402C069E97DE0C9
:1033C0000E9476910E94C9A080918E1490918F14D2
:1033D000DC01ED91FC910680F781E02D199580913B
:1033E0008E1490918F140E945A900E94BC6163E3E6
:1033F0007EE080918E1490918F140E9476910E94AD
:10340000BC6166E27EE080918E1490918F140E94E0
:103410005291E0912514E6300CF0E6E08EE0D60102
:103420001D928A95E9F784E19EE09A8389838DEF66
:103430009DE09C838B838BEE9DE09E838D838CED42
:103440009DE098878F8389EC9DE09A87898781EC3E
:103450009DE09C878B87EE0FFF0BEC0DFD1D6081BF
:10346000718180918E1490918F140E9476910E94A8
:10347000C9A080918E1490918F14DC01ED91FC9184
:103480000680F781E02D19952CE83CE941E05527AD
:103490002BAB3CAB4DAB5EAB80918E1490918F14F7
:1034A0000E945A900E94BC6168E470E180918E1481
:1034B00090918F140E9476910E94BC616FE270E13E
:1034C00080918E1490918F140E94529120915D0CE6
:1034D00080918E1490918F14222319F06BE270E189
:1034E00002C066E270E10E94769180915D0C8823B3
:1034F00049F16DE070E180918E1490918F140E94DB
:1035000052916091231470912414072E000C880BA3
:10351000990B0E9441C820E030E04AE754E40E9441
:1035200046CAAB01BC0122E080918E1490918F14A9
:103530000E94749068E070E180918E1490918F14D5
:103540000E9476919EE4E92E93E1F92E29E2622E03
:103550003AE0232E312C44E6842E912CD7012C9175
:10356000222309F4FFC1F70132970081118101156F
:10357000110509F4F7C186EE9BE9A1E0BB27820F94
:10358000911DA11DB11DABBFFC01879177247394E0
:10359000811101C0712C20918E1430918F14C801BB
:1035A0000197849790F568EE7FE0C9010E945291DF
:1035B00009500C3148F4E02FF0E0EE0FFF1FEF5DF3
:1035C000FD4F6081718102C06EE37EE080918E14B8
:1035D00090918F140E9452910C3130F4E02FF0E062
:1035E000E75AFD4F808101C080E090E08252904F09
:1035F000092E000CAA0BBB0BABBFFC0187919EE010
:10360000981B892F09F053C154C1C80184569109F0
:103610008438934008F03FC06EEC7FE0C9010E94FF
:103620005291C801B4010E9479CB6130710531F02B
:103630006230710559F46AEC7FE002C06CEC7FE007
:1036400080918E1490918F140E9452910E94B461C7
:10365000A0908E14B0908F147720B1F0C8010E9412
:10366000D748811107C066EC7FE0C5010E945291E6
:1036700087E01DC1813009F01CC163EC7FE0C5010A
:103680000E94529188E013C16AEB7FE0C5010E945D
:10369000529182E00CC1C801885E93408035964407
:1036A00008F05CC0C80168EE73E00E9479CB5B0152
:1036B0006DEA7FE0C9010E945291FAE0AF16B104B1
:1036C00010F40E94AC61B50180918E1490918F141A
:1036D0000E9403840E94B46140908E1450908F1415
:1036E0007720B1F1C8010E94D748782E68EA7FE0C0
:1036F000C2010E945291672D80918E1490918F1477
:103700000E94518262EA7FE080918E1490918F1422
:103710000E94529128E13CEFA29EC001A39E900D11
:10372000B29E900D1124800F911FB1010E948DCB8C
:10373000772780918E1490918F140E94038460EA01
:103740007FE080918E1490918F140E945291B1C0AD
:1037500067E97FE0C2010E94529161C0F801E8531D
:10376000FA44E83E43E0F40708F046C0EC30F105C7
:1037700008F09FC08827EE58FF4F8F4F0C94A0CBC6
:1037800068E87FE019C06DE77FE0C9010E945291AF
:1037900083E18DC06BE67FE027C06BE57FE016C05C
:1037A0006EE47FE055C062E47FE0C9010E9452915F
:1037B00082E17DC063E37FE0C9010E9452918FE006
:1037C00076C064E27FE0F8CF64E17FE0C9010E9447
:1037D00052918EE06CC061E07FE0C9010E9452917D
:1037E0008BE065C06FEE7EE0C9010E9452918CE0D3
:1037F0005EC062EE7EE02CC0C80180529E44883ECE
:10380000934078F400526BEC7EE0C9010E94529123
:103810000A3010F40E94AC61802F0E946E6184E037
:1038200046C0C80188509245883E934020F4085015
:1038300064EB7EE0EACF013FB5E51B0719F463EACC
:103840007EE01CC0023FE5E51E0739F466E97EE034
:10385000C9010E94529181E12AC0033FF5E51F078B
:1038600039F468E87EE0C9010E94529180E11FC0EE
:10387000043F45E5140739F467E77EE0C9010E947B
:1038800052918DE014C0053F55E5150739F46FE5F9
:103890007EE0C9010E94529186E009C0063F1545AD
:1038A00041F466E47EE0C9010E94529185E00E94E5
:1038B00005A863E070E180918E1490918F140E94AE
:1038C000529168EF7FE080918E1490918F140E9446
:1038D0005291D7016C9170E080918E1490918F1469
:1038E0000E940384F70180818A3020F482E00E94E4
:1038F00005A804C0843610F40E94AC610E94B46133
:10390000D7014C91649EA0011124052E000C660B7A
:10391000770B8BA99CA9ADA9BEA9480F591F6A1F97
:103920007B1FD6018A019B010F5F1F4F2F4F3F4F17
:103930006BBFFA0187918D93B901A8018111F2CF74
:10394000B60180918E1490918F140E945D908091A9
:103950008E1490918F14DC01ED91FC910680F7811B
:10396000E02D1995B3E0EB0EF11CE6ECEE16E3E169
:10397000FE0609F0F3CD0E94C9A080918E149091AB
:103980008F14DC01ED91FC910680F781E02D1995F3
:1039900080918E1490918F140E945A900E94BC6165
:1039A00069EA70E180918E1490918F140E94769153
:1039B0000E94BC6166E970E180918E1490918F1431
:1039C0000E9452910E94954D20E030E040E050E48A
:1039D0000E943BC820918E1430918F1487FF3FC006
:1039E00063E970E1C90159C0F090F9130091FC132B
:1039F00011E00C94711265E37AE080918E1490913D
:103A00008F140E9452916091101580918E149091A4
:103A10008F140E94518263E37AE080918E1490911A
:103A20008F140E9452910C94FA126AEE79E0809100
:103A30008E1490918F140E94529160911215809172
:103A40008E1490918F140E94518268EE79E08091DB
:103A50008E1490918F140E9452910C9459136FE818
:103A600070E1C9010E9476916CE770E180918E143B
:103A700090918F140E9452910E94954DAB01BC0110
:103A800022E080918E1490918F140E9474906AE7C6
:103A900070E180918E1490918F140E94769167E668
:103AA00070E180918E1490918F140E9452918091B8
:103AB0006F140E947D6120916F1480918E149091FB
:103AC0008F14222379F064E670E10E9452910E94E3
:103AD00044A86AE570E180918E1490918F140E9441
:103AE000769102C00E945A900E94C9A080918E14C3
:103AF00090918F14DC01ED91FC910680F781E02D0F
:103B0000199580918E1490918F140E945A900E9462
:103B1000BC6161E071E180918E1490918F140E94DC
:103B200076910E94BC616DEE70E180918E1490914F
:103B30008F140E94529140915F14509160146091D3
:103B400061147091621480918E1490918F140E9470
:103B5000F08369ED70E180918E1490918F140E9432
:103B6000529140916714509168146091691470915A
:103B70006A1480918E1490918F140E94F08365ECEA
:103B800070E180918E1490918F140E945291409117
:103B9000631450916414609165147091661480915F
:103BA0008E1490918F140E94F08361EB70E18091EC
:103BB0008E1490918F140E94529140916B145091E9
:103BC0006C1460916D1470916E1480918E149091AC
:103BD0008F140E94F0830E94C9A080918E1490914E
:103BE0008F14DC01ED91FC910680F781E02D199591
:103BF00080918E1490918F140E945A900E94BC6103
:103C0000E6960FB6F894DEBF0FBECDBFDF91CF9121
:103C10001F910F91FF90EF90DF90CF90BF90AF90EA
:103C20009F908F907F906F905F904F903F902F90DC
:103C300008952F923F924F925F926F927F928F9250
:103C40009F92AF92BF92CF92DF92EF92FF920F932B
:103C50001F93CF93DF93CDB7DEB7AB970FB6F89432
:103C6000DEBF0FBECDBF8DED91E00E946CC9603FFD
:103C70007F4B8105910519F00E949C6B08C041EEB5
:103C800051E060E070E087EA92E10E9454C940E0B0
:103C900052EC61E070E081EF99E00E94CF7E4091AC
:103CA000631450916414609165147091661484E5F6
:103CB00099E00E94CF7E4091671450916814609102
:103CC000691470916A1487EB98E00E94CF7E40914E
:103CD0006B1450916C1460916D1470916E148AE1A4
:103CE00098E00E94CF7E87E19FE090931208809336
:103CF000110888ED9CE09093100880930F088AE0EB
:103D000080931D0F81EF99E090932A1580932915D8
:103D100010922B151092210F10921E0F1092200F4F
:103D200010921F0F11E01093A3140E94587B8091F2
:103D300083148093C807109290141092800082E040
:103D4000809381008FE286BB10926F0010928500F5
:103D5000109284009AEA9093A0001093A10089BB6E
:103D6000109272001092A5001092A4001092A90067
:103D70001092A8001092AB001092AA001092AD0011
:103D80001092AC0090932001109321018ABB1092F5
:103D900073001092250110922401109229011092B3
:103DA000280110922B0110922A0110922D011092DD
:103DB0002C01809144139091451380935D0790935B
:103DC0005E07813001F58FE38093800C1092810CA7
:103DD00061E00E94675886E79CE00E948AA71092E3
:103DE000820C1092850C1092840C80915E078823BF
:103DF00029F086E79CE00E94F2A711C086E79CE0CC
:103E00000E94CBA70CC080915E07882311F062E06E
:103E100001C060E08FE30E9467580E941E4E8091AF
:103E20004613909147138093630790936407813002
:103E300001F58EE38093B10C1092B20C61E00E9408
:103E4000675887EA9CE00E948AA71092B30C1092F0
:103E5000B60C1092B50C80916407882329F087EA8C
:103E60009CE00E94F2A711C087EA9CE00E94CBA7C9
:103E70000CC080916407882311F062E001C060E00B
:103E80008EE30E9467580E94EB4D60E085E40E943B
:103E9000675860E08DE30E94675862E08CE30E94FF
:103EA000675862E08BE30E94675862E080E40E94FA
:103EB000675862E081E40E94675862E082E40E94F1
:103EC000675862E081E20E94675862E084E40E94E1
:103ED000675861E082E20E94675861E083E20E94D5
:103EE00067580E94294C0E94604C61E085E30E9463
:103EF000675861E085E00E94675861E070E085E006
:103F00000E94A35861E084E00E94675861E08BE062
:103F10000E94675861E089E20E94EF5661E089E201
:103F20000E946758519A60E085E30E94EF5660E076
:103F300085E00E94EF5660E084E00E94EF5660E06A
:103F40008BE00E94EF56599861E08DE00E9467581F
:103F500080E090E09C0129553D4EF901E955FF4F65
:103F600040814F3629F4329720813181232B31F45F
:103F700003968837910571F760E001C061E08DE03C
:103F80000E94EF5661E08EE20E94675861E08DE288
:103F90000E94675861E086E00E94675861E087E010
:103FA0000E94675861E088E00E94675861E08BE2F8
:103FB0000E94675860E08BE20E94EF560E94604CBE
:103FC0000E9481838091660C813009F058C08091F5
:103FD000690C90916A0CA0916B0CB0916C0C4091A3
:103FE0006D0C50916E0C60916F0C7091700C841B75
:103FF000950BA60BB70B84379E40A105B10500F3C6
:104000000E949C6B0E94A6610E94A6610E94BC61F6
:104010006FE071E180918E1490918F140E94529103
:1040200001E010E00E942D4C0E94604C6EEE72E0A8
:1040300080E090E00E94EC5A6CE071E180918E1477
:1040400090918F140E9452910E94294C0E945C4CC6
:104050000530110531F064EF71E080E090E00E94DE
:10406000EC5A0F5F1F4F06301105E1F60E94A66162
:104070000E94BC610E94A6610E94A66102C08111DB
:104080009FCF80916F00826080936F008091840049
:10409000909185008056904F90938900809388007E
:1040A0000E94762C89ED9CE09093D10F8093D00FE5
:1040B00010911E1420911D1480910C1490910E14D7
:1040C00030910F143093170890932C0780932D078D
:1040D00030E0AFEFB0E00E94D2C924E630E040E02B
:1040E00050E00E9484C920931415612F70E080E095
:1040F00090E00E943FC820ED34E448E55BE30E9475
:10410000A0C826E636E646E25FE30E94E2C9609375
:104110001308709314088093150890931608109351
:1041200013151092950010929400109290008CE05C
:104130008093910084EF90E0909399008093980091
:1041400081E088BB82E080937100809100020E9430
:10415000F47A80912514863040F01092251460E0A6
:1041600070E08EE791E00E941283109125141230C6
:1041700009F444C008F5112309F466C0113009F0B0
:104180005BC08CE090E00E94B4CB2DE433E0DC0116
:1041900011963C932E9327EB38E01B963C932E937D
:1041A0001A979093C5078093C4071093211010931A
:1041B00024101093271067C0133009F45EC0143028
:1041C000D9F586E090E00E94B4CB8C0127EB33E078
:1041D000DC012D933D93CD0141E069ED7CE00E942F
:1041E000A46989E792E0F801918380831093C50761
:1041F0000093C40781E08093211041C086E090E0E5
:104200000E94B4CB23EE32E0FC01318320839093F3
:10421000C5078093C4078FB7F8942CED35E0309331
:10422000E7112093E6111092EC118FBF81E080938B
:1042300021108093241025C01092251460E070E0B6
:104240008EE791E00E94128386E090E00E94B4CB5A
:104250008C0127EB33E0DC012D933D93CD0140E051
:1042600069ED7CE00E94A46989E792E0F8019183FE
:1042700080831093C5070093C407109221101092F9
:104280002410109227108091C4079091C507DC017B
:10429000ED91FC910190F081E02D19958091151020
:1042A00081111FC08091181081111BC080911B10BB
:1042B000811117C080911E10811113C080912110AF
:1042C00081110FC08091241081110BC080912710A3
:1042D000811107C081E00E94547B882309F419C32F
:1042E00011C3A12CB12C912C1DA2412C512C612C5D
:1042F000712C812C01E716E0EE24EA94A3E0FA2E5B
:10430000CC24CA94DD24D39485E6282E86E0382E6A
:10431000C50189559D4EFC01E955FF4FE081EE2313
:1043200009F4E7C2DC01AB55BF4F8D919C91892BFD
:1043300009F4DFC28E2F90E0FC01F797EB32F10514
:1043400008F0D7C28827E258FF4F8F4F0C94A0CBBC
:1043500080911510882309F4CCC28110CAC289E16A
:1043600090E00E94B4CB9C01FC011183008387E0A4
:1043700090E09383828315821482F782E682D1864D
:10438000C086108EC9012AA73BA70E94A1422AA578
:104390003BA5E9E3F4E0D901ED93FC9330930610DB
:1043A00020930510C9010E948F947DC1809118103F
:1043B000882309F49EC271109CC289E190E00E949A
:1043C000B4CB9C01DC0111961C930E93E6E0F0E067
:1043D0001396FC93EE93129715961C921E921497C7
:1043E0001796FC92EE9216971996DC92CE92189739
:1043F00058961C922AA73BA70E94A1422AA53BA53A
:10440000E9E3F4E0D901ED93FC9330930810209395
:104410000710C9010E948F9474C180911B108823DA
:1044200009F467C2611065C289E190E00E94B4CBD3
:104430009C01DC0111961C930E93E5E0F0E01396CD
:10444000FC93EE93129715961C921E921497179652
:10445000FC92EE9216971996DC92CE921897589687
:104460001C922AA73BA70E94A1422AA53BA5E9E3EB
:10447000F4E0D901ED93FC9330930A1020930910D6
:10448000C9010E948F946BC180911E10882309F48A
:1044900030C251102EC289E190E00E94B4CB9C0141
:1044A000DC0111961C930E93E4E0F0E01396FC936C
:1044B000EE93129715961C921E9214971796FC92E3
:1044C000EE9216971996DC92CE92189758961C92F7
:1044D0002AA73BA70E94A1422AA53BA5E9E3F4E055
:1044E000D901ED93FC9330930C1020930B10C9016C
:1044F0000E948F9462C180912110882309F4F9C130
:104500004110F7C189E190E00E94B4CB9C01DC012D
:1045100011961C930E93E2E0F0E01396FC93EE9359
:10452000129715961C921E9214971796FC92EE9273
:1045300016971996DC92CE92189758961C922AA735
:104540003BA70E94A1422AA53BA5E9E3F4E0D901DB
:10455000ED93FC9330930E1020930D10C9010E942F
:104560008F9459C180912410882309F4C2C12DA1D0
:104570002111BFC189E190E00E94B4CB9C01DC0114
:1045800011961C930E93E1E0F0E01396FC93EE93EA
:10459000129715961C921E9214971796FC92EE9203
:1045A00016971996DC92CE92189758961C922AA7C5
:1045B0003BA70E94A1422AA53BA5E9E3F4E0D9016B
:1045C000ED93FC933093101020930F10C9010E94BB
:1045D0008F9459C180912710882309F48AC19110C2
:1045E00088C189E190E00E94B4CB9C01DC01119666
:1045F0001C930E9313961C921E92129715961C9262
:104600001E9214971796FC92EE9216971996DC92CA
:10461000CE92189758961C922AA73BA70E94A142B7
:104620002AA53BA589E394E0F90191838083309327
:10463000121020931110C9010E948F9458C18091CB
:104640001510882309F455C1811053C18CE190E005
:104650000E94B4CB9C01DC0111961C930E93E7E001
:10466000F0E01396FC93EE93129715961C921E920F
:1046700014971796FC92EE9216971996DC92CE92AA
:10468000189758961C922AA73BA70E94A1422AA5D8
:104690003BA5D9012D923C92309314102093131016
:1046A000C9010E946A958824839423C180911810BF
:1046B000882309F41EC171101CC18CE190E00E9496
:1046C000B4CB9C01FC011183008386E090E09383CE
:1046D000828315821482F782E682D186C086108E8C
:1046E000C9012AA73BA70E94A1422AA53BA5D9013F
:1046F0002D923C923093171020931610C9010E94FE
:104700006A9577247394F5C080911B10882309F46F
:10471000F0C06110EEC08CE190E00E94B4CB9C012F
:10472000FC011183008385E090E0938382831582EE
:104730001482F782E682D186C086108EC9012AA72C
:104740003BA70E94A1422AA53BA5D9012D923C92EC
:1047500030931A1020931910C9010E946A9566249B
:104760006394C7C080911E10882309F4C2C0511001
:10477000C0C08CE190E00E94B4CB9C01FC0111838D
:10478000008384E090E09383828315821482F78211
:10479000E682D186C086108EC9012AA73BA70E9457
:1047A000A1422AA53BA5D9012D923C9230931D1020
:1047B00020931C10C9010E946A955524539499C0F6
:1047C00080912110882309F494C0411092C08CE19B
:1047D00090E00E94B4CB9C01FC011183008382E035
:1047E00090E09383828315821482F782E682D186D9
:1047F000C086108EC9012AA73BA70E94A1422AA504
:104800003BA5D9012D923C923093201020931F108C
:10481000C9010E946A95442443946BC0809124107E
:10482000882309F466C02DA1211163C08CE190E0BA
:104830000E94B4CB9C01DC0111961C930E93E1E025
:10484000F0E01396FC93EE93129715961C921E922D
:1048500014971796FC92EE9216971996DC92CE92C8
:10486000189758961C922AA73BA70E94A1422AA5F6
:104870003BA5D9012D923C92309323102093221016
:10488000C9010E946A9521E02DA333C080912710B1
:10489000882379F191102DC08CE190E00E94B4CB77
:1048A0009C01DC0111961C930E9313961C921E9290
:1048B000129715961C921E9214971796FC92EE92E0
:1048C00016971996DC92CE92189758961C922AA7A2
:1048D0003BA70E94A1422AA53BA5F9013182208273
:1048E0003093261020932510C9010E946A959924BF
:1048F0009394F3E0AF0EB11C28E7A216B10409F0BF
:1049000007CDE8CC82E00E94547B882311F01FA2DF
:1049100016C081E00E94547B882329F082E00E9427
:10492000387B81119CC78CE30E945593892B09F039
:1049300087C78CE30E945593892B09F087C786E0CF
:10494000E5E5F4E1DE01549601900D928A95E1F7D8
:1049500080914E1490915E14B0904F1400915014B9
:104960001091511470915214609153145091541439
:1049700040915B1420915C1430915D14E091C40768
:10498000F091C507FEA3EDA3A091770FB091780F2A
:10499000B9A7A8A79090811460907C14E09075143A
:1049A000F090761480907F1470907E14C090DA138B
:1049B000D090DB135090DD134090D8133090D91372
:1049C000BFA1BB8B8A8F9B8FBC8E0D8F1E8F7F8F5D
:1049D00068A359A34AA33CA32BA3F2E1AF2EFE0187
:1049E0007396DE01119601900D92AA94E1F7E9ED1C
:1049F000FCE0F0933607E0933507EFA1E983888761
:104A00009987BA860B871C877D876E875F87488B5F
:104A10003A8B298B22E1FE013196A5E4B7E00190A3
:104A20000D922A95E1F7992321F0863011F010922A
:104A30004D073092E40F4092E50F50926B10D092E8
:104A40006410C09263106092790F70926810809227
:104A50006710F0926610E092651090926C1088A535
:104A600099A590936A10809369108DA19EA190934F
:104A70003807809337078BE08093120B1092130B4B
:104A800061E00E94675888E09BE00E948AA710922C
:104A9000140B1092170B1092160B80915007811176
:104AA00002C01092510790914C07911105C08111DD
:104AB00003C010924D0C98C08091480C9091490C05
:104AC0000E94D66581E080934D0C80914507882334
:104AD00059F1813071F08330C1F488E293E2909310
:104AE00047078093460789E080934A0780E197E271
:104AF00017C088EB9BE0909347078093460783E0BD
:104B000080934A0788E99AE30BC088E893E1909381
:104B100047078093460786E080934A0780EE9EE22F
:104B2000909349078093480780914C078823E9F1C7
:104B30008091500760914A0770E08823C9F0809106
:104B400052078823A9F080E090E00E943FC89B01B3
:104B5000AC0160E070E088EC92E40E9446CA609389
:104B6000390770933A0780933B0790933C0725C021
:104B700080E090E00E943FC89B01AC0160E070E0E3
:104B800088EC92E40E9446CA6093390770933A0712
:104B900080933B0790933C071092300710923107A7
:104BA00010923207109233071FC0109239071092EB
:104BB0003A0710923B0710923C0760914B0770E058
:104BC00080E090E00E943FC89B01AC0160E070E093
:104BD00088EC92E40E9446CA6093300770933107D4
:104BE00080933207909333071092A61210923D07DC
:104BF0001092340710923E0710923F071092400720
:104C0000109241070E9458565098589AE8988091FF
:104C100069008C7F809369008091E50F882321F0E3
:104C200080916900826003C08091690083608093F5
:104C30006900E8980E94455880E090E040E09C01BF
:104C400029553D4EF901E955FF4F5081552331F06B
:104C5000329720813181232B09F04F5F03968837EB
:104C6000910569F740935807A5E6B7E020E030E0EA
:104C700088EE282E80E6382E94EE492E9BE4592E9D
:104C80004EEE642E46E7742E51E0852E57E7952EA2
:104C90006BEEA62E60E6B62E45E05FE50BEE1EE558
:104CA00078EFE72E7EE5F72EE1E3CE2EEEE5DE2E61
:104CB000C90189559D4EFC01E955FF4F608166236E
:104CC00009F4B0C38B559F4FFC0180819181892BE2
:104CD00009F4A8C370E0FB013197E53AF10508F04B
:104CE000A1C38827E755FF4F8F4F0C94A0CB80EDD1
:104CF00098E411969C938E9395C38EEC98E411964C
:104D00009C938E938FC38CEC98E411969C938E9316
:104D100089C384EC98E411969C938E9383C381ECB1
:104D200098E411969C938E937DC382ED97E411963F
:104D30009C938E9377C389E398E411969C938E930A
:104D400071C385EB97E411969C938E936BC382EAB3
:104D500097E411969C938E9365C383E997E411962B
:104D60009C938E935FC38BE397E411969C938E93F1
:104D700059C38BEF95E411969C938E9353C38FE2A6
:104D800097E411969C938E934DC382EC96E4119612
:104D90009C938E9347C384E297E411969C938E93E1
:104DA00041C38DE297E411969C938E933BC386E2B8
:104DB00097E411969C938E9335C38DEE96E41196ED
:104DC0009C938E932FC385E197E411969C938E93C9
:104DD00029C38EE097E411969C938E9323C38FEDA5
:104DE00096E411969C938E931DC38EED96E41196D6
:104DF0009C938E9317C38DED96E411969C938E939E
:104E000011C38FEC96E411969C938E930BC38EEC9A
:104E100096E411969C938E9305C381EC96E41196CB
:104E20009C938E93FFC283EB96E411969C938E9392
:104E3000F9C282EB96E411969C938E93F3C281EBB8
:104E400096E411969C938E93EDC28FEC94E41196A8
:104E50009C938E93E7C28EEC94E411969C938E9370
:104E6000E1C28DEC94E411969C938E93DBC281E8B1
:104E70009AE411969C938E93D5C280EB96E411969A
:104E80009C938E93CFC282EA96E411969C938E9364
:104E9000C9C286E695E411969C938E93C3C289E4B9
:104EA00095E411969C938E93BDC281EA96E4119687
:104EB0009C938E93B7C286E796E411969C938E934B
:104EC000B1C28FE696E411969C938E93ABC280E4B8
:104ED00096E411969C938E93A5C289E19FE9119661
:104EE0009C938E939FC289EF95E411969C938E9329
:104EF00099C287EF95E411969C938E9393C284EFA9
:104F000095E411969C938E938DC280ED95E4119655
:104F10009C938E9387C281E599E411969C938E931E
:104F200081C281EF95E411969C938E937BC28DECA8
:104F300095E411969C938E9375C28FE499E4119633
:104F40009C938E936FC28EEE95E411969C938E93F4
:104F500069C28AEC95E411969C938E9363C28DE4AA
:104F600099E411969C938E935DC28BEE95E4119615
:104F70009C938E9357C287EC95E411969C938E93E5
:104F800051C28BE499E411969C938E934BC288EEA8
:104F900095E411969C938E9345C284EC95E411960A
:104FA0009C938E933FC289E499E411969C938E93CF
:104FB00039C285EE95E411969C938E9333C281ECB1
:104FC00095E411969C938E932DC287E499E41196F3
:104FD0009C938E9327C282EE95E411969C938E93B8
:104FE00021C28EEB95E411969C938E931BC285E4AF
:104FF00099E411969C938E9315C28FED95E41196CA
:105000009C938E930FC28BEB95E411969C938E9399
:1050100009C283E499E411969C938E9303C28CEDAC
:1050200095E411969C938E93FDC188EB95E41196BF
:105030009C938E93F7C181E499E411969C938E938F
:10504000F1C189ED95E411969C938E93EBC185EBAC
:1050500095E411969C938E93E5C18FE399E41196A4
:105060009C938E93DFC186ED95E411969C938E936D
:10507000D9C182EB95E411969C938E93D3C18DE3B5
:1050800099E411969C938E93CDC183ED95E411968E
:105090009C938E93C7C18FEA95E411969C938E934F
:1050A000C1C18BE399E411969C938E93BBC18DEDA6
:1050B00094E411969C938E93B5C186E398E411967F
:1050C0009C938E93AFC183E398E411969C938E9347
:1050D000A9C180E398E411969C938E93A3C18DE2BD
:1050E00098E411969C938E939DC18AE298E4119660
:1050F0009C938E9397C187E298E411969C938E932C
:1051000091C184E298E411969C938E938BC181E2C5
:1051100098E411969C938E9385C188EA95E4119644
:105120009C938E937FC18CEC94E411969C938E9308
:1051300079C18BEC94E411969C938E9373C183E8B0
:1051400095E411969C938E936DC187EF94E411962C
:105150009C938E9367C185E691E611969C938E93FE
:1051600061C188ED9EE511969C938E935BC186ED9F
:105170009EE511969C938E9355C18FE391E611960F
:105180009C938E934FC18DEE90E611969C938E93D7
:1051900049C180EF9FE511969C938E9343C185EAA8
:1051A0009FE511969C938E933DC181E497E71196FC
:1051B0009C938E9337C18DE297E711969C938E93C3
:1051C00031C189E197E711969C938E932BC182E6BA
:1051D0009FE911969C938E9325C188EB90E61196DA
:1051E0009C938E931FC18BEA90E611969C938E93AD
:1051F00019C185E990E611969C938E9313C183E7BC
:1052000090E611969C938E930DC183E990E61196DA
:105210009C938E9307C185E790E611969C938E939D
:1052200001C18FE19EE511969C938E93FBC085EDA5
:105230009DE511969C938E93F5C087EF9DE51196A1
:105240009C938E93EFC087EE9DE511969C938E9371
:10525000E9C089E09EE511969C938E93E3C08DEAA8
:105260009DE511969C938E93DDC08DE99DE5119689
:105270009C938E93D7C08FEB9DE511969C938E9354
:10528000D1C089E99FE511969C938E93CBC08DE8A0
:105290009FE511969C938E93C5C081E89FE511967A
:1052A0009C938E93BFC085E79FE511969C938E9348
:1052B000B9C089E69FE511969C938E93B3C08DE5A6
:1052C0009FE511969C938E93ADC081E59FE5119665
:1052D0009C938E93A7C08DE99EE511969C938E9327
:1052E000A1C08BE89EE511969C938E939BC089E7A5
:1052F0009EE511969C938E9395C087E69EE5119648
:105300009C938E938FC085E59EE511969C938E931A
:1053100089C083E49EE511969C938E9383C0119679
:10532000DC92CE927FC01196FC92EE927BC01196D9
:105330001C930E9377C08BE29FE511969C938E93FE
:1053400071C011965C934E936DC01196BC92AE9253
:1053500069C011969C928E9265C011967C926E9255
:1053600061C011965C924E925DC011963C922E9255
:1053700059C0E5EEF0E61196FC93EE9353C08CED28
:1053800090E611969C938E934DC0E9EDF0E6119650
:10539000FC93EE9347C086ED90E611969C938E9316
:1053A00041C0E3EDF0E61196FC93EE933BC080ED37
:1053B00090E611969C938E9335C0E5ECF0E611963D
:1053C000FC93EE932FC08EEC90E611969C938E93F7
:1053D00029C0E7ECF0E61196FC93EE9323C089EC2C
:1053E0009EE511969C938E931DC0ECEBFEE5119605
:1053F000FC93EE9317C08FEA9EE511969C938E93D3
:1054000011C0EEE4F0E61196FC93EE930BC08BE333
:1054100090E611969C938E9305C0E1E6F0E6119616
:10542000FC93EE932D5F3F4F12962837310509F01C
:105430003FCC1092590780915D07811114C080E024
:1054400090E0FC01E45BFC4E20813181245631095F
:105450002436310528F003968837910591F703C06B
:1054600081E08093590710925F0780916307811153
:1054700014C080E090E0FC01E45BFC4E20813181AF
:10548000285C31092436310528F0039688379105C8
:1054900091F703C081E080935F078091C4079091EA
:1054A000C507DC01ED91FC91EE5AFF4F20912814C5
:1054B0003091291440912614509127140190F081C5
:1054C000E02D61E019958091C4079091C507DC013A
:1054D000ED91FC91EE5AFF4F20912C1430912D1438
:1054E00040912A1450912B140190F081E02D62E03C
:1054F00019958091C4079091C507DC01ED91FC914D
:10550000EE5AFF4F209130143091311440912E14F7
:1055100050912F140190F081E02D63E01995809156
:10552000C4079091C507DC01ED91FC91EE5AFF4F45
:1055300020913B1430913C144091391450913A140D
:105540000190F081E02D64E019958091C40790915D
:10555000C507DC01ED91FC91EE5AFF4F20913F14FD
:105560003091401440913D1450913E140190F081CF
:10557000E02D65E019958091C4079091C507DC0185
:10558000ED91FC91EE5AFF4F209143143091441459
:1055900040914114509142140190F081E02D66E059
:1055A00019958091C4079091C507DC01ED91FC919C
:1055B000EC5AFF4F0190F081E02D4091321461E0F0
:1055C00019958091C4079091C507DC01ED91FC917C
:1055D000EC5AFF4F0190F081E02D4091331462E0CE
:1055E00019958091C4079091C507DC01ED91FC915C
:1055F000EC5AFF4F0190F081E02D4091341463E0AC
:1056000019958091C4079091C507DC01ED91FC913B
:10561000EC5AFF4F0190F081E02D4091451464E079
:1056200019958091C4079091C507DC01ED91FC911B
:10563000EC5AFF4F0190F081E02D4091461465E057
:1056400019958091C4079091C507DC01ED91FC91FB
:10565000EC5AFF4F0190F081E02D4091471466E035
:1056600019958091C4079091C507DC01ED91FC91DB
:1056700002ACF3ADE02D6091361419958091C4070A
:105680009091C507DC01ED91FC9106ACF7ADE02DE2
:1056900060914B1419958091C4079091C507DC0166
:1056A000ED91FC9100A8F1A9E02D609137141995B6
:1056B0008091C4079091C507DC01ED91FC9106A88B
:1056C000F7A9E02D6091381419958091C407909145
:1056D000C507DC01ED91FC91E65BFF4F0190F08185
:1056E000E02D40914C1460E019958091C407909191
:1056F000C507DC01ED91FC91E65BFF4F0190F08165
:10570000E02D40914D1461E0199580E090E09C01FE
:1057100029553D4EF901E955FF4F4081423731F49B
:10572000329720813181232B09F09FC0039688375F
:10573000910569F70E94CD9F8091C4079091C5079C
:10574000DC01ED91FC91EC59FF4F0190F081E02DCF
:1057500040E06091481419958091C4079091C50765
:10576000DC01ED91FC91EC59FF4F0190F081E02DAF
:1057700041E060914A1419958091C4079091C50742
:10578000DC01ED91FC91EC59FF4F0190F081E02D8F
:1057900042E06091491419952091731430E0AFEF05
:1057A000B0E00E94D2C924E630E040E050E00E9420
:1057B00084C92093830F8091721481110E94B94C87
:1057C0000E9473A80E94245B6B017C0110E0111100
:1057D0000FC08091C807882359F02AED3EE540EDBF
:1057E00057E060E070E089ED9CE00E94E63F11E048
:1057F0000E949E97882351F00E94D34C0E94A54E90
:105800000E94604C0E942B970E94F04B0E94AA506D
:10581000029711F00E9454540E94C9A00E94AA50FD
:105820000297A9F60E94245BDC01CB018C199D092B
:10583000AE09BF098C3B9240A105B10540F218C0EA
:1058400082E00E94547B81110DC073C882E00E94E7
:10585000387B882309F473C8A3E0AFA370C881E044
:105860008FA36DC892E09FA36AC80E94C19F64CFB6
:105870000E947A760E94604C8091610C811102C076
:105880000E9493840E947D5086E30E94A85ABC0126
:10589000990F880B990B611571058105910511F020
:1058A0000E94BCC728E93DE548EE53E060E070E0A7
:1058B00089ED9CE00E94E63FAB960FB6F894DEBF00
:1058C0000FBECDBFDF91CF911F910F91FF90EF9051
:1058D000DF90CF90BF90AF909F908F907F906F9010
:1058E0005F904F903F902F900C94DA615F926F928F
:1058F0007F928F929F92AF92BF92CF92DF92EF9260
:10590000FF920F931F93CF93DF9381E08093151045
:105910008093181080931B1080931E1080932A1080
:1059200080932D10809319088093180890910F147C
:105930009150963040F080930F1461E070E088E65B
:1059400091E00E94128390910F142DEF290F809106
:10595000C413233008F058C28A3089F03CF48830F0
:1059600009F465C0893009F407C2FDC18C3009F41F
:1059700030C10CF4A4C0803109F4E6C0F4C184E263
:1059800090E00E94B4CBFC018091821428E030E0CA
:10599000338322838824839499249A9495828482E1
:1059A000AA24AA94B12CB782A68211861086108EE2
:1059B00053E8752E718E67EBC62E68E0D62ED38E17
:1059C000C28E75E7E72E74E0F72EF182E082C7E61B
:1059D000D4E1D1A3C0A312A283A3F093BB07E093A9
:1059E000BA07CF010E945D8884E290E00E94B4CBA8
:1059F000FC018091821429E030E033832283958278
:105A00008482B782A68211861086108E718ED38E04
:105A1000C28EF182E082D1A3C0A312A283A3F0932D
:105A2000B907E093B807CF010E945D888FC380E279
:105A300090E00E94B4CBFC0188E090E093838283E5
:105A40008824839499249A9495828482AA24AA947F
:105A5000B12CB782A68211861086108E9AE0D92EBC
:105A6000D18E27EBE22E28E0F22EF38EE28ECDE5EA
:105A7000D4E0D183C083F093BB07E093BA07CF0192
:105A80000E94E78680E290E00E94B4CBFC0189E0AE
:105A900090E09383828395828482B782A682118666
:105AA0001086108ED18EF38EE28ED183C083F09358
:105AB000B907E093B807CF010E94E78647C389E1A1
:105AC00090E00E94B4CBFC0188E090E09383828355
:105AD000CC24C394DD24DA94D582C482EE24EA94E3
:105AE000F12CF782E68211861086108EC1E5D4E093
:105AF000D183C083F093BB07E093BA07CF010E9424
:105B0000D29510922A1080910F14843009F01EC390
:105B100089E190E00E94B4CBFC0189E090E093839E
:105B20008283D582C482F782E68211861086108E27
:105B3000D183C083F093B907E093B807CF010E94E7
:105B4000D29510922D1002C389E190E00E94B4CB4F
:105B5000FC0188E090E093838283CC24C394DD240D
:105B6000DA94D582C482EE24EA94F12CF782E6829C
:105B700011861086108EC5E4D4E0D183C083F093E3
:105B8000BB07E093BA07CF010E94949510921908C1
:105B900080910F14843009F0D9C289E190E00E940D
:105BA000B4CBFC0189E090E093838283D582C482E8
:105BB000F782E68211861086108ED183C083F0931F
:105BC000B907E093B807CF010E9494951092180886
:105BD000BDC2943009F04BC089E190E00E94B4CB83
:105BE000EC0131E7832E36E0932E9982888287E09C
:105BF00090E09B838A83AA24A394BB24BA94BD8299
:105C0000AC82CC24CA94D12CDF82CE82198618862D
:105C1000188ECE010E94A14269E3E62E64E0F62EC2
:105C2000F982E882D093BB07C093BA07CE010E94E5
:105C30008F941092151089E190E00E94B4CBEC0192
:105C40009982888286E090E09B838A83BD82AC82C1
:105C5000DF82CE8219861886188ECE010E94A1425C
:105C6000F982E882D093B907C093B8074DC0953048
:105C700009F050C089E190E00E94B4CBEC01B1E79B
:105C80008B2EB6E09B2E9982888287E090E09B83E2
:105C90008A83AA24A394BB24BA94BD82AC82CC2468
:105CA000CA94D12CDF82CE8219861886188ECE0136
:105CB0000E94A14229E3E22E24E0F22EF982E8823A
:105CC000D093B907C093B807CE010E948F94109269
:105CD000151089E190E00E94B4CBEC019982888292
:105CE00086E090E09B838A83BD82AC82DF82CE8295
:105CF00019861886188ECE010E94A142F982E88288
:105D0000D093BB07C093BA07CE010E948F94109224
:105D100018101CC289E190E00E94B4CBEC0181E72D
:105D200096E09983888387E090E09B838A8381E073
:105D30009FEF9D838C838FEF90E09F838E831986E6
:105D40001886188ECE010E94A14289E394E09983BF
:105D50008883D093BB07C093BA07CE010E948F946B
:105D600010921510F3C189E08093C41369E070E0CC
:105D70008DE191E00E94128380E290E00E94B4CB1A
:105D8000FC0188E090E093838283882483949924A3
:105D90009A9495828482AA24AA94B12CB782A6826E
:105DA00011861086108E70E8D72ED18EA7EBEA2EC2
:105DB000A8E0FA2EF38EE28EC9E6D4E0D183C08348
:105DC000F093BB07E093BA07CF010E94988780E267
:105DD00090E00E94B4CBFC0189E090E09383828341
:105DE00095828482B782A68211861086108ED18E0B
:105DF000F38EE28ED183C083F093B907E093B807A6
:105E0000CF010E949887A2C18A3009F44AC03CF4AD
:105E1000883009F494C0893009F441C137C18C300D
:105E200009F4EAC00CF4AEC0803109F02FC189E159
:105E300090E00E94B4CBFC0188E090E093838283E1
:105E4000CC24C394DD24DA94D582C482EE24EA946F
:105E5000F12CF782E68211861086108EC5E4D4E01C
:105E6000D183C083F093BD07E093BC0789E190E044
:105E70000E94B4CBFC0189E090E093838283D582B9
:105E8000C482F782E68211861086108ED183C08389
:105E9000F093BF07E093BE071092190810921808FC
:105EA0003FC184E290E00E94B4CBFC017090821468
:105EB00060901B1488E090E093838283882483940D
:105EC00099249A9495828482AA24AA94B12CB782A8
:105ED000A68211861086108E23E8522E518E37EB43
:105EE000C32E38E0D32ED38EC28E45E7E42E44E095
:105EF000F42EF182E082C7E6D4E1D1A3C0A362A26E
:105F000073A2F093BD07E093BC0784E290E00E9487
:105F1000B4CBFC0189E090E09383828395828482F4
:105F2000B782A68211861086108E518ED38EC28EB5
:105F3000F182E082D1A3C0A362A273A2EDC080E28D
:105F400090E00E94B4CBFC0188E090E093838283D0
:105F50008824839499249A9495828482AA24AA946A
:105F6000B12CB782A68211861086108ECAE0DC2E74
:105F7000D18ED7EBED2ED8E0FD2EF38EE28ECDE55F
:105F8000D4E0AFC089E190E00E94B4CBFC0188E08E
:105F900090E093838283CC24C394DD24DA94D58269
:105FA000C482EE24EA94F12CF782E68211861086F0
:105FB000108EC1E5D4E0D183C083F093BD07E09398
:105FC000BC0789E190E00E94B4CBFC0189E090E03D
:105FD00093838283D582C482F782E68211861086FB
:105FE000108ED183C083F093BF07E093BE07109259
:105FF0002A1010922D1094C089E190E00E94B4CB39
:10600000EC0181E7882E86E0982E9982888287E0CD
:1060100090E09B838A83AA24A394BB24BA94BD8274
:10602000AC82CC24CA94D12CDF82CE821986188609
:10603000188ECE010E94A14239E3E32E34E0F32E04
:10604000F982E882D093BD07C093BC0789E190E054
:106050000E94B4CBEC019982888286E090E09B8319
:106060008A83BD82AC82DF82CE8219861886188E22
:10607000CE010E94A142F982E882D093BF07C0936B
:10608000BE0710921510109218104AC089E0809334
:10609000C41369E070E08DE191E00E94128380E218
:1060A00090E00E94B4CBFC0188E090E0938382836F
:1060B0008824839499249A9495828482AA24AA9409
:1060C000B12CB782A68211861086108EA0E8DA2E37
:1060D000D18EB7EBEB2EB8E0FB2EF38EE28EC9E645
:1060E000D4E0D183C083F093BD07E093BC0780E286
:1060F00090E00E94B4CBFC0189E090E0938382831E
:1061000095828482B782A68211861086108ED18EE7
:10611000F38EE28ED183C083F093BF07E093BE0776
:106120008091BE079091BF07DC01ED91FC91028048
:10613000F381E02D19958091BC079091BD07DC019A
:10614000ED91FC910280F381E02D199580910F145F
:10615000833039F0823009F06CC08091C4138C30E8
:1061600051F189E190E00E94B4CBEC0181E796E027
:106170009983888386E090E09B838A8381E09FEF08
:106180009D838C838FEF90E09F838E831986188682
:10619000188ECE010E94A14289E394E099838883FE
:1061A000D093B607C093B507CE010E948F9410928A
:1061B0001810C6E029C089E190E00E94B4CBEC0140
:1061C00081E796E09983888384E090E09B838A83CB
:1061D00081E09FEF9D838C838FEF90E09F838E8380
:1061E00019861886188ECE010E94A14289E394E098
:1061F00099838883D093B607C093B507CE010E94D8
:106200008F9410921E10C4E06091D3137091D41338
:106210008C2F0E94BA416091D5137091D6138C2FA8
:106220000E94B6418091D713E091B507F091B6076F
:10623000808FE091C5138E2FEE0F990BAA0BBB0B2D
:10624000FC013897E830F10508F0BBC08827E25B15
:10625000FE4F8F4F0C94A0CB84E290E00E94B4CB11
:10626000FC018091821428E030E03383228321E016
:106270003FEF358324832FEF30E037832683118669
:106280001086108E94E8918F27EB38E0338F228FA1
:1062900025E734E03183208327E634E131A320A3CE
:1062A00012A283A31EC080E290E00E94B4CBFC0146
:1062B00088E090E09383828381E09FEF95838483DD
:1062C0008FEF90E09783868311861086108E87E883
:1062D000818F87EB98E0938F828F89E694E091839A
:1062E0008083F093C307E093C20799C080E290E0F7
:1062F0000E94B4CBFC0188E090E09383828381E02C
:106300009FEF958384838FEF90E097838683118638
:106310001086108E8DE0818F87EB98E0938F828FAF
:106320008DE594E0DCCF89E190E00E94B4CBFC01E4
:1063300088E090E09383828381E09FEF958384835C
:106340008FEF90E09783868311861086108E81E50B
:1063500094E091838083F093C307E093C207109287
:106360002A105DC08CE190E00E94B4CBEC0181E783
:1063700096E09983888385E090E09B838A8381E01F
:106380009FEF9D838C838FEF90E09F838E83198690
:106390001886188ECE010E94A14285E696E037C08D
:1063A00089E190E00E94B4CBFC0113821282158235
:1063B00014821782168211861086108E81E294E074
:1063C0008ECF8CE08093C5136CE070E08EE191E09D
:1063D0000E94128389E190E00E94B4CBEC0181E736
:1063E00096E09983888385E090E09B838A8381E0AF
:1063F0009FEF9D838C838FEF90E09F838E83198620
:106400001886188ECE010E94A14289E394E09983F8
:106410008883D093C307C093C20710921B1080914A
:10642000C2079091C307DC01ED91FC910280F381DA
:10643000E02D19958091CD13843658F4853608F0F7
:1064400084E664E6681B8091C2079091C3070E94AE
:10645000F0888091C5138C508230A8F46091CE13DF
:106460007091CF1385E00E94EC406091D013709141
:10647000D11385E00E94D1408091D213E091C207F0
:10648000F091C307808F2091C613822F022E000C3B
:10649000990BAA0BBB0BFC013897E830F10508F00B
:1064A00089C08827EA5AFE4F8F4F0C94A0CB84E214
:1064B00090E00E94B4CBFC018091821429E030E08E
:1064C0003383228321E03FEF358324832FEF30E0B5
:1064D0003783268311861086108E94E8918F27EBE0
:1064E00038E0338F228F25E734E03183208327E69D
:1064F00034E131A320A312A283A357C080E290E02D
:106500000E94B4CBFC0189E090E09383828381E018
:106510009FEF958384838FEF90E097838683118626
:106520001086108E87E8818F87EB98E0938F828F9B
:1065300089E694E038C080E290E00E94B4CBFC0190
:1065400089E090E09383828381E09FEF9583848349
:106550008FEF90E09783868311861086108E8DE0F2
:10656000818F87EB98E0938F828F8DE594E01BC03D
:1065700080910F14823009F0C9C28091C4138C300D
:1065800009F0C4C21FC089E190E00E94B4CBFC01B5
:106590001382128215821482178216821186108647
:1065A000108E81E294E091838083F093C707E0939B
:1065B000C6075EC080910F14823061F58091C413CC
:1065C0008C3041F58BE08093C6136BE070E08FE177
:1065D00091E00E94128389E190E00E94B4CBFC011B
:1065E00089E090E09383828381E09FEF95838483A9
:1065F0008FEF90E09783868311861086108E81E559
:1066000094E091838083F093C707E093C6071092CC
:106610002D102EC08CE08093C6136CE070E08FE1EB
:1066200091E00E94128389E190E00E94B4CBEC01DA
:1066300081E796E09983888384E090E09B838A8356
:1066400081E09FEF9D838C838FEF90E09F838E830B
:1066500019861886188ECE010E94A14289E394E023
:1066600099838883D093C707C093C60710921E10E2
:106670008091C6079091C707DC01ED91FC910280E3
:10668000F381E02D19958091CC13843658F485362A
:1066900008F084E664E6681B8091C6079091C707FE
:1066A0000E94F0888091C6138C50823000F5609172
:1066B000C7137091C81384E00E94EC406091C91325
:1066C0007091CA1384E00E94D1408091CB13E09175
:1066D000C607F091C707808F8091C6138D3039F4BB
:1066E0008091CB13E0919A10F0919B10808F8EE1F6
:1066F00090E00E94B4CBEC01D090DC13A090E013AA
:10670000B090E1138090DE139090DF1381E796E064
:106710009983888383E090E09B838A8381E09FEF65
:106720009D838C83EE24EA94F12CFF82EE821986FD
:106730001886188ECE010E94A1428DE294E09983C2
:1067400088839A8E898EBC8EAB8EDD8ED093780F27
:10675000C093770F6091E2137091E31383E00E947E
:10676000EC406091E4137091E51383E00E94D14006
:106770008091DC13E091770FF091780F808F8091FA
:10678000DC130E94DD828091770F9091780FDC01FD
:10679000ED91FC910280F381E02D19958091E71332
:1067A0008823A1F18BE390E00E94B4CBFC0180919F
:1067B000F1139091F0132091F6133091F71340915B
:1067C000F4135091F5136091F2137091F313A091AB
:1067D000EC13B091ED13C091EA13D091EB13C0907C
:1067E000E813D090E91311821082F382E2821582BD
:1067F0001482D4A2C3A2D6A3C5A3B0A7A7A372A78D
:1068000061A754A743A736A725A72FC08BE390E025
:106810000E94B4CBFC018091F1139091F013209170
:10682000F6133091F7134091F4135091F5136091E2
:10683000F2137091F313A091EA13B091EB13C0918E
:10684000E813D091E91311821082F382E28215825B
:106850001482D4A3C3A3B6A3A5A370A767A352A70A
:1068600041A734A723A7F6A6E5A627EB38E030AB6F
:1068700027A727E634E132AB21AB93AB84ABF0938F
:106880004407E0934307C0914307D09144072FA1E9
:1068900038A54BA15CA18DA19EA1421753071CF402
:1068A000821793077CF0281739071CF448175907FB
:1068B00064F0241735075CF48417950744F4142F0B
:1068C000052F05C0122F032F02C0182F092F1F827A
:1068D0001E82188709871B861A861D861C861E87BE
:1068E0000F87198A188A2DA53EA549A55AA58BA5FB
:1068F0009CA5421753071CF4821793077CF02817B6
:1069000039071CF44817590764F0241735075CF45D
:106910008417950744F4142F052F05C0122F032F59
:1069200002C0182F092F1B8A1A8A1C8B0D8B1F8AF5
:106930001E8A198E188E1A8F0B8F1D8E1C8E1AAE02
:1069400019AE18A28BA9813069F08230E9F081116B
:1069500083C061E088E00E9467581092AD001092F9
:10696000AC007AC061E088E00E9467581092AD00E8
:106970001092AC0061E08DE00E94675860E070E02A
:106980008DE00E94A35868C0E9A9FAA9808191818D
:10699000A281B38181159649A105B10509F457C0BB
:1069A00040E056E960E070E08FA598A90E94CF7E94
:1069B00064E170E080E090E00E94EC5AE9A9FAA955
:1069C00080819181A281B38181152BE49207A10579
:1069D000B105E9F068F4803629E09207A105B10518
:1069E000A1F080389542A105B105C1F442E012C082
:1069F000811521EE9207A105B10559F08115924C40
:106A0000A140B10559F445E005C041E003C043E0B1
:106A100001C046E06FE0CE010E94543D8FA598A9C9
:106A2000DC01ED91FC910680F781E02D1995E9A933
:106A3000FAA940815181628173818FA598A90E9432
:106A4000CF7E64E170E080E090E00E94EC5A4AE082
:106A50006EE0CE010E94543D8091F11380930E08A8
:106A600080912A108823F9F089E190E00E94B4CB4C
:106A7000FC0188E090E093838283158214828FEF7B
:106A800093E0978386838FEF91E091878087108EC4
:106A900081E594E091838083F0932910E09328109E
:106AA000CF010E94D29580912D10882309F478C0DF
:106AB00089E190E00E94B4CBFC0189E090E09383EF
:106AC0008283158214828FEF93E0978386838FEF02
:106AD00091E091878087108E81E594E09183808397
:106AE000F0932C10E0932B10CF01DF91CF911F91E9
:106AF0000F91FF90EF90DF90CF90BF90AF909F905D
:106B00008F907F906F905F900C94D2952C3009F409
:106B10008ACD8CE190E00E94B4CBEC0191E7692E24
:106B200096E0792E7982688224E0822E912C9B82D5
:106B30008A82AA24A394BB24BA94BD82AC82CC24BA
:106B4000CA94D12CDF82CE8219861886188ECE0187
:106B50000E94A14255E6E52E56E0F52EF982E88224
:106B6000D093C707C093C6078CE190E00E94B4CBD6
:106B7000EC01798268829B828A82BD82AC82DF824C
:106B8000CE8219861886188E0E94A142F982E88268
:106B9000D0939B10C0939A10CE010E946A9566CD47
:106BA000DF91CF911F910F91FF90EF90DF90CF90E9
:106BB000BF90AF909F908F907F906F905F9008955F
:106BC0002F923F924F925F926F927F928F929F92FD
:106BD000AF92BF92CF92DF92EF92FF920F931F93EB
:106BE000CF93DF93CDB7DEB7CE5AD1090FB6F89465
:106BF000DEBF0FBECDBFCDB6DEB6C455DF4F1882A7
:106C0000CC5AD040C555DF4F1882CB5AD040809126
:106C1000220F8B3709F4E8C180F4873709F4D7C213
:106C200038F48F3109F440C5863709F4E0C102C653
:106C30008937B9F008F4DAC234C0803809F472C474
:106C400038F48C3709F4E1C28E3709F42DC3F2C54C
:106C5000823809F408C508F418C5833809F4E6C475
:106C6000E9C50E94B4440E94245B2B013C010E94B0
:106C7000AA50029709F423C50E94245BDC01CB01D2
:106C800084199509A609B70980329340A105B10579
:106C900008F015C50E9454540E94B4440E94CCA32D
:106CA000E6CF0E94AA50029729F060E084E80E9493
:106CB0007DA48BC18091620C823031F0833039F435
:106CC00082E080939B0F03C081E08093520F81E0AC
:106CD00080932C0F8E0104551F4F2FE0AE014057BB
:106CE0005F4F68E871E90E9409A40E947D508930D5
:106CF00058F0015011092FE0AE014F575F4F68E87F
:106D000072E981E00E9409A410922B0F77247394FA
:106D10000E949350882309F43DC1198222961FAE28
:106D2000229710912B0F11110EC0BE0160577F4F9B
:106D3000CE018F5B9F4F0E94D2CDC455DF4F08819B
:106D4000CC5AD04011C0113071F4BE016F577F4F43
:106D5000CE018F5B9F4F0E94D2CDC555DF4F08817A
:106D6000CB5AD04001C000E0ADB6BEB680915E0CFB
:106D7000EDB7FEB722E0829FE019F10911240FB6AA
:106D8000F894FEBF0FBEEDBF8DB79EB701967C0194
:106D900064ED76E0CE018B559F4F0E94DA8F809193
:106DA000620C823089F0833061F1813009F0A1C03A
:106DB00040915E0C50E0B7018091D90F9091DA0FAD
:106DC0000E94C1A210E039C020915E0C30E05FB794
:106DD000F89440E0842F90E08217930774F4880FB2
:106DE000991FF701E80FF91FDC01AF5CB04F8D91DF
:106DF0009C91918380834F5FEDCF5FBF1092510FC5
:106E00001CC020915E0C30E05FB7F89440E0842F06
:106E100090E08217930774F4880F991FF701E80F29
:106E2000F91FDC01AC54B04F8D919C91918380830C
:106E30004F5FEDCF5FBF1092D60F6DE270E0CE01D5
:106E40008B559F4F0E94DD8E20915E0C293048F0BB
:106E5000112321F0113021F418E004C028E001C012
:106E600020E010E0121758F5F701E10FF11DE10FD6
:106E7000F11D608171814AE0CE0181569F4FC3555B
:106E8000DF4F2883CD5AD0400E94838FBE016156C8
:106E90007F4FCE018B559F4F0E94048FCE018156AC
:106EA0009F4F0E947E8FCE018B559F4F0E9404A55D
:106EB0001F5FC355DF4F2881CD5AD040D3CF40E468
:106EC00050E0BE016F5F7F4FCE018B559F4F0E94F8
:106ED000FBA4C755DF4F1881C95AD040CE018B554E
:106EE0009F4F0E947E8F0FB6F894BEBE0FBEADBE00
:106EF0000BC0CE018B559F4F0E947E8F0FB6F8942A
:106F0000BEBE0FBEADBE10E0BE016F5F7F4FCE01B3
:106F10008F5B9F4F0E94D2CD010F10E0E1E4F0E0C3
:106F2000EC0FFD1FE00FF11F1082BE016F5B7F4F62
:106F30008091291590912A150E945191B801CE0196
:106F40008F5B9F4F0E94E9A3BC018091291590910E
:106F50002A150E9403846AE08091291590912A15D0
:106F60000E946D908091291590912A15DC01ED9178
:106F7000FC910680F781E02D19950E947D508930A3
:106F800048F080912B0F811103C070922B0F02C02B
:106F900010922B0F0E94B4440E94CCA30E942C9606
:106FA00081110EDE8091210F81110FC080912C0F75
:106FB000882359F080912B15811107C080911F0FF4
:106FC0009091200F0A970CF4A3CE8091620C82302E
:106FD00039F0833009F02EC481E080939B0F2AC4DE
:106FE00081E08093520F26C410922C0F5AC3109147
:106FF000250F8FEF810F853028F060E089E80E942F
:107000007DA418C4133079F018F41230F9F004C0DC
:10701000143079F0153099F040E6442E49E0542EB2
:10702000612C712C19C0412C3BE4532E612C712C26
:1070300013C0412C26E9522E612C712C0DC0412C1D
:1070400092EC592E66246394712C06C080E8482E79
:1070500085E2582E612C712C00E0E12EF12C5701B5
:10706000BFE8AB0EB11C1501E89427F83324E6E91C
:10707000EE0EF11CE894E7F8FF24023091F018F4CA
:10708000013051F004C0033089F00430A1F040E633
:1070900059E060E070E013C040E855E260E070E065
:1070A0000EC040E05BE460E070E009C040E056E9FB
:1070B00060E070E004C040E052EC61E070E087EB1B
:1070C00098E00E94CF7E87EB98E00E94438E0E945A
:1070D000245B4B015C01F2E38F0E911CA11CB11CDF
:1070E0000E948CA30E94245B681579058A059B0584
:1070F000B8F360E870E087EB98E00E941C986FE0BE
:1071000070E087EB98E00E941C98612F87EB98E075
:107110000E94FD8DB10187EB98E00E941C980E94AF
:10712000245B4B015C012AE0820E911CA11CB11C66
:107130000E948CA30E94245B681579058A059B0533
:10714000B8F367E870E087EB98E00E941C986FE066
:1071500070E087EB98E00E941C98612F87EB98E025
:107160000E94FD8DB70187EB98E00E941C9887EB89
:1071700098E00E94438E0E94245B4B015C013EE537
:10718000830E31E0931EA11CB11C0E948CA30E94AF
:10719000245B681579058A059B05B8F30F5F0530F8
:1071A00009F06BCFB301A20187EB98E00E94CF7E7C
:1071B00040926714509268146092691470926A1435
:1071C000B301A20180EC91E00E9437A56AC283E07E
:1071D00090E00E94B4CB2AE0DC012C9327EB38E04E
:1071E00012963C932E9311976AE00CC083E090E0D6
:1071F0000E94B4CB2DE0FC01208327EB38E03283E2
:1072000021836DE00E940FA24CC24091250F509146
:10721000260F0091270F1091280F6091230F709176
:10722000240FCE010196C355DF4F4883CD5AD0407D
:10723000C255DF4F5883CE5AD0400E943F6EC3558F
:10724000DF4F4881CD5AD040C255DF4F5881CE5ACA
:10725000D040892BE9F08D81873050F4853080F45F
:107260008130B0F0642F8B819C810E946E840DC0B0
:10727000893070F4B8018B819C810E9437A505C0CC
:10728000BA018B819C810E9412830E94F8A404C0E1
:1072900061E085E80E947DA480911E0F8111CAC221
:1072A00081E080931E0FC6C2B090230FE090240FA0
:1072B000C156DF4F1882CF59D04064ED76E0CE0141
:1072C0008F579F4F0E94DA8F6B2D7E2DCE018057F6
:1072D0009F4F0E943F6E892B09F4BEC0CC56DF4FF2
:1072E000E881C459D0404E2F50E0FA013197E83080
:1072F000F10508F0B1C08827E25AFE4F8F4F0C9479
:10730000A0CBCE56DF4F88819981C259D0400E94D0
:1073100064C94AE0682FCE0101960E94AE8F1BC05F
:10732000CE56DF4F88819981C259D0400E9464C9EE
:10733000682F880F770B4AE00AC0CE56DF4F88814E
:107340009981C259D0400E9471C94AE0BC01CE0166
:1073500001960E94838FBE016F5F7F4FCE018F57D2
:107360009F4F0E94A48ECE01019663C0CE56DF4F80
:1073700088819981C259D0400E9471C923961FAE5D
:107380001EAE239725961FAE1EAE259727961FAEDD
:107390001EAE27974AE0BE016F5F7F4F0E9412C862
:1073A00035C0CE56DF4F88819981C259D0400E94A6
:1073B0006CC923961FAE1EAE239725961FAE1EAE38
:1073C000259727961FAE1EAE27972AE0AE014F5F86
:1073D0005F4F0E94D9C71AC0CE56DF4F888199816E
:1073E000C259D0400E946CC923961FAE1EAE23978F
:1073F00025961FAE1EAE259727961FAE1EAE279769
:107400002AE0AE014F5F5F4F0E94E7C7BE016F5F8A
:107410007F4FCE018F5B9F4F0E945E8FBE016F5BDF
:107420007F4FCE018F579F4F0E94A48ECE018F5B5E
:107430009F4F0E947E8F4FE050E0BE016F5B7F4FF9
:10744000CE018F579F4F0E94FBA4CB57DF4FF88090
:10745000C558D04011E002C0F12C10E0CE018F578A
:107460009F4F0E947E8F112309F4C7CD8E010156D4
:107470001F4F20E4AE014F5F5F4F68E87B2D8E2DDC
:107480000E9409A4BE016F5B7F4FCE0101960E944E
:10749000D2CDC156DF4F8881CF59D040F80E81E060
:1074A0008F0DC156DF4F8883CF59D040E1E0F0E027
:1074B000EC0FFD1FEF0DF11D9CE79083E1E0F0E084
:1074C000EC0FFD1FE80FF11D1082BE016F5F7F4FB3
:1074D0008091291590912A150E945191C156DF4F34
:1074E0006881CF59D04070E0CE0101960E94E9A397
:1074F000BC018091291590912A150E9403846AE0AD
:107500008091291590912A150E946D9080912915DE
:1075100090912A15DC01ED91FC910680F781E02D18
:10752000199588C18091230F9091240F803891057F
:1075300009F080C18E0100571F4F20E4AE014F5F5C
:107540005F4F68E870E880E00E9409A46DE876E08B
:10755000CE018F579F4F0E94DA8FCE018F579F4FDA
:107560000E9404A5C057DF4F2881C059D040CB5797
:10757000DF4F88819981C558D040820F911DC05737
:10758000DF4F8883C059D04022961FAE22974FE02C
:1075900050E0BE016F5B7F4FCE018F579F4F0E941F
:1075A0002686BE016F5B7F4FCE0101960E94D2CD31
:1075B000C057DF4F8881C059D040E1E0F0E0EC0FC8
:1075C000FD1FE80FF11D1082BE016F5F7F4F80919C
:1075D000291590912A150E945191C057DF4F68815B
:1075E000C059D04070E0CE0101960E94E9A3BC01D1
:1075F0008091291590912A150E9403846AE0809158
:10760000291590912A150E946D90809129159091CD
:107610002A15DC01ED91FC910680F781E02D19958A
:10762000CE018F579F4F0E947E8F04C18091230F00
:107630009091240F8338910509F0FCC08E0100570A
:107640001F4F20E4AE014F5F5F4F68E873E880E0B2
:107650000E9409A44AE060911D0FCE018F579F4FF1
:107660000E94AE8F7ACF8091230F9091240F8238A1
:10767000910509F0DFC08E0100571F4F20E4AE01D5
:107680004F5F5F4F68E872E85ECF8091230F909163
:10769000240F8138910509F0CDC080912C0F811104
:1076A000C9C00E94F8A4C6C08091230F9091240FF6
:1076B0004F9709F0BFC081E08093210FBBC00E94AB
:1076C000AA50029719F060E084E899CC8091610C8F
:1076D000811102C00E9493840E947D50F82E64EDB7
:1076E00076E0CE0180579F4F0E94DA8FC156DF4F60
:1076F0001882CF59D0408E0101561F4F20E4AE01B1
:107700004F5F5F4F68E879E780E00E9409A4CF5798
:10771000DF4F19821882C158D040CD57DF4F1982F0
:107720001882C358D040CB57DF4F19821882C558F2
:10773000D0406F2D70E080E090E02AE0AE014F5B1A
:107740005F4F0E94D9C7BE016F5B7F4FCE018F573D
:107750009F4F0E945E8FBE016F577F4FCE018057B3
:107760009F4F0E94A48ECE018F579F4F0E947E8F05
:107770004FE050E0BE016F5B7F4FCE0180579F4FBF
:107780000E942686CC56DF4F1881C459D040BE01D6
:107790006F5B7F4FCE0101960E94D2CDC156DF4F65
:1077A0008881CF59D040810F91E0980FC156DF4FAB
:1077B0009883CF59D040E1E0F0E0EC0FFD1FE80FD7
:1077C000F11D8CE78083E1E0F0E0EC0FFD1FE90F95
:1077D000F11D1082BE016F5F7F4F8091291590913E
:1077E0002A150E945191C156DF4F6881CF59D04070
:1077F00070E0CE0101960E94E9A3BC018091291599
:1078000090912A150E9403846AE080912915909135
:107810002A150E946D908091291590912A15DC01FE
:10782000ED91FC910680F781E02D1995CE018057EE
:107830009F4FF9CE0FB6F894DEBE0FBECDBEC25537
:10784000DF4F0FB6F894DEBF0FBECDBFDF91CF91F3
:107850001F910F91FF90EF90DF90CF90BF90AF906E
:107860009F908F907F906F905F904F903F902F9060
:107870000895FC0182810895482F50E095E1899F89
:10788000F0011124EB51FE4E2181328180859185DA
:10789000280F391F838194818217930728F08581EF
:1078A000968128173907E8F485E1849FF001859FC8
:1078B000F00D1124EB51FE4E858196812817390772
:1078C00028F52581368185E1849FF001859FF00DA3
:1078D0001124EB51FE4E8285823019F411861086F8
:1078E000128685E1849FF001859FF00D1124EB51F4
:1078F000FE4E328321838091840090918500280F71
:10790000391F3093890020938800089583819481E2
:1079100082179307C0F623813481D5CF63E30C949B
:107920005A8C62E30C945A8C61E30C945A8C60E399
:107930000C945A8C64E50C945A8C6FE20C945A8C1B
:107940006DE20C945A8C6CE20C945A8C77FF03C055
:1079500071956195710920E0462F6EE20C94128CAE
:10796000462F20E06DE40C94128CFC0162836111BF
:1079700005C020E040E06BE40C94128C089577FF82
:1079800003C071956195710920E0462F6BE40C945A
:10799000128C4F925F926F927F928F929F92AF92D2
:1079A000BF92CF92DF92EF92FF920F931F93CF93EC
:1079B000DF936C01A4ECCA1AADEFDA0AD601ED919F
:1079C000FC917E970CF05DC0FC01E858FF4F812CC4
:1079D000912CA191B191AB2B21F42115310549F4E2
:1079E00050C0BFEF8B1A9B0AAEE18A16910489F74B
:1079F00048C0EC015401AA0CBB1CAA0CBB1CAC0E69
:107A0000BD1EF501EC54FF4F4083518362837383A5
:107A10007401EE0CFF1CEC0EFD1EF701E858FF4F41
:107A200031832083EC54FF4F11830083BE01680D26
:107A3000791DFB01EC55FE4F81E080830E94245BA1
:107A4000F5016083718382839383C65CDD4F8881F7
:107A50009981F701E250FE4F91838083D6012D91E9
:107A60003C9111972F5F3F4F2D933C939C012F5FCB
:107A70003F4F1216130614F021E030E039832883BB
:107A800002C08FEF9FEFDF91CF911F910F91FF9079
:107A9000EF90DF90CF90BF90AF909F908F907F90AE
:107AA0006F905F904F9008950F931F93CF93DF9344
:107AB0008C01C62FD42F65E870E0DC019F968D9174
:107AC0009C91D0970E941C98F80187A590A9DC0191
:107AD000ED91FC910190F081E02D6C2F1995F8014A
:107AE00087A590A9DC01ED91FC910190F081E02D3A
:107AF0006D2F19952C2F30E0B9016B577F4F6D0F0B
:107B0000711D6F777727F80187A590A9DF91CF9135
:107B10001F910F910C941C98262F2B7FA1F49A0192
:107B20004F3F510519F014F02FEF30E0A90141301B
:107B30002FEF520714F441E05FEF57FF03C0519558
:107B400041955109B1CF0895CF93DF93EC0189ADF1
:107B50009AAD892B11F01AAE19AECE010E94A77E04
:107B60008BA9813029F0823069F0811117C005C0DE
:107B700060E070E08DE00E94A3581092AD0010927A
:107B8000AC0008C040E064E0CE018EDF40E060E081
:107B9000CE018ADF1AA219A21F8E1E8E0E94245BBC
:107BA0006DAB7EAB8FAB98AFDF91CF9108958F9285
:107BB0009F92AF92BF92CF92DF92EF92FF920F937C
:107BC0001F93DC0114968D919C9115975696CD903C
:107BD000DC9057976817790709F455C09096FC9088
:107BE00090974C01092E000CAA08BB088B01072EA8
:107BF000000C220B330B861797073CF41296ED917D
:107C0000FC911397FF2031F014C0ED91FC91119776
:107C1000FF2079F00D2C000CEE08FF08A901980157
:107C2000281939094A095B0954966D917C91559739
:107C30000EC00D2C000CEE08FF08A90198012819B0
:107C400039094A095B0952966D917C915397CB0192
:107C5000770FAA0BBB0BBC01CD016C197D098E09F6
:107C60009F090E946ACB8F01FF0F220B330BA901E2
:107C70009801281939094A095B090E9484C9C20E72
:107C8000D31EE41EF51EC6011F910F91FF90EF90C9
:107C9000DF90CF90BF90AF909F908F9008958F927C
:107CA0009F92AF92BF92CF92DF92EF92FF920F938B
:107CB0001F93DC0114968D919C9115971A96CD9087
:107CC000DC901B976817790709F455C09096FC90D3
:107CD00090974C01092E000CAA08BB088B01072EB7
:107CE000000C220B330B861797073CF41296ED918C
:107CF000FC911397FF2031F014C0ED91FC91119786
:107D0000FF2079F00D2C000CEE08FF08A901980166
:107D1000281939094A095B0918966D917C911997C0
:107D20000EC00D2C000CEE08FF08A90198012819BF
:107D300039094A095B0916966D917C911797CB0119
:107D4000770FAA0BBB0BBC01CD016C197D098E0905
:107D50009F090E946ACB8F01FF0F220B330BA901F1
:107D60009801281939094A095B090E9484C9C20E81
:107D7000D31EE41EF51EC6011F910F91FF90EF90D8
:107D8000DF90CF90BF90AF909F908F900895EF922B
:107D9000FF920F931F93CF93DF93EC0189AD9AADC0
:107DA000892B11F01AAE19AE8BA98130B1F0823057
:107DB00059F1811143C0CB0177FF03C091958195A3
:107DC0009109BC01CE016BDF9093AD008093AC00B4
:107DD0009AA389A39F8F8E8F31C08B0177FF03C039
:107DE000119501951109B801CE0159DF7C01B80147
:107DF000CE01DDDE8C01B7018DE00E94A358109307
:107E0000AD000093AC0016C08B0177FF03C0119545
:107E100001951109B801CE0142DF7C01B801CE0104
:107E2000C6DE8C01A70164E0CE0176DEA80160E029
:107E3000CE0172DEFAA2E9A21F8F0E8F0E94245B90
:107E40006DAB7EAB8FAB98AFDF91CF911F910F9150
:107E5000FF90EF900895CF93DF93EC0189AD9AAD39
:107E6000892B11F01AAE19AE2FA138A58DA19EA1B4
:107E70009F838E83398728879B878A872DA53EA578
:107E80008BA59CA59B8B8A8B3D8B2C8B9F8B8E8B84
:107E900060E070E0CE017BDF0E94245B6DAB7EABC7
:107EA0008FAB98AFDF91CF910895CF93DF93EC0123
:107EB00089AD9AAD892B11F01AAE19AE2FA138A554
:107EC0008BA19CA19F838E83398728879B878A8774
:107ED0002DA53EA589A59AA59B8B8A8B3D8B2C8BC6
:107EE0009F8B8E8B60E070E0CE0151DF0E94245B9F
:107EF0006DAB7EAB8FAB98AFDF91CF910895DC0176
:107F0000A250BE4F20E030E04D915D9146175707DB
:107F100039F4280F391FF901EC55FE4F808108957F
:107F20002F5F3F4F2E31310579F780E00895CF93D1
:107F3000DF93EC01C45CDD4FA881B981109709F48F
:107F400042C0FC01E250FE4F20E030E041915191EF
:107F50004617570799F5A901440F551F480F591F98
:107F6000FA01E858FF4F60817181672B61F111823E
:107F70001082FC01E20FF31FEC55FE4F1082FA0154
:107F8000EE53FE4F11821082235D3F4F220F331FAD
:107F9000220F331FFC01E20FF31F108211821282A5
:107FA0001382FA01E859FE4F11821082EA56FF4F00
:107FB000118210821197B983A88305C02F5F3F4FAC
:107FC0002E31310519F6DF91CF9108950F931F934C
:107FD00001E010E0DEDC1F910F9108950F931F93D5
:107FE00000E010E0D6DC1F910F9108952F923F9290
:107FF0004F925F926F927F928F929F92AF92BF92B9
:10800000CF92DF92EF92FF920F931F93CF93DF9364
:1080100000D000D0CDB7DEB78C010E94245B980160
:108020002E533E4F3C832B831E830D83D801AC55CA
:10803000BE4FBA83A9831801B2E02B1ABEEF3B0AE8
:10804000F901AA24A394B12C32E0832E912C118241
:1080500010829F012A543140D9012D913C91232B4C
:1080600009F44DC0AD81BE812D913D914D915C9142
:1080700013977D01B4EBEB0EF11CD701CD90DD9091
:10808000ED90FC902B013C01421A530A640A750AD8
:108090004C145D046E047F0490F1C20ED31EE41EE6
:1080A000F51EAD81BE81CD92DD92ED92FC921397CB
:1080B000A981BA812C91222311F19F0126593109FE
:1080C000D9012D913C912115310519F4B182A0827D
:1080D00016C07F01BAE5EB1AF108D7014D915C910A
:1080E0001197421753075CF4B182A0824F5F5F4F34
:1080F0004D935C934217530714F09182808232961D
:108100002D813E812C5F3F4F3E832D83A981BA8113
:108110001196BA83A983E215F30509F098CFEB8194
:10812000FC8181919191FC83EB838130910599F0E1
:108130000297C9F4EB81FC81EC54F1400190F0818D
:10814000E02D1995AB81BC81DA966D917C91DB971E
:10815000C801EDDE08C0EB81FC81EC54F1400190D8
:10816000F081E02D19952B813C8122153305B9F65C
:1081700026960FB6F894DEBF0FBECDBFDF91CF912C
:108180001F910F91FF90EF90DF90CF90BF90AF9035
:108190009F908F907F906F905F904F903F902F9027
:1081A00008956E3E22E0720738F06B3C98E0790744
:1081B00028F06AEC78E002C06EEE72E0660F771F7E
:1081C0009FB7F89425E1829FF0011124EB51FE4EF8
:1081D000748363839FBF08956E3E22E0720738F078
:1081E0006B3C98E0790728F06AEC78E002C06EEE0C
:1081F00072E0660F771F9FB7F89425E1829FF00128
:108200001124EB51FE4E768365839FBF0895660F60
:10821000771F282F30E095E1899FF0011124EB5161
:10822000FE4E858196816817790718F465817681FD
:1082300007C0838194818617970710F46381748146
:108240008FB7F89495E1929FF001939FF00D112460
:10825000EB51FE4E728361838FBF0895982F8FB7C5
:10826000F89425E1929FF0011124EB51FE4E21E09C
:1082700027838FBF41B121E030E0B90102C0660F12
:10828000771F9A95E2F7CB01842B81B908958A3044
:1082900058F49FB7F89425E1829FF0011124EB5127
:1082A000FE4E118610869FBF08951F93CF93DF93D4
:1082B00025E1829FC0011124EC01CB51DE4E8A855D
:1082C00081110FC01FB7F89481E08A8789899A8944
:1082D0009A8389830E94245B6B877C878D879E8726
:1082E0001FBFDF91CF911F910895CF93DF938A3005
:1082F000D0F56233710538F061369DE6790728F0D4
:1083000060E67DE602C062E370E0D42FC82F80E013
:1083100090E00E943FC820E030E04AE754E40E9429
:1083200046CA20E030E04CE852E40E94A0C89B011D
:10833000AC0160E070E08AEF94E40E9446CA0E94BB
:10834000AECA9B01DD2321F022273327261B370BE2
:108350008FB7F89495E1C99FF0011124EB51FE4EBF
:10836000318720878FBFDF91CF9108958A3008F43D
:1083700018CF08958A3008F42FCF08958A3058F422
:1083800095E1899FF0011124EB51FE4E818192818C
:1083900096958795089580E090E008958A3008F4D6
:1083A00036CF08951F920F920FB60F9211240BB67D
:1083B0000F920F931F932F933F934F935F936F935E
:1083C0007F938F939F93AF93BF93CF93EF93FF933D
:1083D0008091740F893048F01092740F809194123C
:1083E000882399F080918D120DC0E091740FE150B7
:1083F00025E1E29FF0011124EB51FE4E8781882395
:1084000021F0808192B1892782B9E091740F85E1D2
:10841000E89FF0011124EB51FE4E8781882321F063
:10842000808192B1892B82B9E091740FC5E1CE9F12
:10843000F0011124EB51FE4E80859185892B09F0C6
:108440004DC0E091740FCE9FF0011124EB51FE4E10
:108450008285813009F060C00E94245BE091740F36
:10846000CE9FF0011124EB51FE4E03851485258526
:108470003685E091740FCE9FF0011124EB51FE4E32
:108480000784F089E02DAB01BC01401B510B620B4E
:10849000730BCF01A0E0B0E084179507A607B707DC
:1084A000D8F5E091740FA091740FCA9FD0011124E8
:1084B000AB51BE4E53968D919C915497CE9FF00137
:1084C0001124EB51FE4E91878087E091740FCE9F6F
:1084D000F0011124EB51FE4E82E082878091740FEF
:1084E000CBD98091740F8F5F8093740FFF91EF91C0
:1084F000CF91BF91AF919F918F917F916F915F913C
:108500004F913F912F911F910F910F900BBE0F90A4
:108510000FBE0F901F901895E091740F809184000A
:108520009091850025E1E29FF0011124EB51FE4E70
:1085300021813281820F931F90938900809388005C
:10854000D0CF1F93CF93DF938091730F811173C0AE
:108550001092740F9FB7F89485E128EB3BE04CED47
:1085600055E064E971E1A1E0B0E0E091740FE93019
:1085700008F052C0E091740F8E9FF0011124EB516E
:10858000FE4E32832183E091740F8E9FF0011124FF
:10859000EB51FE4E56834583E091740F8E9FF001A0
:1085A0001124EB51FE4E74836383E091740FF091BC
:1085B000740FED0101C0CC0FFA95EAF78E9FF00120
:1085C0001124EB51FE4EC083E091740F8E9FF00199
:1085D0001124EB51FE4E1782E091740F8E9FF00133
:1085E0001124EB51FE4E11861086E091740F8E9F80
:1085F000F0011124EB51FE4E1286E091740F8E9F14
:10860000F0011124EB51FE4E148A138AE091740F8D
:10861000EF5FE093740FA9CF9FBF8FB7F89420EA64
:108620003FE030938F1220938E1210928D128FBFE5
:1086300081E08093730FDF91CF911F9108950F9385
:108640001F93CF93DF938C01C62FD42FDC0111969B
:108650008D919C911297DC01ED91FC910190F0813C
:10866000E02DD8016C911995F80181819281DC018E
:10867000ED91FC910190F081E02D6C2F1995F8019E
:1086800081819281DC01ED91FC910190F081E02DDE
:108690006D2F1995F80180816C2F70E0680F711DA6
:1086A0006D0F711D6F77772781819281DF91CF9157
:1086B0001F910F910C941C980F931F93CF93DF93EE
:1086C0008C01C62FD42FDC0111968D919C911297AD
:1086D000DC01ED91FC910190F081E02DD8016C91CD
:1086E0001995F80181819281DC01ED91FC91019055
:1086F000F081E02D6C2F1995F80181819281DC01C8
:10870000ED91FC910190F081E02D6D2F1995F8010C
:1087100080816C2F70E0680F711D6D0F711D6F7778
:10872000772781819281DF91CF911F910F910C94D6
:108730001C984F925F926F927F92AF92BF92CF92AE
:10874000DF92EF92FF921F93CF93DF93DD24D394B8
:1087500045E0C42EC2E0D0E053E0E52EF12CAA247F
:10876000A394B12C8091570F9091580FDC01ED919B
:10877000FC910084F185E02D1995892B09F4D1C075
:10878000109130018091570F9091580FDC01ED91BD
:10879000FC910284F385E02D199596B3B39A20914C
:1087A0008400309185002059384E30938D002093FD
:1087B0008C00212F2C7119F01092720F2AC093FB9C
:1087C000992790F9E091720FE11116C0992351F2A7
:1087D0008F3041F6D092720F8093590F8091550FD0
:1087E0009091560F892B09F0BDCFB092560FA092F1
:1087F000550F1092540FB6CF992381F01092720F3B
:108800001092540F8091550F9091560F029709F0D6
:10881000A9CFF092560FE092550FA4CF91E09E0F92
:108820009093720FF0E0E75AF04F8083993109F08E
:1088300099CF811173C08091700F82FF05C0F092B3
:10884000560FE092550F6AC083FDF9CF8091550F06
:108850009091560F019761F48091540F8F5F809330
:10886000540F843058F0D093560FC093550F06C064
:10887000D093560FC093550F1092540F8091530F01
:108880008F5F8093530F9091520F981708F044C058
:10889000D092510FA1E3BFE0EAE5FFE040E050E0F5
:1088A000BA0110E0CF01FC011B3098F40196408022
:1088B000512C612C712C012E04C0440C551C661CDB
:1088C000771C0A94D2F74429552966297729185F1D
:1088D000EACF9A013770205E3340C29EC001C39E2A
:1088E000900D112497FD079623E0959587952A957D
:1088F000E1F784529A4F8D939D931B503BE0769500
:108900006795579547953A95D1F78FE0A135B80708
:1089100049F61092530F02C01092510F1092720F2D
:1089200021CFDF91CF911F91FF90EF90DF90CF90FB
:10893000BF90AF907F906F905F904F90089580911F
:10894000620C833031F480912F0F9091300F0C9492
:10895000BC6A08958091620C823029F480912D0FB9
:1089600090912E0FE6CE0895F5DFE9CF1092BE115B
:108970001092C8111092D2111092DC11109266114F
:1089800080E090E0FC01E759FE4E118207968435A5
:108990009105C1F70895C0C6FBC6E2C51CC680910B
:1089A000810F882311F0DCD501C015D69091810F7D
:1089B00081E089278093810F08958091C407909169
:1089C000C507DC01ED91FC91EA5BFF4F0190F0815E
:1089D000E02D199580919014882341F06DEE72E19D
:1089E00080918E1490918F140C9476910895CF936A
:1089F000DF93CDB7DEB765970FB6F894DEBF0FBE35
:108A0000CDBF80914A1390914B1320914813309120
:108A100049133A8329839C838B8381E08D8B82E089
:108A20008F938DB79EB745970FB6F8949EBF0FBE34
:108A30008DBFADB7BEB7119685E1FE0131960190AD
:108A40000D928A95E1F786E79CE00E949EA70FB6FB
:108A5000F894DEBF0FBECDBF80919014882381F0C3
:108A600065E173E180918E1490918F1465960FB635
:108A7000F894DEBF0FBECDBFDF91CF910C947691FD
:108A800065960FB6F894DEBF0FBECDBFDF91CF91D4
:108A9000089566D5409175145091761460E070E0A9
:108AA0002BEE3AE489ED9CE091DA90934E15809399
:108AB0004D1580919014882341F060EA72E1809115
:108AC0008E1490918F140C947691089584D54091D2
:108AD00075145091761460E070E020EB3AE489ED73
:108AE0009CE074DA90934E1580934D15809190140C
:108AF000882341F06DE872E180918E1490918F147B
:108B00000C947691089580915E07882339F086E76A
:108B10009CE00E94CBA728EC3BE406C086E79CE0E3
:108B20000E94F2A72CE83BE44CE251E060E070E0E8
:108B300089ED9CE04BDA80919014882341F062E04B
:108B400073E180918E1490918F140C947691089516
:108B500086E79CE00E94DEA78111DEC519C68CE085
:108B60000C94799F8BE00C94799F8AE00C94799F08
:108B700089E00C94799F88E00C94799F87E00C94AD
:108B8000799F86E00C94799F85E00C94799F84E02E
:108B90000C94799F83E00C94799F82E00C94799FE8
:108BA00081E00C94799F8CE00C94A19F8BE00C9455
:108BB000A19F8AE00C94A19F89E00C94A19F88E07A
:108BC0000C94A19F87E00C94A19F86E00C94A19F38
:108BD00085E00C94A19F84E00C94A19F83E00C9409
:108BE000A19F82E00C94A19F81E00C94A19F0C9422
:108BF000C19F0C94CD9F0F931F93CF93DF93009150
:108C00007C0F10917D0FC0913507D0913607B801C8
:108C1000CE0175D9882371F0B801CE0188D9809131
:108C2000370790913807DC01ED91FC9102A0F3A188
:108C3000E02D199500917A0F10917B0FC0913507A7
:108C4000D0913607B801CE015AD9882319F0B8015E
:108C5000CE016DD9599880919014882361F06FE20C
:108C600072E180918E1490918F14DF91CF911F91BA
:108C70000F910C947691DF91CF911F910F910895F0
:108C8000CF93DF9380914C15882311F110924C15EE
:108C900060E08DE00E94EF56C0914D15D0914E15C9
:108CA000BE0189ED9CE02BD9882321F0BE0189ED1E
:108CB0009CE03DD980919014882371F064ED72E1BD
:108CC00080918E1490918F14DF91CF910C947691B6
:108CD000DF91CF910C9419A8DF91CF9108958091E5
:108CE0004C15811102C00C9419A80895CF93DF93FD
:108CF00080914F158823F9F033D410924F15C0910D
:108D00004D15D0914E15BE0189ED9CE0F8D8882311
:108D100021F0BE0189ED9CE00AD98091901488234E
:108D200069F06BEB72E180918E1490918F14DF915A
:108D3000CF910C947691DF91CF9162C4DF91CF9166
:108D400008955EC48091820F882311F009D401C078
:108D5000E6D59091820F81E089278093820F089554
:108D6000DEC5F0C506C68091800F882311F0EAD5D4
:108D700001C0FFD59091800F81E089278093800FFB
:108D8000089542C641D68091C4079091C507DC0181
:108D9000ED91FC9106A0F7A1E02D199472C6809187
:108DA0007F0F882311F030D601C06BD690917F0FD2
:108DB00081E0892780937F0F08957FC69AC68091AE
:108DC0007E0F882311F079D601C093D690917E0F43
:108DD00081E0892780937E0F08950E941A5D80911B
:108DE00090148823D1F020914E1480918E1490918C
:108DF0008F14211107C020915114211103C067E382
:108E000072E109C020914D0C222319F066E772E14E
:108E100002C062E672E10C947691089580914D0C47
:108E200081110C94125D0C941A5D0E94125D809168
:108E30009014882341F061E872E180918E14909142
:108E40008F140C94769108950C94047C8091E40F17
:108E500081110C94EE7B0C94047C0C94EE7B0CD46E
:108E60008091C4079091C507DC01ED91FC9104A0AD
:108E7000F5A1E02D1994CF93DF93C0913507D091E0
:108E8000360760917C0F70917D0FCE0138D881112B
:108E900027C04091790F50E060E070E027EE35E6A2
:108EA000CE019CD890937D0F80937C0F80913707E3
:108EB00090913807DC01ED91FC9100A0F1A1E02D2B
:108EC000199580915107882359F060917A0F70911C
:108ED0007B0F809135079091360711D8882371F068
:108EE000809190148823E1F066E272E180918E1403
:108EF00090918F14DF91CF910C9476910E940F6620
:108F00002FE036E644E650E060E070E080913507FF
:108F10009091360763D890937B0F80937A0FE0CFC0
:108F2000DF91CF9108950E94305D80919014882345
:108F300041F06BEF71E180918E1490918F140C943D
:108F400076910895E091770FF091780F8281ADD9F5
:108F500080919014882341F06DED71E180918E1421
:108F600090918F140C94769108958091E50F882349
:108F700019F00E948C6602C00E94835D809190145B
:108F8000882379F02091D81380918E1490918F14BA
:108F9000222319F061EA71E102C06AEB71E10C94DD
:108FA000769108950C949C77CF93DF93D82FC62F9A
:108FB0008091C4079091C507DC01ED91FC91E85BBD
:108FC000FF4F0190F081E02D462F6D2F1995809174
:108FD0009014882399F16DE371E180918E14909142
:108FE0008F140E945291DD2329F0D13059F468E3A7
:108FF00071E102C063E371E180918E1490918F144E
:109000000E945291C73069F028F4C130B9F469E484
:1090100071E10CC0C83041F0C93081F463E571E101
:1090200005C06DE671E102C06FE571E180918E14BB
:1090300090918F14DF91CF910C947691DF91CF9125
:10904000089569E081E0B0CF68E081E0ADCF67E0EE
:1090500081E0AACF61E081E0A7CF69E080E0A4CF02
:1090600068E080E0A1CF67E080E09ECF61E080E033
:109070009BCFCF9380914E0C882309F480C00E942F
:10908000A26690914C0C882341F0911178C0809198
:109090005707882309F45BC072C0911170C080919A
:1090A00090148823D1F062E871E180918E14909140
:1090B0008F140E94529180914D0C882341F067E7F4
:1090C00071E180918E1490918F140E945291809141
:1090D0008E1490918F140E945A900E944A6781E0EA
:1090E0008093420780911C14882309F448C0809122
:1090F000E40F882349F18091D813882379F028E67A
:1091000037E742E350E060E070E089ED9CE00E94C8
:10911000EE3F9093760F8093750F31C080910702D8
:10912000813069F54091DA135091DB13141615065E
:109130005CF4052E000C660B770B23EE36E789ED09
:109140009CE0CF910C94E63FCF910C94E37682E0C3
:109150008093570780919014882341F06EE871E165
:1091600080918E1490918F140E947691C1E0C093EB
:1091700088140E949C770E944A67C0934207CF914F
:10918000089581E00C94CA778091891481110C9420
:109190009C7781E00C94CA770C9458820C94C77821
:1091A0008091921481110C9458820C94C7789C0180
:1091B0000197849710F4822F0895C901845691096C
:1091C0008438934040F4C90164E670E00E9479CB92
:1091D000822F94E61BC0283E43E03407D8F0C90133
:1091E00068EE73E00E9479CB48E15CEF649FC001B8
:1091F000659F900D749F900D1124280F391FC90190
:109200006AE070E00E948DCB822F9AE0699F8019FE
:109210001124089580E0089567E271E180918E1431
:1092200090918F140C945291CF93C82F8091C407C2
:109230009091C507DC01ED91FC91EC5BFF4F019033
:10924000F081E02D6C2F199580919014882389F07E
:10925000E3DF6C2F80918E1490918F140E945182C5
:109260006FE171E180918E1490918F14CF910C94E5
:109270007691CF9108958CE0D7CF8BE0D5CF8AE05F
:10928000D3CF89E0D1CF88E0CFCF87E0CDCF86E0C4
:10929000CBCF85E0C9CF84E0C7CF83E0C5CF82E0E4
:1092A000C3CF81E0C1CF60E082E20E94EF5660E070
:1092B00083E20E94EF5660E085E30E94EF5660E093
:1092C00085E00E94EF5660E084E00E94EF5660E087
:1092D0008BE00E94EF5659980895CF93C0910E02EB
:1092E0006C2F82E20E94EF5681E0C8276C2F83E248
:1092F0000E94EF56C0930E02CF910895CF93DF9353
:10930000C0910D026C2F82E20E94EF56D1E0DC2763
:109310006D2F83E20E94EF566C2F85E30E94EF567B
:109320006D2F85E00E94EF566D2F84E00E94EF566E
:109330006C2F8BE00E94EF56CC2311F0599801C09E
:10934000599A90910D0281E0892780930D02DF9157
:10935000CF910895CF93DF938091980F81110DC025
:109360001092970F1092960F81E090E09093950FD6
:109370008093940F8093980F36C08091960F9091B0
:10938000970F863191057CF18F38910534F48091E7
:10939000940F9091950F019609C08D3521E09207A9
:1093A00054F48091940F9091950F02969093950F9D
:1093B0008093940F18C0863222E0920734F4809193
:1093C000940F9091950F0496F1CF883E93403CF412
:1093D0008091940F9091950F8A5B9F4FE7CF1092E9
:1093E000950F1092940F8ADFC091960FD091970F2E
:1093F000C93E83E0D80754F01092980F54DF22E260
:109400003AE448EE53E060E070E007C02AEA39E44D
:10941000AE010D2E000C660B770B89ED9CE00E94CF
:10942000E63F9093930F8093920F8091940F9091C9
:10943000950F8C0F9D1F9093970F8093960FDF9140
:10944000CF910895CF93DF938091CA07882319F0B5
:10945000DF91CF917FCFC091920FD091930FBE013A
:1094600089ED9CE00E947F3F882329F0BE0189EDB1
:109470009CE00E94973FDF91CF9115CFCF93C09191
:109480008F0F6C2F70E08DE00E94A35889E18093CC
:109490008E0F90910C02992311F0CD5F01C0C35043
:1094A000C0938F0F80918F0F873970F0992321F02F
:1094B0008FEF80938F0F08C08D3D30F086E9809349
:1094C0008F0F88E780938E0F80918F0F8F3F19F455
:1094D00010920C0205C08A3118F481E080930C02CE
:1094E00040918E0F50E060E070E02EE33AE489EDA9
:1094F0009CE00E94E63F90934E1580934D15CF91CE
:109500000895CF92DF92EF92FF92CF93DF93EC0119
:109510009C01AFEFB0E00E94D2C9CC24CA9423E0F2
:10952000D22EE12CF12CA70196010E9484C9B90129
:109530008DE00E94A3589E01A4E6B0E00E94D2C92B
:10954000A70196010E9484C980917B148213209305
:109550007B14DF91CF91FF90EF90DF90CF90089533
:10956000CF93DF93C0914D15D0914E15BE0189ED7B
:109570009CE00E947F3F882329F0BE0189ED9CE09A
:109580000E94973F60E08DE00E94EF56809190141A
:109590008823D1F080914F15882319F064E674E197
:1095A0000DC080914C15882319F06BE474E106C05E
:1095B00080919910811108C06CE374E180918E1440
:1095C00090918F140E94769110924F1510924C1525
:1095D000DF91CF91089561E08DE00E94EF56809178
:1095E0009014882361F080914F15811108C06EE2BC
:1095F00074E180918E1490918F140C94769108955B
:1096000080914F15811110C0ABDF81E080934F1521
:1096100080919014882341F063E974E180918E1465
:1096200090918F140E94769180918D0F882329F05C
:1096300060E08DE00E94EF5601C0CDDF90918D0F6C
:1096400081E0892780938D0F882329F0409177143A
:109650005091781404C04091791450917A1460E0CC
:1096600070E020E03BE489ED9CE00E94E63F9093AF
:109670004E1580934D150895CF9380918B0F8111D6
:109680000FC081E080938B0F80919014882341F06C
:109690006CEF73E180918E1490918F140E947691FB
:1096A000C0918A0F6C2F85E00E94EF564091801484
:1096B00050E060E070E02CE33BE489ED9CE00E9428
:1096C000E63F9093890F8093880F81E06C2F682785
:1096D00060938A0FCF9108958091070180FF1BC08E
:1096E00080919014882351F087EA9CE00E94DEA7C5
:1096F000811108C08091B30C811104C087EA9CE0FD
:109700000C94CBA763E773E180918E1490918F1432
:109710000E947691F3CF08958091070181FF1BC0CD
:1097200080919014882351F086E79CE00E94DEA788
:10973000811108C08091820C811104C086E79CE0F1
:109740000C94CBA766E473E180918E1490918F14F2
:109750000E947691F3CF08958091070180FF17C092
:1097600080919014882331F087EA9CE00E94DEA764
:10977000882321F087EA9CE00C94F2A76DE573E161
:1097800080918E1490918F140E947691F3CF08955A
:109790008091070181FF17C080919014882331F0D8
:1097A00086E79CE00E94DEA7882321F086E79CE004
:1097B0000C94F2A760E373E180918E1490918F1462
:1097C0000E947691F3CF089580912D07882321F090
:1097D00080E090E00C94EE7680E090E00C940177CD
:1097E0006091900F7091910F89ED9CE00E947F3FF6
:1097F00081112EC060E082E20E94EF5660E083E2B9
:109800000E94EF5660E085E30E94EF5660E085E03D
:109810000E94EF5660E084E00E94EF5660E08BE02B
:109820000E94EF56599880917D14882319F02EE7F5
:1098300039E402C02DE639E442E350E060E070E034
:1098400089ED9CE00E94EE3F9093910F8093900FE2
:10985000089560E083E20C94EF5661E083E20C949B
:10986000EF560F931F93CF93DF938C01C1E0D0E0AD
:109870000C171D079CF0F1DF64E670E080E090E0DB
:109880000E94EC5AE6DFC017D10734F46AE570E0B5
:1098900080E090E00E94EC5A2196EACFDF91CF91D0
:1098A0001F910F91089583E090E0DBCF82E090E07C
:1098B000D8CF81E090E0D5CF60E082E20C94EF5603
:1098C00061E082E20C94EF560F931F93CF93DF93E6
:1098D0008C01C1E0D0E00C171D079CF0F1DF64E6BD
:1098E00070E080E090E00E94EC5AE6DFC017D107FC
:1098F00034F46AE570E080E090E00E94EC5A219632
:10990000EACFDF91CF911F910F91089583E090E00E
:10991000DBCF82E090E0D8CF81E090E0D5CF6091BE
:109920007B1470E08DE00E94A358809190148823EE
:1099300041F06DE774E180918E1490918F140C9436
:109940007691089510928C0F8091B707811104C011
:1099500060E084E00E94EF5680919014882341F0EB
:109960006BE174E180918E1490918F140C94769138
:10997000089581E080938C0F8091B707811106C014
:109980006091830F70E084E00E94A358809190144E
:10999000882341F069E074E180918E1490918F14D6
:1099A0000C9476910895CF93DF93C091900FD0914E
:1099B000910FBE0189ED9CE00E947F3F882351F00A
:1099C000BE0189ED9CE00E94973F1092910F10928A
:1099D000900F69DC80917214882319F0DF91CF9188
:1099E000C8CFDF91CF9108951092B70780918C0F67
:1099F000811104C060E084E00C94EF566091830F05
:109A000070E084E00C94A358CF93DF9360E085E08E
:109A10000E94EF5680918B0F81110BC08091C4077B
:109A20009091C507DC01ED91FC9104ACF5ADE02D02
:109A30001995C091880FD091890FBE0189ED9CE0E6
:109A40000E947F3F882329F0BE0189ED9CE00E949F
:109A5000973F80919014882379F020918B0F80910B
:109A60008E1490918F14222319F060EF73E102C0DD
:109A700064EE73E10E94769110928B0FDF91CF918B
:109A8000089561E085E00E94EF568091C4079091AF
:109A9000C507DC01ED91FC9104ACF5ADE02D199505
:109AA00080919014882341F069ED73E180918E14C8
:109AB00090918F140C947691089560E085E30E9454
:109AC000EF568091C4079091C507DC01ED91FC91A0
:109AD00000ACF1ADE02D199580919014882341F0F0
:109AE0006DEC73E180918E1490918F140C947691AB
:109AF000089561E085E30E94EF568091C40790913C
:109B0000C507DC01ED91FC9100ACF1ADE02D19959C
:109B100080919014882341F062EC73E180918E145F
:109B200090918F140C94769108958F929F92AF929A
:109B3000BF92CF92DF92EF92FF9285E40E94A85AE3
:109B4000BC01990F880B990B0E9441C86B017C01E5
:109B500080910B02882351F0C092840FD092850F20
:109B6000E092860FF092870F10920B0226E636E6FF
:109B700046E65FE36091840F7091850F8091860FB8
:109B80009091870F0E94A0C84B015C0120ED3CEC36
:109B90004CEC5DE3C701B6010E94A0C89B01AC017B
:109BA000C501B4010E94E2C96093840F7093850FD0
:109BB0008093860F9093870F23E23BED49E75CE3A8
:109BC0000E94A0C8FF90EF90DF90CF90BF90AF9021
:109BD0009F908F900895CF93DF938091070180FD30
:109BE0002AC0C0916007D0916107809164078823E3
:109BF00071F08EE30E94A85A813092402CF01092AE
:109C00006107109260070AC081E090E003C08EE314
:109C10000E94A85A90936107809360078091600723
:109C2000909161078C179D0719F41092620703C089
:109C300081E080936207DF91CF910895CF93DF9306
:109C40008091070181FD2AC0C0915A07D0915B071E
:109C500080915E07882371F08FE30E94A85A8130BB
:109C600092402CF010925B0710925A070AC081E0D4
:109C700090E003C08FE30E94A85A90935B07809303
:109C80005A0780915A0790915B078C179D0719F42A
:109C900010925C0703C081E080935C07DF91CF9155
:109CA000089580910F14833059F02CF48130E9F03D
:109CB0008230D9F030C0863044F08630B1F02BC00D
:109CC0008091BA079091BB071FC08091BA0790910D
:109CD000BB07DC01ED91FC910480F581E02D199525
:109CE0008091B8079091B9070FC08091BE079091FD
:109CF000BF07DC01ED91FC910480F581E02D199501
:109D00008091BC079091BD07DC01ED91FC9104802E
:109D1000F581E02D19958091C4079091C507DC016C
:109D2000ED91FC91E25BFF4F0190F081E02D1995E0
:109D30008091C4079091C507DC01ED91FC910484EA
:109D4000F585E02D60E070E01994ABDF0E94EC5CDB
:109D50008091921481110E9458828091C60790913F
:109D6000C707DC01ED91FC910480F581E02D199588
:109D70008091C2079091C307DC01ED91FC910480B2
:109D8000F581E02D19958091E713882331F08091BA
:109D90004307909144070C94A43D089580910A02D2
:109DA000882351F0C2DE20E030E040E050E40E9421
:109DB0003BC887FF39C00895B8DE20E030E04AE7AD
:109DC00054E40E94A0C80E94B3CA2091701430913C
:109DD00071144091CA076217730710F4442351F1BC
:109DE000442309F444C0A1DE20E030E04AE754E413
:109DF0000E94A0C80E94B3CA2091701430917114BF
:109E000062177307A0F11092CA0781E08093C90717
:109E100080919014882359F16AE873E180918E143F
:109E200090918F140C94769110920A0281E08093A5
:109E3000C907089581E08093CA071092C9078091ED
:109E40009014882391F069EA73E180918E149091C7
:109E50008F140E9452910E9444A866EA73E1809197
:109E60008E1490918F140E9476916FDFEBCA089543
:109E700080915C0C811157C0E091C511F091C61121
:109E8000858196819093C2118093C1111092C41163
:109E90001092C311E091CF11F091D011858196817C
:109EA0009093CC118093CB111092CE111092CD11C2
:109EB000E091D911F091DA11858196819093D611B4
:109EC0008093D5111092D8111092D711E091E3111F
:109ED000F091E411858196819093E0118093DF11D8
:109EE0001092E2111092E11182E190E090936511DD
:109EF0008093641181E08093BE118093C811809398
:109F0000D2118093DC118093661180E090E021E013
:109F1000FC01E759FE4E2183079684359105C1F770
:109F200081E080935C0C08951092DE1108951092E8
:109F3000D41108958F929F92AF92BF92CF92DF92E9
:109F4000EF92FF921F93CF93DF93EC0111E08E818C
:109F50009F81892B09F410E02C813D81E885F985EA
:109F6000C580D680878190E0A601480F591F24172D
:109F7000350764F180850D2C000CEE08FF08A9015F
:109F8000330F660B770B0380F481E02D9A01AB0150
:109F90002C193D094E095F09882329F0A1E0BFEF84
:109FA0000E94ACC904C0AFEFB0E00E94A0C94F014D
:109FB000FF0FAA08BB08A50194012C193D094E0901
:109FC0005F090E9484C93F832E834BC0A601481BB2
:109FD000590B421753070CF43FC080850D2C000C21
:109FE000EE08FF08A901330F660B770B8180928082
:109FF000092C000CAA08BB089A01AB0128193909E1
:10A000004A095B09882399F0A1E0BFEF0E94ACC91F
:10A01000A7019601281939094A095B090E9484C9D8
:10A02000DA01C90181509F4FAF4FBF4F12C0AFEF50
:10A03000B0E00E94A0C9A7019601281939094A0970
:10A040005B090E9484C9DA01C9018F5F9109A109E6
:10A05000B1099F838E8305C01F821E82111101C02A
:10A0600019828E819F81009789F08F3F910519F0A9
:10A0700014F08FEF90E081305FEF950714F481E0EA
:10A080009FEF9F838E8381E018271A83DF91CF9102
:10A090001F91FF90EF90DF90CF90BF90AF909F9077
:10A0A0008F90089581E08093590C089581E080930A
:10A0B0005A0C089581E080935B0C0895CF93DF9351
:10A0C000C091D00FD091D10F6091E00F7091E10F4E
:10A0D000CE010E947F3F81110DC028E33FE444EF91
:10A0E00051E060E070E0CE010E94E63F9093E10F06
:10A0F0008093E00FDF91CF9108958091620C8230C0
:10A1000039F0833049F0813049F48091D80F01C093
:10A1100080E180935E0C04C08EE0FBCF10925E0C59
:10A1200080915E0C08958091620C823039F083300A
:10A1300051F0813069F48091D70F08950E94AA44AC
:10A140008091510F08950E949F448091D60F0895E9
:10A1500080E008958091620C823049F0833071F084
:10A16000813099F48091D20F9091D30F08950E947D
:10A17000AA448091550F9091560F08950E949F44D4
:10A180008091D40F9091D50F089581E090E00895CB
:10A190002F923F924F925F926F927F928F929F92F7
:10A1A000AF92BF92CF92DF92EF92FF920F931F93E5
:10A1B000CF93DF9300D000D0CDB7DEB74DB65EB6FB
:10A1C0000E94AA440E949F44C5DF029709F0E8C29A
:10A1D000AADF882309F4DFC2C090E00FD090E10F1E
:10A1E000E090D00FF090D10FB601C7010E947F3FE1
:10A1F0008823F1F0F701E250FE4F00E010E081917A
:10A2000091918C159D0571F40E94245B000F111F24
:10A21000000F111FF701E00FF11F6083718382832C
:10A22000938307C00F5F1F4F0E31110541F701C027
:10A2300045DF10925C0CEDB6FEB640915F0C50917C
:10A24000600CCA01880F991FADB6BEB6A81AB90A2C
:10A250000FB6F894BEBE0FBEADBE0DB71EB70F5FF2
:10A260001F4F8091620C823069F0833029F1813078
:10A2700009F071C0B8018091D90F9091DA0F0E9456
:10A28000C1A233C03FB7F89420E0822F90E084173A
:10A29000950774F4880F991FF801E80FF91FDC0186
:10A2A000AF5CB04F8D919C91918380832F5FEDCFF8
:10A2B0003FBF1092510F19C03FB7F89420E0822F92
:10A2C00090E08417950774F4880F991FF801E80F40
:10A2D000F91FDC01AC54B04F8D919C919183808328
:10A2E0002F5FEDCF3FBF1092D60F20E06AE071E004
:10A2F000822F90E040915F0C5091600C841795077D
:10A3000054F5689FF001699FF00D1124EC53FF4E46
:10A31000A085B1858C918823E1F0A081B1813C9129
:10A32000C801830F911D830F911DDC0112978D9140
:10A330009C91A281B3814D915C9111970480F5812C
:10A34000E02D4817590711F4108203C070838D93D4
:10A350009C932F5FCDCF0FB6F894FEBE0FBEEDBE1F
:10A360008091BE11882319F08DEB91E1E3DD80919E
:10A37000C811882319F087EC91E1DCDD8091D211BE
:10A38000882319F081ED91E1D5DD8091DC118823DE
:10A3900019F08BED91E1CEDD80915D0C882309F4FD
:10A3A00065C08091D211811105C08091DC11882394
:10A3B00009F450C08091D5119091D611E091D91136
:10A3C000F091DA11238134812817390724F480852C
:10A3D000811109C00EC0218132818217930734F4A4
:10A3E0008085811106C088E090E005C080E190E0A2
:10A3F00002C080E290E02091DF113091E011E09105
:10A40000E311F091E411438154814217530724F47E
:10A410002085222349F00AC0418152812417350743
:10A420003CF42085222311F0816003C0846001C0C8
:10A43000826020916411309165112817390719F451
:10A440001092661107C0909365118093641181E0AA
:10A45000809366118091641190916511429709F47F
:10A46000A3C181E08093DE118093D411AAE6B1E10B
:10A470006DE671E188EE682E83E0782E2224239425
:10A48000FD0131978081882309F47CC11496CD9019
:10A49000DC901597DE82CD82F6018781882309F44E
:10A4A00071C18C91882309F46DC111964D915C9115
:10A4B000129730847301E41AF50A1E141F042CF05D
:10A4C0007A01F8EEEF1AF3E0FF0A20E030E001E055
:10A4D00010E0EFE0F7E290E0832C912CA32CB12C5C
:10A4E000C12CD12CA982BA82CB82DC82650182E0A8
:10A4F000C81AD108081519050CF04AC08BE0C81617
:10A50000D104E0F5F6018827EA59FE4F8F4F0C94ED
:10A51000A0CBF901E35AF94F27C0F901E95AF94FE5
:10A5200023C0F901E15BF94F1FC0F901EB5BF94F63
:10A530001BC0F901E75CF94F17C0F901E55DF94F60
:10A5400013C0F901E55EF94F0FC0F901E75FF94F5C
:10A550000BC0F901EB50FA4F07C0F901E152FA4F75
:10A5600003C0F901E953FA4F0280F381E02DE41BA7
:10A57000F50BF7FF03C0F195E195F109EE15FF0525
:10A5800014F4902F7F010F5F1F4F2E5F3F4FB2CF0C
:10A590009F5FED81FE818185882309F4EAC0032D48
:10A5A00010E0F8013297EB30F10508F0E2C088279F
:10A5B000EF58FE4F8F4F0C94A0CB913009F0ACC0F8
:10A5C000C3C0913009F4D4C0933009F0D2C0A4C004
:10A5D000913009F4CBC0923009F4CAC0933009F429
:10A5E000B3C0943009F0C5C097C0913009F4BCC025
:10A5F000923009F4BBC0943009F4A6C0953009F03C
:10A60000B8C08AC0913009F4ADC0923009F4ACC032
:10A61000933009F4ABC0943009F4AAC0953009F422
:10A6200093C0963009F0A5C077C0913009F498C066
:10A63000923009F497C0933009F496C0953009F42C
:10A6400097C0963009F480C0973009F092C064C07A
:10A65000913009F483C0923009F482C0933009F438
:10A6600081C0943009F480C0953009F47FC09630E1
:10A6700009F47EC0973009F467C0983009F079C0BA
:10A680004BC0913009F468C0923009F467C0933030
:10A6900009F466C0943009F465C0963009F466C0C8
:10A6A000973009F465C0983009F44EC0993009F02C
:10A6B00060C032C0913009F44DC0923009F44CC0F2
:10A6C000933009F44BC0943009F44AC0953009F432
:10A6D00049C0963009F448C0973009F447C0983013
:10A6E00009F446C0993081F19A3009F042C014C093
:10A6F000913071F1923071F1933071F1943071F1C8
:10A70000953071F1973081F1983081F1993081F174
:10A710009A30D1F09B3069F591E02BC09130B1F0C7
:10A720009230B1F09330B1F09430B1F09530B1F097
:10A730009630B1F09730B1F09830B1F09930B1F077
:10A740009A30B1F09B30A9F492E013C09CE011C0A4
:10A750009BE00FC09AE00DC099E00BC098E009C0E3
:10A7600097E007C096E005C095E003C094E001C003
:10A7700093E0FB018081891302C01C9203C02C92DC
:10A78000FB0190831796695F7F4FF1E1AE3BBF07F6
:10A7900009F076CE03C00E94B64490DC81E066C02A
:10A7A0000E94B64480E062C0E0906711F0906811AA
:10A7B0001E141F040CF055C08091D3110091D00FCE
:10A7C0001091D10F6091DE0F7091DF0F8823B1F0EF
:10A7D00081E08093D411C8010E947F3F811115C090
:10A7E000A701FF0C660B770B27E93FE4C8010E9425
:10A7F000E63F9093DF0F8093DE0F07C0C8010E94F1
:10A800007F3F811102C01092D4118091DD1100911F
:10A81000D00F1091D10F6091DC0F7091DD0F882364
:10A82000D1F081E08093DE11C8010E947F3F811149
:10A830001DCE4091671150916811052E000C660BDA
:10A84000770B24E93FE4C8010E94E63F9093DD0FB7
:10A850008093DC0F0BCEC8010E947F3F811106CE92
:10A8600002C01092D4111092DE1100CE0FB6F894EF
:10A870005EBE0FBE4DBE26960FB6F894DEBF0FBE6D
:10A88000CDBFDF91CF911F910F91FF90EF90DF909F
:10A89000CF90BF90AF909F908F907F906F905F9080
:10A8A0004F903F902F900895CF938091DB0FC091F0
:10A8B0000F02811100C1C23009F44FC0C33009F446
:10A8C0009CC0C13009F027C180915B0C811123C16C
:10A8D00081E090E00E94B4CB9093DA0F8093D90F7F
:10A8E00062E083E0F4D31092B10F1092D30F109274
:10A8F000D20F1092D70F80E090E0FC01EE0FFF1F07
:10A90000E156F04F11821082019688309105A9F727
:10A910001092B00F1092AF0F80916A008C608093FC
:10A920006A00ED9A8FB7F8942091840030918500E9
:10A9300030939A0F2093990F8FBF2AE530E54AEFA5
:10A9400050E060E070E08091D00F9091D10F0E94B4
:10A95000E63F81E08093DB0FDEC080915A0C8111CD
:10A96000DAC081E090E00E94B4CB90932E0F8093E8
:10A970002D0F809104018E7F809304018091050149
:10A980008160809305018AE198E09093580F80934D
:10A99000570F2EE240EA56E861E070E00E94F09224
:10A9A000809165008B7F809365001092350189E06E
:10A9B000809334018EE2809332018CEF80933001DA
:10A9C00080E9809331011092560F1092550F10922A
:10A9D000540F1092530F1092510FE1E3FFE08CEDF2
:10A9E00095E0819391932FE0E135F207D1F7C1E033
:10A9F000C093520F26E530E551C08091590C81116A
:10AA00008AC081E090E00E94B4CB9093300F809395
:10AA10002F0F809104018E7F8093040180910501A6
:10AA20008160809305018AE198E09093B30F809351
:10AA3000B20F26E040E052EC61E070E00E94F0923C
:10AA4000809165008B7F809365001092350180E1D5
:10AA50008093340186E0809332018EEF8093300141
:10AA600080E9809331011092D50F1092D40F10928B
:10AA70009E0F10929D0F1092D60FE4EBFFE08CED2D
:10AA800095E0819391932FE0E03DF207D1F710928A
:10AA90009C0FC1E0C0939B0F22E530E54AEF50E0E8
:10AAA00060E070E08091D00F9091D10F0E94E63F5E
:10AAB000C093DB0F30C0C23069F0C330D1F0C13079
:10AAC00051F580915B0C811126C08091D20F90913D
:10AAD000D30F1DC080915A0C81111DC080912D0F84
:10AAE00090912E0F0E9499438091550F9091560F8F
:10AAF0000EC08091590C81110EC080912F0F909142
:10AB0000300F0E94BC6A8091D40F9091D50F0297AC
:10AB100011F4C093620C80910F028230A1F1833056
:10AB200009F454C0813009F074C080915B0C882313
:10AB300009F46FC0ED98E59A1092B10F1092D80FFA
:10AB40001092D30F1092D20F1092D70F80E090E0A6
:10AB5000FC01EE0FFF1FE156F04F118210820196AB
:10AB600088309105A9F71092B00F1092AF0F809125
:10AB7000D90F9091DA0F0E9449CC1092DB0F1092FE
:10AB80005A0C82E044C080915A0C882309F441C0D9
:10AB90008091570F9091580F0E94CE928091310171
:10ABA0008F7780933101809131018F7E80933101C5
:10ABB0001092300180912D0F90912E0F0E9449CC60
:10ABC0001092DB0F1092590C83E021C08091590C38
:10ABD0008823F9F08091B20F9091B30F0E94CE922A
:10ABE000809131018F7780933101809131018F7E87
:10ABF000809331011092300180912F0F9091300F8E
:10AC00000E9449CC1092DB0F10925B0C81E0809384
:10AC10000F028091D00F9091D10FCF910C94F63FFD
:10AC2000CF93DF9300D01F921F92CDB7DEB7FE0106
:10AC3000319625E0DF011D922A95E9F724E8298362
:10AC400025E52C832AE22D836A834B8345E050E07F
:10AC5000BF010E94CBA165E070E080E090E0BCD431
:10AC600080E00F900F900F900F900F90DF91CF9199
:10AC700008951092A61210923D0710923407109278
:10AC80003E0710923F07109240071092410781E063
:10AC900080934A0C409148075091490760E070E06A
:10ACA00028E536E580913507909136070C94E63F0C
:10ACB00080914D0C882361F18091FB0A81111CC0A9
:10ACC00010923D0B10923E0B10923F0B1092400BD6
:10ACD0001092410B1092420B1092450B8091480C40
:10ACE0009091490CDC01ED91FC910190F081E02DF7
:10ACF000199510924A0C089528E536E545E050E094
:10AD000060E070E080913507909136070C94E63F43
:10AD100008956091EE0F7091EF0F8091350790913B
:10AD200036070E947F3F882319F081E08093ED0F62
:10AD3000089590E0FC013197E231F10508F04EC032
:10AD40008827E458FE4F8F4F0C94A0CB8091800051
:10AD50008F7703C0809180008F7D8093800008955D
:10AD600080918000877FF9CF84B58F7702C084B54A
:10AD70008F7D84BD08958091B0008F7703C080914E
:10AD8000B0008F7D8093B0000895809190008F7700
:10AD900007C0809190008F7D03C080919000877FD5
:10ADA0008093900008958091A0008F7707C08091D4
:10ADB000A0008F7D03C08091A000877F8093A000BA
:10ADC0000895809120018F7707C0809120018F7DA9
:10ADD00003C080912001877F8093200108951F93F5
:10ADE000CF93DF93282F30E0F901E358F34E84919D
:10ADF000F901E95CF34ED491F901EF50F44EC4919E
:10AE0000CC23C1F0162F811194DFEC2FF0E0EE0F70
:10AE1000FF1FE953FB4EA591B4918FB7F894111120
:10AE200005C09C91ED2FE095E92302C0EC91ED2B3C
:10AE3000EC938FBFDF91CF911F91089560E08BE07D
:10AE4000CEDF10924B0C089561E08BE0C8DF81E00B
:10AE500080934B0C0895CF93DF938091FB0F81116A
:10AE600010C084EF91E09093FA0F8093F90F8BE27A
:10AE700090E09093F80F8093F70F81E08093FB0FA1
:10AE800020C08091F70F9091F80F8532910514F052
:10AE9000049709C08331910514F0029704C08230F1
:10AEA00091052CF001979093F80F8093F70F809104
:10AEB000F70F9091F80F97FF04C01092F80F1092BF
:10AEC000F70FC091F60FCC2311F0B8DF01C0BCDF43
:10AED00081E08C278093F60FC091F90FD091FA0F83
:10AEE0001C161D0654F01092FB0FA8DF2BE937E566
:10AEF0004AEF50E060E070E007C02BE237E5AE01BA
:10AF00000D2E000C660B770B80913507909136075C
:10AF10000E94E63F9093F50F8093F40F8091F70F16
:10AF20009091F80FC81BD90BD093FA0FC093F90F6B
:10AF3000DF91CF9108950F931F93CF93DF9380916B
:10AF40004C0C882329F0DF91CF911F910F9183CF73
:10AF50000091F40F1091F50FC0913507D09136078D
:10AF6000B801CE010E947F3F882321F0B801CE01B5
:10AF70000E94973FDF91CF911F910F915FCFCF92AA
:10AF8000DF92EF92FF9210924C0C20913907309192
:10AF90003A0740913B0750913C0760913E07709102
:10AFA0003F0780914007909141070E94E1C96B01E2
:10AFB0007C0120E030E0A9010E943BC887FD09C068
:10AFC000C0923E07D0923F07E0924007F0924107BF
:10AFD00008C010923E0710923F071092400710924F
:10AFE0004107FF90EF90DF90CF90A5CFEF92FF92B7
:10AFF0001F93CF93DF9300D0CDB7DEB784E689836C
:10B000008CE38A8388E28B831091F00F1330E8F48D
:10B01000E12EF12C10FF02C011DF01C015DFE1E0CD
:10B02000F0E0EC0FFD1FEE0DFF1D408150E060E0F1
:10B0300070E026EF37E580913507909136070E9442
:10B04000E63F1F5F1093F00F03C0F8DE1092F00F81
:10B050000F900F900F90DF91CF911F91FF90EF9085
:10B06000089580914B0C882311F0E8DE01C0ECDEDE
:10B0700090914B0C81E0892780934B0C089560E000
:10B080008DE0ADCE61E089E2AACE0F931F93CF93FE
:10B09000DF9360E08BE2A3DE0091E20F1091E30FFB
:10B0A000C0913507D0913607B801CE010E947F3F8D
:10B0B000882341F0B801CE01DF91CF911F910F910C
:10B0C0000C94973FDF91CF911F910F910895CF93EB
:10B0D000DF9390E0FC01E95CF34E2491FC01EF501A
:10B0E000F44E8491882361F190E0880F991FFC0150
:10B0F000E355FB4EC591D491FC01E953FB4EA5915C
:10B10000B491611109C09FB7F8948881209582237A
:10B110008883EC912E230BC0623061F49FB7F894C2
:10B120003881822F809583238883EC912E2B2C935A
:10B130009FBF06C08FB7F894E8812E2B28838FBF5E
:10B14000DF91CF9108951F93CF93DF93182FEB01D9
:10B1500061E0BDDF209711F460E004C0CF3FD1056E
:10B1600031F461E0812FDF91CF911F9138CEE12F33
:10B17000F0E0E358F34EE4914E2F50E0FA0131979E
:10B18000E231F10508F09DC08827E257FE4F8F4F4E
:10B190000C94A0CB84B5806884BDC7BD97C084B52E
:10B1A000806284BDC8BD92C0809180008068809319
:10B1B0008000D0938900C093880088C0809180006F
:10B1C000806280938000D0938B00C0938A007EC001
:10B1D00080918000886080938000D0938D00C09320
:10B1E0008C0074C08091B00080688093B000C093E0
:10B1F000B3006CC08091B00080628093B000C093B7
:10B20000B40064C080919000806880939000D093D7
:10B210009900C09398005AC08091900080628093FA
:10B220009000D0939B00C0939A0050C080919000F2
:10B23000886080939000D0939D00C0939C0046C08E
:10B240008091A00080688093A0008091A0008F7BF7
:10B250008093A000D093A900C093A80037C080912C
:10B26000A00080628093A000D093AB00C093AA009E
:10B270002DC08091A00088608093A000D093AD0085
:10B28000C093AC0023C0809120018068809320018E
:10B29000D0932901C093280119C0809120018062B8
:10B2A00080932001D0932B01C0932A010FC080917D
:10B2B0002001886080932001D0932D01C0932C0140
:10B2C00005C0C038D1050CF04CCF46CFDF91CF91EF
:10B2D0001F9108950F931F93CF93DF939091F30FD6
:10B2E0008091A61291112AC0882309F44FC00091C1
:10B2F000F10F1091F20FC0913507D0913607B801C8
:10B30000CE010E947F3F882321F0B801CE010E9428
:10B31000973F9ADD2AE639E542EC51E060E070E0C3
:10B3200080913507909136070E94EE3F9093F20F7F
:10B330008093F10F81E08093F30F52C0882329F0AE
:10B34000DF91CF911F910F918CCE80914B0C882370
:10B35000B9F36091F10F7091F20F809135079091E0
:10B3600036070E94973F2AE639E544E150E060E065
:10B3700070E080913507909136070E94EE3F9093E0
:10B38000F20F8093F10F1092F30F2AC0C0911002B8
:10B39000D09111022297D0931102C09310021C1673
:10B3A0001D066CF4BE0177278BE0CDDECC2321F0A7
:10B3B00081E080934B0C14C010924B0C11C0609133
:10B3C000F10F7091F20F80913507909136070E942E
:10B3D000973F34DD8FEF90E090931102809310023D
:10B3E000DF91CF911F910F9108950F931F93CF93EA
:10B3F000DF930091E90F1091EA0FC091EB0FD0910C
:10B40000EC0FC00FD11FD093EC0FC093EB0FBE0118
:10B4100077278BE098DECC2321F081E080934B0CE2
:10B4200002C010924B0C10161106ECF58091E70F3C
:10B430009091E80FC817D9070CF485C08091ED0FE3
:10B44000882371F01092E80F1092E70F8CEF9FEFB6
:10B450009093EA0F8093E90F81E08093E60F73C029
:10B4600068E770E080E090E00E94EE8FDC01CB01A5
:10B470000A96A11DB11D9093E80F8093E70F68E233
:10B4800070E080E090E00E94EE8FDC01CB010A9634
:10B49000A11DB11D66277727681B790B7093EA0FF2
:10B4A0006093E90F50C0012B09F44DC08091E70F64
:10B4B0009091E80F8C179D070CF445C08091E60F22
:10B4C000882311F10091EE0F1091EF0FC091350715
:10B4D000D0913607B801CE010E947F3F882399F1B1
:10B4E000B801CE010E94973FA9DC1092EC0F109298
:10B4F000EB0F1092E60F8091A612882321F1DF91C5
:10B50000CF911F910F91E6CE69E670E080E090E068
:10B510000E94EE8FDC01CB018A569F4FAF4FBF4F89
:10B520009093E80F8093E70F68E270E080E090E08E
:10B530000E94EE8FDC01CB010A96A11DB11D9093F4
:10B54000EA0F8093E90FDF91CF911F910F9108953A
:10B55000863308F0865390917B00282F2870977FC0
:10B56000922B90937B008770806480937C00809105
:10B570007A00806480937A0080917A0086FDFCCF07
:10B58000809178002091790090E0922B08953FB748
:10B59000F8948091011090910210A0910310B09145
:10B5A000041026B5A89B05C02F3F19F00196A11DD8
:10B5B000B11D3FBFBA2FA92F982F8827820F911D49
:10B5C000A11DB11DBC01CD0142E0660F771F881F90
:10B5D000991F4A95D1F708958F929F92AF92BF928B
:10B5E000CF92DF92EF92FF926B017C01D0DF4B0193
:10B5F0005C01C114D104E104F104E9F0C8DFDC010D
:10B60000CB0188199909AA09BB09883E9340A10575
:10B61000B10578F321E0C21AD108E108F10888EEFB
:10B62000880E83E0981EA11CB11CC114D104E10452
:10B63000F10421F7DECFFF90EF90DF90CF90BF9025
:10B64000AF909F908F9008952FB7F8946091FD0F61
:10B650007091FE0F8091FF0F909100102FBF089501
:10B660001F920F920FB60F9211242F933F938F9337
:10B670009F93AF93BF938091FD0F9091FE0FA09188
:10B68000FF0FB09100103091FC0F23E0230F2D37F6
:10B6900020F40196A11DB11D05C026E8230F0296D6
:10B6A000A11DB11D2093FC0F8093FD0F9093FE0F01
:10B6B000A093FF0FB09300108091011090910210A1
:10B6C000A0910310B09104100196A11DB11D8093AB
:10B6D000011090930210A0930310B0930410BF9137
:10B6E000AF919F918F913F912F910F900FBE0F902F
:10B6F0001F9018950F931F93CF93DF930091F40F32
:10B700001091F50FC0913507D0913607B801CE01E1
:10B710000E947F3F8823A1F0B801CE010E94973F8D
:10B7200029E836E548EB5BE060E070E080913507A2
:10B73000909136070E94E63F9093F50F8093F40FA7
:10B740006091EE0F7091EF0F809135079091360761
:10B750000E947F3F81114BC01092ED0F8FEF90E060
:10B760009093EC0F8093EB0F6FDB68E770E080E065
:10B7700090E00E94EE8FDC01CB010A96A11DB11D65
:10B780009093E80F8093E70F68E270E080E090E02C
:10B790000E94EE8FDC01CB010A96A11DB11D662728
:10B7A0007727681B790B7093EA0F6093E90F25EFF9
:10B7B00039E544E150E060E070E080913507909118
:10B7C00036070E94EE3F9093EF0F8093EE0F29E82B
:10B7D00036E548EB5BE060E070E0809135079091E2
:10B7E00036070E94E63F9093F50F8093F40FDF91A8
:10B7F000CF911F910F9108958F929F92AF92BF9218
:10B80000CF92EF92FF920F931F93CF93DF932091EC
:10B810005307223008F07AC07B018C0180903E07EC
:10B8200090903F07A0904007B090410720E030E0A3
:10B83000A901C501B4010E943BC8181654F520E0C7
:10B8400030E0A901C501B4010E94DFCA181654F402
:10B8500020E030E048E452E4C501B4010E943BC856
:10B860001816D4F420E030E048E452E4C501B401F5
:10B870000E94DFCA18169CF420E030E048EC52E445
:10B88000C501B4010E943BC887FF09C0CBE4D0E0EA
:10B8900008C0C0E0D0E005C0C2E3D0E002C0C4E60A
:10B8A000D0E08FEF8C0D823070F4209739F06C2F40
:10B8B000C8010E94F0886C2FC7010DC0C8010E940A
:10B8C000C17EC70116C08DEF8C0D8330F8F4209730
:10B8D00079F06C2FC801DF91CF911F910F91FF90EC
:10B8E000EF90CF90BF90AF909F908F900C94F08886
:10B8F000C801DF91CF911F910F91FF90EF90CF90F2
:10B90000BF90AF909F908F900C94C17EDF91CF91AC
:10B910001F910F91FF90EF90CF90BF90AF909F90AD
:10B920008F9008958F929F92AF92BF92CF92DF92A5
:10B93000EF92FF92C0903E07D0903F07E090400703
:10B94000F090410720E030E0A901C701B6010E9454
:10B95000DFCA20E030E040E05FE387FD0BC0C701B5
:10B96000B6010E94E2C94B015C010E94AECA97FD7C
:10B9700027C010C0C701B6010E94E1C90E94AECA2B
:10B9800097FD1EC06536710581059105DCF424E63E
:10B99000822F14C0C501B4010E94AECA653671057C
:10B9A000810591057CF420E030E040E05FE3C701D1
:10B9B000B6010E94E2C90E94AECA84E6861B03C09B
:10B9C00084E601C080E0FF90EF90DF90CF90BF90C1
:10B9D000AF909F908F9008950F931F93CF93DF9315
:10B9E00000912E0710912F07C0913507D09136078F
:10B9F000B801CE010E947F3F882321F0B801CE011B
:10BA00000E94973F80914C0C882339F010924C0C87
:10BA1000DF91CF911F910F918ECADF91CF911F912E
:10BA20000F910895EC9810924D0C68EC70E082E054
:10BA30000C94DF7E80914C07811105C080915007E6
:10BA4000811101C0EFCF8091480C9091490C0E9468
:10BA5000D66581E080934D0C64E670E00C94DF7E47
:10BA600060E089E2BCD922E438E542E350E060E0DE
:10BA700070E080913507909136070C94E63F1F9255
:10BA80000F920FB60F9211240BB60F922F933F9384
:10BA90004F935F936F937F938F939F93AF93BF93D6
:10BAA000EF93FF938091E50F8823B1F0489918C078
:10BAB000E89825E438E54CE251E060E070E08091E0
:10BAC0003507909136070E94E63F8091E40F882366
:10BAD00039F00E94FC6604C0489B02C0E898D5DAA1
:10BAE000FF91EF91BF91AF919F918F917F916F9156
:10BAF0005F914F913F912F910F900BBE0F900FBE12
:10BB00000F901F90189561E08BE269D9E89A25E4BF
:10BB100038E548E853E160E070E0809135079091A6
:10BB200036070E94E63F9093E30F8093E20F08955B
:10BB30008091C80780939014089580912D108823D8
:10BB400059F080912B1090912C10DC01ED91FC911B
:10BB50000480F581E02D1994089580912D1088239B
:10BB600069F080912B1090912C10DC01ED91FC91EB
:10BB70000190F081E02D6FEF73E0199408958091AA
:10BB80002D10882389F080913810882321F080E0DF
:10BB900090E0D3DF03C080E090E0DFDF90913810C9
:10BBA00081E0892780933810089520912D10222359
:10BBB00069F0A0912B10B0912C10ED91FC91119790
:10BBC0000190F081E02DBC01CD0119940895809180
:10BBD0002A10882359F08091281090912910DC01B7
:10BBE000ED91FC910480F581E02D199408958091E8
:10BBF0002A10882369F08091281090912910DC0187
:10BC0000ED91FC910190F081E02D6FEF73E01994BC
:10BC1000089580912A10882389F080913710882315
:10BC200021F080E090E0D3DF03C080E090E0DFDF30
:10BC30009091371081E089278093371008952091E3
:10BC40002A10222369F0A0912810B0912910ED91BB
:10BC5000FC9111970190F081E02DBC01CD01199468
:10BC6000089520912710222369F0A0912510B0910A
:10BC70002610ED91FC9111970190F081E02DBC010F
:10BC8000CD011994089520912410222369F0A091E8
:10BC90002210B0912310ED91FC9111970190F08149
:10BCA000E02DBC01CD01199408952091211022238B
:10BCB00069F0A0911F10B0912010ED91FC911197A7
:10BCC0000190F081E02DBC01CD01199408952091DF
:10BCD0001E10222369F0A0911C10B0911D10ED914F
:10BCE000FC9111970190F081E02DBC01CD011994D8
:10BCF000089520911B10222369F0A0911910B09192
:10BD00001A10ED91FC9111970190F081E02DBC018A
:10BD1000CD011994089520911810222369F0A09163
:10BD20001610B0911710ED91FC9111970190F081D0
:10BD3000E02DBC01CD011994089520911510222306
:10BD400069F0A0911310B0911410ED91FC9111972E
:10BD50000190F081E02DBC01CD01199408958091EE
:10BD6000C4079091C507DC01ED91FC91EE59FF4F9E
:10BD70000190F081E02D19948091C4079091C5073E
:10BD8000DC01ED91FC91E05AFF4F0190F081E02D34
:10BD900019948091C4079091C507DC01ED91FC9145
:10BDA000E25AFF4F0190F081E02D19940C946C4BF6
:10BDB0000C94AC4B8091C807882361F00E94AA5074
:10BDC000029741F06DEC75E180918E1490918F1483
:10BDD0000C947691089580919014882341F06FE13E
:10BDE00075E180918E1490918F140C947691089542
:10BDF00080919014882341F06FE075E180918E145A
:10BE000090918F140C9476910895CF93DF932091A5
:10BE10003F103091401028173907D1F0909340100F
:10BE200080933F1020919014222391F0EC016EE951
:10BE300075E180918E1490918F140E945291BE01F1
:10BE400080918E1490918F14DF91CF910C94947FF8
:10BE5000DF91CF910895CF93DF9320913D103091E2
:10BE60003E1028173907D1F090933E1080933D1073
:10BE700020919014222391F0EC0164E875E1809107
:10BE80008E1490918F140E945291BE0180918E1455
:10BE900090918F14DF91CF910C94947FDF91CF918B
:10BEA000089520912710222339F0BC0180911110B0
:10BEB000909112100C94239808952091241022231D
:10BEC00039F0BC0180910F10909110100C942398C0
:10BED000089520912110222339F0BC0180910D108A
:10BEE00090910E100C942398089520911E102223F7
:10BEF00039F0BC0180910B1090910C100C94239898
:10BF0000089520911B10222339F0BC018091091063
:10BF100090910A100C9423980895209118102223D0
:10BF200039F0BC0180910710909108100C9423986F
:10BF3000089520911510222339F0BC01809105103D
:10BF4000909106100C9423980895CF92DF92EF926F
:10BF5000FF9220910002213019F42091FC1304C0BB
:10BF60002230C9F5209102142223A9F19C01211548
:10BF700084E0380710F02FEF33E0ADE0B0E00E942E
:10BF8000D2C92FEF33E040E050E00E9484C969013C
:10BF90007A018FEFC81AD80AE80AF80A80911215B8
:10BFA0008C15C9F0C092121580919014882399F0D5
:10BFB0006DE675E180918E1490918F140E945291DC
:10BFC0006C2D80918E1490918F14FF90EF90DF90E4
:10BFD000CF900C943A82FF90EF90DF90CF9008952D
:10BFE000CF92DF92EF92FF9220910002213019F45C
:10BFF0002091F91304C02230C9F52091FF132223A8
:10C00000A9F19C01211584E0380710F02FEF33E0EF
:10C01000ADE0B0E00E94D2C92FEF33E040E050E045
:10C020000E9484C969017A018FEFC81AD80AE80A08
:10C03000F80A809110158C15C9F0C09210158091E6
:10C040009014882399F066E575E180918E149091A3
:10C050008F140E9452916C2D80918E1490918F14A8
:10C06000FF90EF90DF90CF900C943A82FF90EF908A
:10C07000DF90CF90089583E08093C10781E00E9414
:10C08000CA7780919014882341F069E475E180912A
:10C090008E1490918F140C947691089582E0809381
:10C0A000C10781E00E94CA7780919014882341F0F3
:10C0B0006FE275E180918E1490918F140C947691BB
:10C0C000089581E08093C1070E949C77809190142D
:10C0D000882341F06CE375E180918E1490918F1468
:10C0E0000C94769108950C94EC9F80912F108111FF
:10C0F0000BC081E09091F113911101C080E0809319
:10C100002E1081E080932F1080912E10882329F02B
:10C110000E94D99F10922E1008950E94EC9F81E0FA
:10C1200080932E1008950C94D99F8091E71381116C
:10C1300011C08091430790914407FC0121A132A1D5
:10C14000121613061CF460E070E002C06FEF70E09E
:10C150000C94C73E08958091E713811108C060E0F8
:10C1600070E080914307909144070C94C73E089576
:10C170008091E713811108C06FEF70E08091430751
:10C18000909144070C94C73E08950C94ACA0809104
:10C19000010281110C9492A00C94ACA00C9492A07A
:10C1A00084E60C94527A89E10C94527A82E30C94DE
:10C1B000527A8BE40C94527A80910002813011F40F
:10C1C00082E001C081E00C94F47A82E00C94F47A6D
:10C1D00081E00C94F47A0C94D90ECF93DF93CDB711
:10C1E000DEB765970FB6F894DEBF0FBECDBF809166
:10C1F0004A1390914B1320914813309149133A837D
:10C2000029839C838B8381E08D8B82E08F938DB714
:10C210009EB745970FB6F8949EBF0FBE8DBFADB7C2
:10C22000BEB7119685E1FE01319601900D928A9577
:10C23000E1F787EA9CE00E949EA70FB6F894DEBF64
:10C240000FBECDBF80919014882381F064EF74E11C
:10C2500080918E1490918F1465960FB6F894DEBF7E
:10C260000FBECDBFDF91CF910C94769165960FB63E
:10C27000F894DEBF0FBECDBFDF91CF9108958091BE
:10C280006407882339F087EA9CE00E94CBA72CEA58
:10C290003BE406C087EA9CE00E94F2A72CE63BE460
:10C2A0004CE251E060E070E089ED9CE00E94E63FE6
:10C2B00080919014882341F061EE74E180918E1496
:10C2C00090918F140C947691089587EA9CE00E94D7
:10C2D000DEA781110C946C4B0C94AC4B682F8091B1
:10C2E0008E1490918F140E9451826BEC75E18091B5
:10C2F0008E1490918F140C94529120918E14309141
:10C300008F14882319F062E078E002C066E078E0DC
:10C31000C9010C945291F1DF80918E1490918F1489
:10C320000C945A9020918E1430918F14882319F018
:10C3300060EC75E102C065EC75E1C9010E945291A3
:10C3400080918E1490918F140C945A9080918E1439
:10C3500090918F140C945A906EEB75E180918E142D
:10C3600090918F140C9452916AEB75E180918E1428
:10C3700090918F140C945291CF93CDE268EB75E1BC
:10C3800080918E1490918F140E945291C150B1F7F8
:10C3900080918E1490918F140E945A9080918E14E7
:10C3A00090918F14DC01ED91FC910680F781E02DD6
:10C3B000CF911994EF92FF920F931F93CF93DF9336
:10C3C00000D01F921F92CDB7DEB70E94954D20E09E
:10C3D00030E048EC52E40E94A0C80E94B3CA7B013E
:10C3E0008B0120E030E048EC52E46091061570913A
:10C3F000071580910815909109150E94A0C80E9408
:10C40000B3CA20913B1030913C102617370739F4FE
:10C410002091391030913A1002171307E1F0709310
:10C420003C1060933B10F0923A10E0923910FE01FC
:10C43000319625E0DF011D922A95E9F72BEF29833C
:10C440006A837B83EC82FD8245E050E0BF0184E596
:10C4500099E00E94338D0F900F900F900F900F90E6
:10C46000DF91CF911F910F91FF90EF900895089564
:10C4700008951092460C08950C942398CF93DF935F
:10C48000C8EDDBE081E090E09A8389831092460C4E
:10C490007ED86C837D838E839F83E49AEC9ADF91B0
:10C4A000CF9108958F929F92AF92BF92CF92DF92D9
:10C4B000EF92FF920F931F93DC0118968D919C9140
:10C4C00019971E96CD90DC901F976817790709F48D
:10C4D00056C05896FC9058974C01092E000CAA089B
:10C4E000BB088B01072E000C220B330B8617970716
:10C4F0003CF41696ED91FC911797FF2039F015C08A
:10C500001496ED91FC911597FF2079F00D2C000CFD
:10C51000EE08FF08A9019801281939094A095B09A1
:10C520001C966D917C911D970EC00D2C000CEE0891
:10C53000FF08A9019801281939094A095B091A96C7
:10C540006D917C911B97CB01770FAA0BBB0BBC01A4
:10C55000CD016C197D098E099F090E946ACB8F015C
:10C56000FF0F220B330BA9019801281939094A0939
:10C570005B090E9484C9C20ED31EE41EF51EC601CB
:10C580001F910F91FF90EF90DF90CF90BF90AF90F1
:10C590009F908F900895CF93DF93EC0161E089E045
:10C5A0000E94675860E089E00E94EF561092FB0AF3
:10C5B00081E495E099838883DF91CF910895CF92AC
:10C5C000DF92EF92FF928091FC0A833009F061C004
:10C5D0008091FD0A8130D1F488EE93E0A0E0B0E0D4
:10C5E00080938E0A90938F0AA093900AB093910A39
:10C5F00080E797E1A0E0B0E08093920A9093930ADD
:10C60000A093940AB093950A32E001C030E0E09123
:10C61000FD0AF0E0E250F54F2081A0E1A30F48EEC3
:10C6200053E060E070E088EBC82E8BE0D82EE12C60
:10C63000F12C832F90E0FC01EE0FFF1FEE0FFF1F88
:10C64000E257F54F27FF10C0C082D182E282F38209
:10C65000880F991F880F991FFC01EE56F54F4083F4
:10C660005183628373830FC04083518362837383DA
:10C67000880F991F880F991FFC01EE56F54FC08255
:10C68000D182E282F3823E5F220F3A13D2CF3093FF
:10C69000F70AFF90EF90DF90CF900895CF93DF934C
:10C6A0008091FB0A811153C01092F90A1092F60A88
:10C6B000C1E0C093FB0AD091FA0A61E089E00E94D0
:10C6C000675860E089E00E94EF562D2F30E040E08F
:10C6D00050E060E47FE180E090E00E9484C9C09374
:10C6E000B00089E08093B1002093B3008BEA289FCB
:10C6F000212D112426952093B40080916F008B7F0B
:10C7000080936F008091B00080628093B000209190
:10C71000840030918500E091F60A81E08E0F8093CD
:10C72000F60A84E0E89FF0011124E257F54F80817A
:10C730009181A281B381820F931F90938B0080938C
:10C740008A00B29A80916F00846080936F00DF91BD
:10C75000CF9108954F925F926F927F928F929F92A6
:10C76000AF92BF92CF92DF92EF92FF928AE18093D5
:10C77000F70A2093F80A88E28093FA0A81E080930E
:10C78000FD0A8093FE0A8EE08093FC0A80EC92E121
:10C79000A0E0B0E080938E0A90938F0AA093900A55
:10C7A000B093910A80EB94E0A0E0B0E08093920A0D
:10C7B0009093930AA093940AB093950AA4E1440F2E
:10C7C000551F661F771FAA95D1F722E030E0B0EB26
:10C7D000CB2EB4E0DB2EE12CF12C80E6482E89E054
:10C7E000582E612C712C90E4892E9CE9992EA12C55
:10C7F000B12CC901880F991F880F991FFC01E257BE
:10C80000F54F77FF05C0408251826282738204C077
:10C81000C082D182E282F382C9010196880F991FFA
:10C82000880F991FFC01E257F54F283129F0C0828B
:10C83000D182E282F38204C080829182A282B3829A
:10C84000440F551F661F771F2E5F3F4F2A3131055A
:10C8500081F6FF90EF90DF90CF90BF90AF909F90C8
:10C860008F907F906F905F904F9018CF8F929F9294
:10C87000AF92BF92CF92DF92EF92FF9282E18093CC
:10C88000F70A86E08093F80A96E29093FA0A91E01C
:10C890009093FD0A9093FE0A8093FC0A88ED90E441
:10C8A000A0E0B0E080938E0A90938F0AA093900A44
:10C8B000B093910A8CE19CE0A0E0B0E08093920AF2
:10C8C0009093930AA093940AB093950A742F6627C5
:10C8D0005527442722E030E0ACE1CA2EACE0DA2E46
:10C8E000E12CF12CB8E38B2EB8E19B2EA12CB12CBE
:10C8F000C901880F991F880F991FFC01E257F54F56
:10C9000077FF05C080829182A282B38204C0C08278
:10C91000D182E282F382F901EE0FFF1FEE0FFF1FBB
:10C92000EE56F54FC082D182E282F382440F551F4A
:10C93000661F771F2E5F3F4F22313105C9F68CE10C
:10C9400099E8A0E0B0E08093D20A9093D30AA09334
:10C95000D40AB093D50AFF90EF90DF90CF90BF90AC
:10C96000AF909F908F909ACE1F920F920FB60F921A
:10C9700011240BB60F922F933F934F935F936F93B6
:10C980007F938F939F93AF93BF93EF93FF93909178
:10C99000F60A8091F70A981316C01092F60A809151
:10C9A000FD0A8F5F8093FD0A9091FD0A8091FE0A37
:10C9B000891740F481E08093FD0A8091F90A8F5F26
:10C9C0008093F90AFCDD9091F90A8091F80A981396
:10C9D0000DC08091B0008F7D8093B00080916F007A
:10C9E0008B7F80936F001092FB0A27C08091B0006C
:10C9F00085FF04C08091B0008F7D03C08091B0009E
:10CA000080628093B0002091840030918500E09195
:10CA1000F60A81E08E0F8093F60A84E0E89FF00129
:10CA20001124E257F54F80819181A281B381820F59
:10CA3000931F90938B0080938A00FF91EF91BF9199
:10CA4000AF919F918F917F916F915F914F913F91A6
:10CA50002F910F900BBE0F900FBE0F901F90189547
:10CA60001F920F920FB60F9211240BB60F921F93C5
:10CA70002F933F934F935F936F937F938F939F93E6
:10CA8000AF93BF93EF93FF93CF93DF9300D01F92A9
:10CA9000CDB7DEB78091D80B0E94559311E0892B5A
:10CAA00009F010E00E94C75A69837A838B839C83C4
:10CAB00089819A81AB81BC814091DC0B5091DD0B67
:10CAC0006091DE0B7091DF0B841B950BA60BB70BEF
:10CAD0002091D90B3091DA0B2430310509F44CC088
:10CAE0002530310521F021303105E9F414C02091C1
:10CAF000DB0B222339F02091460C20FF02C0289A3C
:10CB000001C02898112379F0813E2EE29207A105F9
:10CB1000B10548F02BC0112379F125E030E03093C6
:10CB2000DA0B2093D90B2091D90B3091DA0B2530F9
:10CB3000310511F5E091460CF0E0EE0FFF1FE052D9
:10CB4000F44F9183808389819A81AB81BC818093EA
:10CB5000DC0B9093DD0BA093DE0BB093DF0B809189
:10CB6000460C8F5F8093460C833330F084E090E076
:10CB70009093DA0B8093D90B0F900F900F900F903A
:10CB8000DF91CF91FF91EF91BF91AF919F918F91E5
:10CB90007F916F915F914F913F912F911F910F90D6
:10CBA0000BBE0F900FBE0F901F901895CF93DF9381
:10CBB000EC018091D80B62E00E946758E881F9810E
:10CBC0000190F081E02DCE01DF91CF9119948091F9
:10CBD0001202882311F0599801C0599A90911202BB
:10CBE00081E08927809312020895809141109091ED
:10CBF00042109160909342108093411008951092DA
:10CC00004E0C409146075091470760E070E021E2EA
:10CC100036E680913507909136070C94E63F809177
:10CC20005107882369F080914D0C882349F081E0F9
:10CC300080934A0C809150070E94AA7F0C9458560A
:10CC40000895CF93DF93CDB7DEB765970FB6F8940D
:10CC5000DEBF0FBECDBF81E080934E0C80916C1083
:10CC6000882371F182E390E09A83898388E290E0DF
:10CC70009C838B838EE690E09E838D8384EF91E08E
:10CC800098878F831D8A84E08F938DB79EB74597D1
:10CC90000FB6F8949EBF0FBE8DBFADB7BEB711964D
:10CCA00085E1FE01319601900D928A95E1F788E0C9
:10CCB0009BE00E949EA70FB6F894DEBF0FBECDBFCB
:10CCC00065960FB6F894DEBF0FBECDBFDF91CF9152
:10CCD000089580916210811112C082E297EBA1E069
:10CCE000BB27ABBFFC016791769182E00E940741B0
:10CCF00081E080936F10109273101092701008955D
:10CD000081E0809347106CED75E00C9407416CED69
:10CD100075E080E00C94074161E08BE20E94EF56E1
:10CD2000E89A25E438E548E853E160E070E0809156
:10CD30003507909136070E94E63F9093E30F80936A
:10CD4000E20F089581E20E94559321E0892B09F4B6
:10CD500020E0822F089580914C07882309F44BC06E
:10CD600080914D0C882309F446C081E080934A0CE1
:10CD7000E9DF882329F080914F078823D1F106C08D
:10CD800080914D07811105C080914C070E94AA7FB8
:10CD900030C090914C07963061F5823081F083303D
:10CDA000D1F0813031F5E091620BF091630B749713
:10CDB0008081918145E550E060E070E017C0E0912E
:10CDC000620BF091630B7497808191814AE550E08A
:10CDD00060E070E00BC0E091620BF091630B749720
:10CDE000808191814FE550E060E070E08E59944F72
:10CDF0003DDD0C94585608958091E50F882339F055
:10CE00008091E40F882319F081E08093470C809192
:10CE1000370790913807DC01ED91FC91008CF18D82
:10CE2000E02D19958091681081110E94305D8091EC
:10CE30006710882391F061E08DE00E94EF564091E9
:10CE400065105091661060E070E02FE338E5809146
:10CE50003507909136070E94E63F8091E50F8823C1
:10CE600021F08091E40F811101C075DF8091E40F02
:10CE7000882379F08091E50F882359F080916B1019
:10CE8000882339F0E0916910F0916A1082810E9444
:10CE90005541B5CE80914C0C811157C053DF88238A
:10CEA000F1F081E080934C0C809137079091380726
:10CEB000DC01ED91FC910488F589E02D19950E9423
:10CEC0009B572FEB37E548E95AE360E070E080912B
:10CED0003507909136070E94E63F91DE09C08091A8
:10CEE000E40F882331F18091E50F882311F014DFDE
:10CEF00032CF0E94835D80916B10882339F0E091DE
:10CF00006910F0916A1082810E945541409163102E
:10CF10005091641014161506BCF4052E000C660B17
:10CF2000770B2CEF36E680913507909136070C94FD
:10CF3000E63F80916B10882339F0E0916910F09101
:10CF40006A1082810E94554157CF08950F931F9315
:10CF500020916210211135C042E257EB61E0772742
:10CF60009C01220F331F820F931F092E000CAA0B66
:10CF7000BB0B0296A11DB11D840F951FA61FB71FE5
:10CF8000ABBFFC01879102E217EB21E03327409110
:10CF9000731093E0499FA0011124052E000C660B2D
:10CFA000770B4E5F5F4F6F4F7F4F040F151F261F8C
:10CFB000371F2BBFF8010791801718F01F910F91B1
:10CFC00088CE1F910F910895833091F028F481301D
:10CFD00049F0823051F00895853081F060F086305C
:10CFE00081F0089589E090E00EC08AE090E00BC0E7
:10CFF0008BE090E008C08CE090E005C08DE090E010
:10D0000002C08EE090E0A2CF8F929F92AF92BF922B
:10D01000CF92DF92EF92FF920F931F93CF93DF9304
:10D02000EC01A62E8091621081116BC042E257EB99
:10D0300061E077276E01CC0CDD1CCC0EDD1E0D2CC3
:10D04000000CEE08FF08D701C6010296A11DB11D14
:10D05000480F591F6A1F7B1F6BBFFA01879142E27D
:10D0600057EB61E07727B090731093E0B99E800191
:10D070001124012E000C220B330B0E5F1F4F2F4F7C
:10D080003F4F400F511F621F731F6BBFFA01479143
:10D09000481708F036C0809071109090721000917F
:10D0A0005B1010915C10B401C8010E947F3F88237F
:10D0B00021F0B401C8010E94973F82E297EBA1E002
:10D0C000BB278C0D9D1DAE1DBF1DABBFFC01679125
:10D0D000769182E00E940741B0927010C093731065
:10D0E000AA2079F010926F1029E636E642E350E06C
:10D0F00060E070E0C8010E94E63F90937210809358
:10D100007110DF91CF911F910F91FF90EF90DF9001
:10D11000CF90BF90AF909F908F900895CF92DF9265
:10D12000EF92FF9280916210811134C08091611062
:10D13000882381F161E08EE090E066DF60915F100E
:10D1400070916010CB01A0E0B0E0C0905D10D09075
:10D150005E10E12CF12CC816D906EA06FB0664F431
:10D16000BC01CD016C197D098E099F090E94EE8FCB
:10D17000C60ED71EE81EF91E2EE838E6B701A60136
:10D1800080915B1090915C100E94E63F90935A1042
:10D1900080935910FF90EF90DF90CF900895CF9239
:10D1A000DF92EF92FF9280916210811134C08091E2
:10D1B0005810882381F161E08DE090E025DF6091D7
:10D1C000561070915710CB01A0E0B0E0C090541001
:10D1D000D0905510E12CF12CC816D906EA06FB06B2
:10D1E00064F4BC01CD016C197D098E099F090E9470
:10D1F000EE8FC60ED71EE81EF91E2FEC38E6B701DB
:10D20000A60180915B1090915C100E94E63F909384
:10D21000531080935210FF90EF90DF90CF900895BD
:10D22000CF92DF92EF92FF9280916210811134C011
:10D2300080915110882381F161E08CE090E0E4DE80
:10D2400060914F1070915010CB01A0E0B0E0C09001
:10D250004D10D0904E10E12CF12CC816D906EA06DC
:10D26000FB0664F4BC01CD016C197D098E099F0990
:10D270000E94EE8FC60ED71EE81EF91E20E139E689
:10D28000B701A60180915B1090915C100E94E63F6F
:10D2900090934C1080934B10FF90EF90DF90CF90C5
:10D2A00008958091621081112CC080914A108823CA
:10D2B00041F080915110811104C081E080935110A0
:10D2C000AFDF80914910882361F080916210811155
:10D2D00008C080915810811104C081E080935810DB
:10D2E0005EDF80914810882361F080916210811187
:10D2F00008C080916110811104C081E080936110A9
:10D300000DCF08951092471020E836E644EF51E023
:10D3100060E070E080915B1090915C100E94E63FAD
:10D32000909346108093451008958091621081116A
:10D330000AC080914710882331F060ED77E081E0EA
:10D340000E940741DFCF08950F931F93CF93DF9380
:10D35000EC0170935C1060935B104093621081E06D
:10D3600090E00E94B4CB8C010E94A14210936E10F9
:10D3700000936D1091E09093471090936F1010926E
:10D380004610109245101092721010927110109267
:10D390007310109270101092441024EF31E030930B
:10D3A0004E1020934D1028EB3BE03093501020930B
:10D3B0004F1020E233E030935510209354102CEAA4
:10D3C0003DE0309357102093561028E037E030931B
:10D3D0005E1020935D1024E931E1309360102093BA
:10D3E0005F1010924A10109249101092481010923B
:10D3F0005110109258101092611010924310109218
:10D400004C1010924B101092531010925210109218
:10D410005A1010925910988399839A83DF91CF9173
:10D420001F910F910895FC011282138214821582BC
:10D43000168217821286089580E008950F931F9335
:10D44000CF938C0167E976E181EF99E00E945291D8
:10D45000D8011896ED91FC9119976081718181EF47
:10D4600099E00E94947FC1E0D8011A968C91C81768
:10D4700010F562E976E181EF99E00E9452916C2FFC
:10D4800081EF99E00E9451826FE876E181EF99E0A7
:10D490000E945291F80190858185E92FF82FEC0FB9
:10D4A000F11DEC0FF11D6081718181EF99E00E9407
:10D4B000947FCF5FD9CFCF911F910F910895CF93D4
:10D4C000DF93CDB7DEB7A0970FB6F894DEBF0FBEDF
:10D4D000CDBF80310CF080E027E836E13A83298324
:10D4E00020E836E13C832B8322E736E13E832D831F
:10D4F00026E636E138872F832CE536E13A872987FF
:10D5000022E536E13C872B872EE436E13E872D87E6
:10D5100027E436E1388B2F872CE336E13A8B298BD1
:10D520002FE236E13C8B2B8B24E236E13E8B2D8BB8
:10D5300028E136E1388F2F8B26E036E13A8F298FAC
:10D5400025EF35E13C8F2B8F20EF35E13E8F2D8F7E
:10D5500023EE35E138A32F8FE82FEE0FFF0BEC0FF2
:10D56000FD1F81819281A0960FB6F894DEBF0FBE99
:10D57000CDBFDF91CF910895AF92BF92CF92DF924E
:10D58000EF92FF920F931F93CF93DF9389E790E180
:10D590007EE1D72ED80ECC24C39402E010E0C3E085
:10D5A000D0E0E2E0BE2EEE24E394F12C8091B20FA5
:10D5B0009091B30FDC01ED91FC910084F185E02D99
:10D5C0001995892B09F4ADC0A09030018091B20F5C
:10D5D0009091B30FDC01ED91FC910284F385E02D75
:10D5E000199596B3B39A2091840030918500285AFA
:10D5F000344E30938D0020938C002A2D2C7119F01D
:10D6000010929C0F4BC093FB992790F9E0919C0FCF
:10D61000E11116C0992351F2803241F6C0929C0F5D
:10D62000809379108091D40F9091D50F892B09F0B8
:10D63000BDCFF092D50FE092D40F10929E0FB6CFCF
:10D640009111DECFE13041F4803409F0AFCFB092D8
:10D650009C0F80937A10E6CF91E09E0F90939C0FE1
:10D66000F0E0E758FF4E8083903209F09FCF109290
:10D670009C0FE9E7F0E12FEF3FEF8191281B310983
:10D68000DE12FBCF409197108091981090E0982F78
:10D690008827840F911D2817390729F0D093D50FBB
:10D6A000C093D40F83CF8091D40F9091D50F019761
:10D6B00039F480919E0F8F5F80939E0F843020F00D
:10D6C0001093D50F0093D40F80919D0F8F5F80939F
:10D6D0009D0F90919B0F981708F5C092D60F20E0F0
:10D6E00030E0F901E758FF4E4281838190E0982FA6
:10D6F0008827840F911DAC014F5E52404B3D554031
:10D7000028F4F901EC54F04F918380832E5F3F4F52
:10D710002C31310531F710929D0F48CF1092D60F62
:10D7200045CFDF91CF911F910F91FF90EF90DF9048
:10D73000CF90BF90AF900895EF92FF920F931F93F9
:10D74000CF93DF931092A71282E08093A81268EE25
:10D7500073E07093AA126093A91240ED57E05093C2
:10D76000AC124093AB122CED35E03093AE12209307
:10D77000AD128FE08093AF121092B01294E09093AC
:10D78000B1127093B3126093B2125093B5124093DA
:10D79000B4123093B7122093B6128093B81210923D
:10D7A000B91293E09093BA127093BC126093BB12BB
:10D7B0005093BE124093BD123093C0122093BF12FB
:10D7C0008093C1121092C21291E09093C312709391
:10D7D000C5126093C4125093C7124093C61230937F
:10D7E000C9122093C8128093CA121092CB12ECEC8B
:10D7F000F2E1A5EDB2E180E008EE13E060ED77E044
:10D800004CED55E031E022E095E0980F90831283D3
:10D8100001837483638356834583ED01229791E0EE
:10D820003883219628831C928F5F3A961A968C3003
:10D8300059F7109244139093451310924613909306
:10D8400047138AE892E0909349138093481390938A
:10D850004B1380934A1380E090E09C0129553D4E84
:10D86000F901EB55FF4F1182108232961082039618
:10D870008837910591F784E290E090934D1380935F
:10D880004C1381E080934E132CE030E03093501322
:10D8900020934F1394E09093511321E230E03093A2
:10D8A00053132093521327E02093541329E030E0C0
:10D8B000309356132093551320E1209357137AE0A9
:10D8C0007093C4132BE02093C5132093C61348EE26
:10D8D00053E05093C8134093C71320ED37E03093C3
:10D8E000CA132093C9131092CB1364E66093CC1330
:10D8F0006093CD135093CF134093CE133093D11335
:10D900002093D0131092D2135093D4134093D31377
:10D910003093D6132093D5131092D7131092D813A7
:10D920008093D9131092DB131092DA138093DC13D7
:10D930008093DD13E8ECF0E0F093DF13E093DE1367
:10D94000E0E2F3E0F093E113E093E0135093E3138C
:10D950004093E2133093E5132093E4131092E613FF
:10D960008093E713E9E5F0E0F093E913E093E8131F
:10D97000E0E8F0E0F093EB13E093EA13EFEFF0E070
:10D98000F093ED13E093EC13F093EF13E093EE13A9
:10D990001092F0131092F113F093F313E093F2133B
:10D9A000F093F513E093F413F093F713E093F61369
:10D9B0001092F8138093F9139093FA131092FB13BB
:10D9C0008093FC139093FD131092FE131092FF139B
:10D9D0008093001410920114109202148093031487
:10D9E0001092041498E290930514509307144093F6
:10D9F0000614509309144093081430930B14209389
:10DA00000A1480930C1492E390930D14E2E0E093D7
:10DA10000E1480930F1460931014E6E4E093111435
:10DA2000909312141092131410921414109215144F
:10DA3000109216141092171410921814EAEFF0E0D6
:10DA4000F0931A14E093191410921B1410921C14E2
:10DA500060931D1460931E1410921F149093201451
:10DA60001092211490932214EEE5F1E0F093241427
:10DA7000E093231410922514ACEDB5E0B093271475
:10DA8000A093261400EA1FE0109329140093281491
:10DA900030932B1420932A14C8E8D3E1D0932D148B
:10DAA000C0932C1468EBE62E6BE0F62EF0922F1448
:10DAB000E0922E14E0E4FFE1F0933114E09330148F
:10DAC00010923214109233141092341469E160935E
:10DAD0003514809336148093371480933814509300
:10DAE0003A144093391430933C1420933B14F09231
:10DAF0003E14E0923D141093401400933F14D093D1
:10DB00004214C093411420E737E13093441420932A
:10DB10004314109245141092461410924714909397
:10DB200048149093491490934A1410924B141092F5
:10DB30004C1410924D1480934E1410924F1499E08F
:10DB40009093501410925114109252141092531436
:10DB500010925414B0935614A0935514F093581483
:10DB6000E09357148093591470935A1410925B14D5
:10DB700021E030E030935D1420935C1410925E1429
:10DB800040E052EC61E070E040935F145093601409
:10DB900060936114709362144093631450936414FF
:10DBA000609365147093661440E056E960E070E09D
:10DBB00040936714509368146093691470936A14C7
:10DBC00040936B1450936C1460936D1470936E14A7
:10DBD00010926F1420E039E1309371142093701487
:10DBE000109272149EE190937314109274142EE1AB
:10DBF00030E030937614209375143093781420938A
:10DC0000771430937A142093791490937B14909323
:10DC10007C1480937D1480937E1410927F149093D3
:10DC20008014809381149CE09093821480938314D9
:10DC300080EF9FEBA0E0B0E0809384149093851474
:10DC4000A0938614B093871407EA12E1C0E0D0E0F5
:10DC5000CE010E9464C9F80161918F01861719F005
:10DC6000CE010E9476C92196C13EF1E0DF0781F71F
:10DC7000DF91CF911F910F91FF90EF9008954F92F8
:10DC80005F926F927F928F929F92AF92BF92CF924C
:10DC9000DF92EF92FF92CF93DF93EB01A091771089
:10DCA000B09178109D012F5F3F4F45E0429F2001CA
:10DCB000439F500C1124052C000C66087708812C1A
:10DCC000912C54012B34E1E03E07ECF445E557EB91
:10DCD00061E0772775016401C40CD51CE61CF71CB4
:10DCE0004C0D5D1D6E1D7F1D6BBFFA014791569156
:10DCF00065E0860E911CA11CB11CC417D50729F143
:10DD00002F5F3F4FDFCF25E0822E912CA12CB12C2D
:10DD100021E030E0A217B30708F44CC045E557EB0B
:10DD200061E07727480D591D6A1D7B1D6BBFFA0105
:10DD300047915691F5E08F0E911CA11CB11CC417A0
:10DD4000D50719F02F5F3F4FE5CF45E557EB61E071
:10DD50007727E5E0E29F6001E39FD00C11240D2CB2
:10DD6000000CEE08FF084E5F5F4F6F4F7F4F4C0D6A
:10DD70005D1D6E1D7F1D6BBFFA0147915691FC0121
:10DD80005383428345E557EB61E077274C5F5F4F54
:10DD90006F4F7F4FC40ED51EE61EF71EEBBEF60179
:10DDA000C790FC01C4823093781020937710C9018A
:10DDB000019606C0109278101092771080E090E0E3
:10DDC000DF91CF91FF90EF90DF90CF90BF90AF9019
:10DDD0009F908F907F906F905F904F9008951F92CB
:10DDE0000F920FB60F9211242F938F939F9310923F
:10DDF0009500109294008091560C8F5F8093560C82
:10DE000090910C15891784F01092560C2091580CA3
:10DE100080910A1590910B15820F911D27FD9A95FF
:10DE200090930B1580930A158091550C8F5F80930A
:10DE3000550C90917610891784F01092550C209112
:10DE4000570C8091741090917510820F911D27FDD1
:10DE50009A9590937510809374109F918F912F9144
:10DE60000F900FBE0F901F901895CF92DF92EF92F8
:10DE7000FF920F931F93CF93DF93CDB7DEB76597D4
:10DE80000FB6F894DEBF0FBECDBF8C01FC018585B7
:10DE90008823E1F082899389892B09F44EC10E947D
:10DEA000245BF801C080D180E280F380AB01BC012B
:10DEB0004C195D096E097F0982899389A0E0B0E061
:10DEC00084179507A607B70728F137C1F8018085A1
:10DED0009185892B09F494C00E94245BF801C480C9
:10DEE000D580E680F780AB01BC014C195D096E0955
:10DEF0007F0980859185A0E0B0E084179507A6078B
:10DF0000B70708F07DC0C8010E948AA7C8010E9417
:10DF100079A7B9C0F8018685978501969787868786
:10DF2000608971898617970768F580E090E00E9404
:10DF30003FC89B01AC016BED7FE089E490E40E9457
:10DF400046CAF80122A533A544A555A50E94E2C9F9
:10DF5000F80162A773A784A795A70E94E3CA20E0EF
:10DF600030E04FEF52E40E94A0C820E030E04FEFD5
:10DF700052E40E94E2C90E94AECAF80182850E9462
:10DF8000A35870C0F8018585823021F4C8010E9431
:10DF90008AA779C0F80186A5882309F474C0C8014E
:10DFA0000E9467A782E390E09A83898388E290E0E9
:10DFB0009C838B838EE690E09E838D8384EF91E03B
:10DFC00098878F831D8A84E08F938DB79EB745977E
:10DFD0000FB6F8949EBF0FBE8DBFADB7BEB71196FA
:10DFE00085E1FE01319601900D928A95E1F7C80115
:10DFF0000E949EA70FB6F894DEBF0FBECDBF9DC096
:10E00000F80182899389892B09F497C00E94245BC7
:10E01000F801C080D180E280F380AB01BC014C19D3
:10E020005D096E097F0982899389A0E0B0E08417B9
:10E030009507A607B70708F080C0F8018685978581
:10E04000019697878687208931898217930708F080
:10E0500053C080FF29C0C8010E948AA7F8018489A3
:10E06000882331F1C80165960FB6F894DEBF0FBE64
:10E07000CDBFDF91CF911F910F91FF90EF90DF9077
:10E08000CF900C94D27EC80165960FB6F894DEBF8F
:10E090000FBECDBFDF91CF911F910F91FF90EF90F9
:10E0A000DF90CF900C9467A7C8010E9494A7D6CFA9
:10E0B000868597858B309105A0F0C8010E948AA7BC
:10E0C000C80165960FB6F894DEBF0FBECDBFDF91D5
:10E0D000CF911F910F91FF90EF90DF90CF900C9414
:10E0E00079A7880F991FF801E80FF91F858996898C
:10E0F000F801938B828BB6CFF80181A5882351F06C
:10E1000085899689938B828B17861686C8010E9413
:10E1100094A7A8CFF80186A5882379F216A682E0F5
:10E120008587C8010E9479A784E690E0F801918B69
:10E13000808B87A590A9938B828B65960FB6F894F8
:10E14000DEBF0FBECDBFDF91CF911F910F91FF902A
:10E15000EF90DF90CF9008952F923F924F925F9271
:10E160006F927F928F929F92AF92BF92CF92DF92E7
:10E17000EF92FF920F931F93CF93DF9300D01F92E4
:10E18000CDB7DEB75C010E94A54E0E94294C0E94CB
:10E19000604C80918E1490918F140E945A900E942E
:10E1A000BC6124E0A216B10409F49CC00CF04FC07D
:10E1B000A3E0AA16B10409F03CC18CE190E00E94F2
:10E1C000B4CB9C838B8381E796E0AB81BC811196B5
:10E1D0009C938E931396BC92AE92129781E09FEF20
:10E1E00015969C938E9314978FEF90E017969C93BF
:10E1F0008E93169719961C921E92189758961C92F9
:10E200005897CD010E94A14285E696E0EB81FC8102
:10E2100091838083E091770FF091780FD08C0091FB
:10E22000291210912A1216950795E0902712F09066
:10E230002812F694E79462EC77E180918E14909125
:10E240008F140E947691812C9924939412C1B5E089
:10E25000AB16B10409F4A6C0E6E0AE16B10409F0AD
:10E26000E8C08CE190E00E94B4CB9C838B8381E773
:10E2700096E0AB81BC8111969C938E931396BC92D1
:10E28000AE92129781E09FEF15969C938E93149710
:10E290008FEF90E017969C938E93169719961C9289
:10E2A0001E92189758961C925897CD010E94A14231
:10E2B00085E696E0EB81FC8191838083E091B50750
:10E2C000F091B607D08C00916812109169121695E2
:10E2D0000795E0906612F0906712F694E79465EF68
:10E2E00077E1A0C08CE190E00E94B4CB9C838B834B
:10E2F00081E796E0AB81BC8111969C938E93139637
:10E30000BC92AE92129781E09FEF15969C938E93EC
:10E3100014978FEF90E017969C938E93169719960B
:10E320001C921E92189758961C925897CD010E94E5
:10E33000A14285E696E0EB81FC8191838083009188
:10E340003E1210913F1216950795E0903C12F09006
:10E350003D12F694E7948091C6138C50823040F4BD
:10E36000E091C607F091C707D08C65E378E15AC009
:10E3700080910F14823009F07AC08091C4138C30E0
:10E3800009F075C0E091B507F091B607D08C65E152
:10E3900078E180918E1490918F140E947691882458
:10E3A000839466C08CE190E00E94B4CB9C838B8305
:10E3B00081E796E0AB81BC8111969C938E93139676
:10E3C000BC92AE92129781E09FEF15969C938E932C
:10E3D00014978FEF90E017969C938E93169719964B
:10E3E0001C921E92189758961C925897CD010E9425
:10E3F000A14285E696E0EB81FC8191838083E091E8
:10E40000C207F091C307D08C00915312109154129F
:10E4100016950795E0905112F0905212F694E794F9
:10E4200065ED77E180918E1490918F140E94769122
:10E430001EC069EA77E180918E1490918F140F903D
:10E440000F900F900F90DF91CF911F910F91FF9040
:10E45000EF90DF90CF90BF90AF909F908F907F9084
:10E460006F905F904F903F902F900C947691812CFD
:10E47000912C0E94BC616CE977E180918E1490919F
:10E480008F140E94769160E977E180918E149091CB
:10E490008F140E945291B80180918E1490918F1424
:10E4A0000E94398464E877E180918E1490918F14F2
:10E4B0000E945291B70180918E1490918F140E9406
:10E4C000398468E777E180918E1490918F140E94CF
:10E4D00052918D2D0E94926180918E1490918F1493
:10E4E0000E945A90AB81BC81ED91FC911197028002
:10E4F000F381E02DCD011995CA2C8A2D0E94BE41D1
:10E500008D3D9540A8F464E378E08A2D0E94B641E1
:10E51000EB81FC81F78AE68AB70182810E94CE41B5
:10E520006CED75E08A2D0E94BA41DD20C1F01AC061
:10E5300064E873E08A2D0E94BA41AB81BC81579692
:10E540001C930E935697B80112968C910E94CE415F
:10E550006CED75E08A2D0E94B641DD2019F0332460
:10E56000339401C0312C21E02983212C2A830E947D
:10E57000C8508091D211882359F1AB81BC81ED91B3
:10E58000FC9111976091D7117091D8110190F08191
:10E59000E02DCD0119958C2D0E94BE418D3DB5E039
:10E5A0009B075CF48438E3E09E0784F08C018D3D8A
:10E5B000954074F00CED15E00BC07C01853398405C
:10E5C0003CF064E3E62E68E0F62E02C004E813E0B7
:10E5D0002A8121111FC08091C8118823C9F1E091BF
:10E5E000CF11F091D011858196814091CB1150913E
:10E5F000CC119C0121533109421753074CF1C196AC
:10E60000841795072CF10E94245B64157505860517
:10E610009705F0F08091C8118823C1F04091CB118B
:10E620005091CC11E091CF11F091D011858196815C
:10E630009C01285C3109421753072CF088539F4FE7
:10E64000841795071CF481E0382605C021E02A8351
:10E65000222009F47CC0332009F445C0DD20F9F004
:10E6600064E873E08C2D0E94BA41992009F458C0E7
:10E670006091E0137091E11341E08C2D0E9475418F
:10E680000E94C9A0AB81BC8112968C910E94BE41B0
:10E6900008171907ACF38C2D0E94474141C064E371
:10E6A00078E08C2D0E94B6419920B1F06091E01382
:10E6B0007091E11340E08C2D0E9475410E94C9A029
:10E6C000AB81BC8112968C910E94BE418E159F0534
:10E6D000ACF38C2D0E944741EB81FC81F78AE68ADE
:10E6E000B701828110C0DD20B1F064E378E08C2DA9
:10E6F0000E94B641AB81BC815796FC92EE92569730
:10E70000B70112968C910E94CE416CED75E08C2D74
:10E710000E94BA4112C064E873E08C2D0E94BA4195
:10E72000EB81FC81178B068BB80182810E94CE4160
:10E730006CED75E08C2D0E94B6410E94245B2B018C
:10E740003C01F8EC4F0E511C611C711C1A8229818E
:10E750002223D9F18091BE118823A9F14091C111E2
:10E760005091C211E091C511F091C6118581968139
:10E770009C01285C3109421753072CF088539F4FA6
:10E780008417950704F581E0D82680918E14909126
:10E790008F14DD2039F069E677E10E94769182E0FE
:10E7A00090E006C067E577E10E94769181E090E015
:10E7B0000E94314C0E94245BAB81BC815896DC9254
:10E7C0002224239403C0212C1EC0212C8091BE1131
:10E7D000882309F48AC2E091C511F091C6118581A0
:10E7E00096814091C1115091C2119C012153310970
:10E7F000421753070CF479C2C19621E0298384178C
:10E8000095070CF472C20E94B4440E94818389ED82
:10E810009CE00E94F63F8091660C882309F4A7CE05
:10E820008091680C882309F4A2CE0E9481830E9403
:10E8300088848823D1F384E0A816B104D9F134F494
:10E84000B3E0AB16B10409F438C1C4C1E5E0AE16BB
:10E85000B10409F4CDC0F6E0AF16B10409F0BAC1B5
:10E860001093D4130093D313F092D613E092D513E0
:10E87000D092D713B8018CE291E00E941283B701C5
:10E880008EE291E00E9412836D2D80E391E00E9460
:10E890006E84B80186E00E94EC40B70186E00E94D9
:10E8A000D140E091B507F091B607D08E6CED75E0E0
:10E8B00086E091C08820C1F01093D4130093D31345
:10E8C000F092D613E092D513D092D713B8018CE210
:10E8D00091E00E941283B7018EE291E00E941283C0
:10E8E0006D2D80E391E017C01093C8130093C713F8
:10E8F000F092CA13E092C913D092CB13B80180E210
:10E9000091E00E941283B70182E291E00E9412839B
:10E910006D2D84E291E00E946E84B80184E00E9433
:10E92000EC40B70184E00E94D140882049F0E0919A
:10E93000B507F091B607D08E6CED75E084E04BC062
:10E94000E091C607F091C707D08E8091C6138D3035
:10E9500029F4E0919A10F0919B10D08E6CED75E047
:10E9600084E00E94CE4166E970E080E090E00E9481
:10E97000EC5A8091C6138D3011F584E00E94BE419F
:10E98000A091C607B091C7078D3D95404CF0ED9121
:10E99000FC9111970190F081E02D6FEF7FEF08C09F
:10E9A000ED91FC9111970190F081E02D61E070E014
:10E9B000CD0119958091C6079091C7076FC08091CE
:10E9C000C6079091C707DC01ED91FC910480F581A9
:10E9D000E02D1995FFC00E94CE4166E970E080E00D
:10E9E00090E00E94EC5A8091B5079091B607EBCF6A
:10E9F0001093CF130093CE13F092D113E092D01363
:10EA0000D092D213B80187E291E00E941283B7013D
:10EA100089E291E00E9412836D2D8BE291E00E94C9
:10EA20006E84B80185E00E94EC40B70185E00E9449
:10EA3000D140E091C207F091C307D08E6CED75E034
:10EA400085E00E94CE4166E970E080E090E00E949F
:10EA5000EC5A8091C5138D3059F585E00E94BE4176
:10EA6000A091C207B091C3078D3D95404CF0ED9148
:10EA7000FC9111970190F081E02D6FEF7FEF08C0BE
:10EA8000ED91FC9111970190F081E02D61E070E033
:10EA9000CD0119958091C2079091C307DC01ED91DA
:10EAA000FC910190F081E02D60E070E0199592C03A
:10EAB0008091C2079091C30786CF1093E313009310
:10EAC000E213F092E513E092E413D092DC13B80164
:10EAD0008BE391E00E941283B7018DE391E00E94E5
:10EAE00012836D2D85E391E00E946E84B80183E06E
:10EAF0000E94EC40B70183E00E94D1408091DC137A
:10EB0000E091770FF091780F808F8091DC130E9455
:10EB1000DD8283E00E94BE412091DC13222369F153
:10EB2000B9E0BC1538F02091291230912A1236959F
:10EB3000279502C02EEE32E08217930709F44AC0EF
:10EB40006091E0137091E11341E083E00E94754110
:10EB50000E94C9A0EB81FC8182810E94BE410817FE
:10EB60001907B4F383E00E944741AB81BC815796FB
:10EB70001C930E935697B80129C0A9E0AC1508F470
:10EB8000B6C020912712309128123695279582170A
:10EB9000930701F16091E0137091E11340E083E08D
:10EBA0000E9475410E94C9A0EB81FC8182810E9474
:10EBB000BE418E159F05B4F383E00E944741AB81AF
:10EBC000BC815796FC92EE925697B70112968C91A3
:10EBD0000E94CE4180918E1490918F140E945A9081
:10EBE0000E94BC61B4E0AB16B10499F03CF4F3E0D0
:10EBF000AF16B10449F56BED76E120C025E0A21611
:10EC0000B104D1F086E0A816B104F1F46BE077E12D
:10EC100015C08091C6138C50823018F46DE377E1F3
:10EC20000DC080910F14823079F48091C4138C3020
:10EC300059F464E277E102C062EF76E180918E14CC
:10EC400090918F140E9476910E94BC6160ED76E1F4
:10EC500080918E1490918F140E94769164EC76E1ED
:10EC600080918E1490918F140E945291B8018091DE
:10EC70008E1490918F140E94398468EB76E1809114
:10EC80008E1490918F140E945291B70180918E142E
:10EC900090918F140E9439846CEA76E180918E14F1
:10ECA00090918F140E9452918D2D0E9492618091BB
:10ECB0008E1490918F140E945A900F900F900F9085
:10ECC0000F90DF91CF911F910F91FF90EF90DF9008
:10ECD000CF90BF90AF909F908F907F906F905F90FC
:10ECE0004F903F902F900C945C4C19828CCD2AEC65
:10ECF00038E04DCFCF93DF93CDB7DEB728970FB66F
:10ED0000F894DEBF0FBECDBF809199108823E1F14A
:10ED1000109299100E94D34C81E08093030280915D
:10ED2000C807882389F16DE976E180918E1490916E
:10ED30008F140E945291E091620CE4300CF0E0E0FC
:10ED400080EF95E09A8389838CEE95E09C838B839A
:10ED500087EE95E09E838D8382EE95E098878F8382
:10ED6000EE0FFF0BEC0FFD1F6181728180918E14FD
:10ED700090918F1428960FB6F894DEBF0FBECDBFCA
:10ED8000DF91CF910C94769128960FB6F894DEBF60
:10ED90000FBECDBFDF91CF9108958091C4079091B0
:10EDA000C507DC01ED91FC910084F185E02D1995FA
:10EDB0008091C4079091C507DC01ED91FC9104801E
:10EDC000F581E02D199480910702813019F485E0D6
:10EDD0008093070208951092C007089580912D072F
:10EDE000882371F010922D0780919014882341F0B0
:10EDF0006AE67AE180918E1490918F140C9476914A
:10EE0000089580910F14833099F080912D0781111E
:10EE10000FC081E080932D0780919014882341F0EA
:10EE200065E57AE180918E1490918F140C9476911F
:10EE3000089580912C07833079F083E080932C072C
:10EE400080919014882341F064E47AE180918E14DB
:10EE500090918F140C947691089580912C078230B4
:10EE600079F082E080932C0780919014882341F000
:10EE700063E37AE180918E1490918F140C947691D3
:10EE8000089580912C07813079F081E080932C07E0
:10EE900080919014882341F062E27AE180918E148F
:10EEA00090918F140C9476910895809192148823F8
:10EEB00071F00E94588280919014882341F062EE94
:10EEC00079E180918E1490918F140C94769108952D
:10EED0008091470C8823C1F06091750F7091760F77
:10EEE00089ED9CE00E94973F1092760F1092750F6B
:10EEF0001092470C809107028130D9F480911C1444
:10EF00008823B9F060DF15C080919C108F5F8093DB
:10EF10009C10803580F06091750F7091760F89EDAF
:10EF20009CE00E94973F1092760F1092750F1092FE
:10EF3000470C10929C10089580919214882339F107
:10EF400080918914882319F1109289140E9413A0CA
:10EF500080918814882319F0109288140CC0809135
:10EF6000C4079091C507DC01ED91FC910288F389FB
:10EF7000E02D60E0199580919014882341F06BE0BA
:10EF80007AE180918E1490918F140E947691109264
:10EF900089140895CF93909192149923D1F190916F
:10EFA0004C0C911136C090918914911132C0C82F28
:10EFB00081E0809389148091C310882331F081E02F
:10EFC0000E9462A01092C31002C00E9422A08091F1
:10EFD0008814882319F0109288140CC08091C407FB
:10EFE0009091C507DC01ED91FC910288F389E02D39
:10EFF00061E0199580919014882359F0CC2349F051
:10F0000067EF79E180918E1490918F14CF910C94D9
:10F010007691CF91089581E0BDCFCF93DF93C091DA
:10F02000C110D091C210BE0189ED9CE00E947F3FCB
:10F03000882329F0BE0189ED9CE00E94973F109241
:10F04000C2101092C110DF91CF910895CF92DF923C
:10F05000EF92FF920F931F93CF93DF93C0901414FE
:10F06000D0901514E0901614F09017141C141D0481
:10F070001E041F040CF040C080919214882399F163
:10F080000091C1101091C210B80189ED9CE00E945E
:10F090007F3F8823D9F0E7EDFEE0C0E0D0E081912A
:10F0A00091918017910769F40E94245BCC0FDD1FBA
:10F0B000CC0FDD1FC752D34F688379838A839B832C
:10F0C0001BC02196CE31D10551F716C025E537E793
:10F0D000B701A60189ED9CE00E94E63F9093C21023
:10F0E0008093C11009C0DF91CF911F910F91FF90C4
:10F0F000EF90DF90CF9091CFDF91CF911F910F9143
:10F10000FF90EF90DF90CF9008950F931F93809121
:10F11000140281111EC00E94245B0091BD10109149
:10F12000BE102091BF103091C010AB01BC01401B3C
:10F13000510B620B730B8091081490910914A0E09D
:10F14000B0E0481759076A077B0718F081E0809301
:10F1500014021F910F910895809108149091091441
:10F16000892B89F080911402882381F00E94245B0E
:10F170006093BD107093BE108093BF109093C01029
:10F1800010921402089581E0809314020895CF92A2
:10F19000DF92EF92FF92CF93DF9380914C0C81111D
:10F1A0007AC18091C107823040F080919014882309
:10F1B00009F471C160EA79E191C08091F01388236C
:10F1C00009F498C080910E08882309F493C08091B7
:10F1D000911481118FC08091F813882359F1809187
:10F1E000A2129091A312A091A412B091A512892B02
:10F1F0008A2B8B2BF9F00E94245BC090A212D09036
:10F20000A312E090A412F090A5129B01AC012C195E
:10F210003D094E095F0969017A012091F81330E038
:10F22000A8EEB3E00E94D2C9C616D706E806F906D2
:10F2300008F460C0C0914307D091440789AD9AADEE
:10F24000892B11F01AAE19AE8BA9813009F06FC06D
:10F250008FEF90E09093AD008093AC009F8F8E8FE6
:10F260000E94245B6DAB7EAB8FAB98AF8091C407DF
:10F270009091C507DC01ED91FC910284F385E02DAE
:10F28000199581E08093911420910E0830E0A8EE4A
:10F29000B3E00E94D2C9AB01BC0127EC38E789ED8D
:10F2A0009CE00E94E63F90938D1480938C14809193
:10F2B0009014882309F4EFC06EE679E180918E14F2
:10F2C00090918F140E94529160910E0880918E143B
:10F2D00090918F140E94518265E679E180918E149D
:10F2E00090918F14DF91CF91FF90EF90DF90CF90AE
:10F2F0000C9476910ADF80911402882309F4CBC024
:10F30000809192148111C7C081E080939214809300
:10F31000140222DF809190148823A1F06BE179E13F
:10F3200080918E1490918F140E9476910BC0823040
:10F3300009F096CF4FEF60E0CE010E94543D8FEF71
:10F3400090E08CCF80919114811136C08091F013A0
:10F35000882391F180910E08882371F18091F81330
:10F36000882351F18091A2129091A312A091A4122E
:10F37000B091A512892B8A2B8B2BF1F00E94245B74
:10F38000C090A212D090A312E090A412F090A51207
:10F390009B01AC012C193D094E095F0969017A01F5
:10F3A0002091F81330E0A8EEB3E00E94D2C9C6164F
:10F3B000D706E806F906D8F11092911480918A14C4
:10F3C00090918B14806190938B1480938A14809118
:10F3D000C4079091C507DC01ED91FC910280F38197
:10F3E000E02D19958091C10781111AC040910A142E
:10F3F00050910B1481E0809388144115510561F000
:10F4000060E070E02BE038E789ED9CE00E94E63F89
:10F4100080E00E9462A004C08093C31080E0BADD47
:10F42000DF91CF91FF90EF90DF90CF900FCE60E50E
:10F4300079E180918E1490918F140E9452910E94D4
:10F44000245BC090A212D090A312E090A412F0907E
:10F45000A5126C197D098E099F0928EE33E040E062
:10F4600050E00E94B0C9BA01A90121E080918E1438
:10F4700090918F140E9412906AE279E180918E142B
:10F4800090918F140E94529180918E1490918F14BC
:10F490000E945A9091CFDF91CF91FF90EF90DF9033
:10F4A000CF900895AF92BF92CF92DF92EF92FF92EA
:10F4B0000F931F93CF93DF939091B51091110BC0D1
:10F4C0002091CD073091CE073093B4102093B31024
:10F4D00091E09093B5109091AB1091110BC02091D9
:10F4E000CB073091CC073093AA102093A91091E05C
:10F4F0009093AB10A090B310B090B4100091A910ED
:10F500001091AA10D0919014843608F046C0C82FEC
:10F51000682F70E080E090E00E943FC820E030E07B
:10F5200048EC52E40E9446CA6B017C01B501BB0C59
:10F53000880B990B0E9441C89B01AC01C701B60121
:10F540000E94A0C80E94AECA7093CE076093CD07F8
:10F55000B801110F880B990B0E9441C89B01AC01A7
:10F56000C701B6010E94A0C80E94AECA7093CC0722
:10F570006093CB07DD2369F16AEF78E180918E1407
:10F5800090918F140E9452916C2F80918E149091C3
:10F590008F1487D768EF78E10CC0B092CE07A092A5
:10F5A000CD071093CC070093CB07DD2391F06CE0DF
:10F5B00079E180918E1490918F14DF91CF911F91FA
:10F5C0000F91FF90EF90DF90CF90BF90AF900C9491
:10F5D0007691DF91CF911F910F91FF90EF90DF9087
:10F5E000CF90BF90AF900895CF93823069F49091FF
:10F5F000031420910014309104144091011450918F
:10F6000002146091FF130CC09091FD132091FA1326
:10F610003091FE134091FB135091FC136091F9134C
:10F620006093111550930E1540930F1530930D15DF
:10F630002093101590931215909100028917B1F044
:10F640008093000290919014992381F0C82F6FED60
:10F6500078E180918E1490918F140E9452916C2FBA
:10F6600080918E1490918F14CF9104C7CF910895FB
:10F67000833079F030F4813051F0823091F48BE3B3
:10F680000BC0843041F0853061F482E405C08CE326
:10F6900003C080E401C081E40E94559321E0892BDE
:10F6A00009F420E0822F0895E3DF91E0892708958F
:10F6B0000F931F938091A11081110DC00E94245BB4
:10F6C00060939D1070939E1080939F109093A01054
:10F6D00081E08093A110809113028A3AF1F485E0D1
:10F6E000C7DF882371F084E599E090932A15809311
:10F6F000291590938F1480938E148FEF80931302AB
:10F700000CC081EF99E090932A158093291590936E
:10F710008F1480938E14109213020E94245B009128
:10F720009D1010919E1020919F103091A010DC012F
:10F73000CB01801B910BA20BB30BC397A105B105A5
:10F7400008F449C00E94245B60939D1070939E1042
:10F7500080939F109093A01085E08ADF882321F08A
:10F7600080911302882349F085E082DF811133C044
:10F77000809113028F3F79F518C084E599E090934A
:10F780002A158093291590938F1480938E1480915D
:10F790009014882331F065EC78E184E599E00E94CB
:10F7A00076918FEF8093130216C081EF99E09093CA
:10F7B0002A158093291590938F1480938E1480912D
:10F7C0009014882331F060EB78E181EF99E00E949A
:10F7D0007691109213021F910F9108951092E40FE9
:10F7E00080919014882379F02091D81380918E1401
:10F7F00090918F14222319F060E878E102C063E948
:10F8000078E10C947691089581E08093E40F8091E3
:10F810009014882379F02091D81380918E149091C0
:10F820008F14222319F062E578E102C064E678E1E2
:10F830000C94769108950895089508950895089573
:10F84000623039F0633041F0613041F440934A1046
:10F8500008954093491008954093481008956230E8
:10F8600069F06330A1F06130D1F450934E104093B1
:10F870004D103093501020934F1008955093551011
:10F88000409354103093571020935610089550937E
:10F890005E1040935D103093601020935F100895C8
:10F8A000FC01858108950895089508950895209193
:10F8B0006210211102C0FC01628308952091621040
:10F8C000211102C0FC01648308952091621021116E
:10F8D00002C0FC0163830895089508958091621029
:10F8E000811102C00C9480660895089580E0089507
:10F8F00008950895089508950895089580916210D7
:10F90000811104C08FE090E00C94A66708952091C7
:10F910006210211108C0FC018481882321F082E05B
:10F9200090E00C94A667089520916210211108C000
:10F93000FC018381882321F081E090E00C94A6678C
:10F94000089580916210811104C08BE090E00C94C6
:10F95000A667089580916210811105C060E080E182
:10F9600090E00C940468089580916210811105C0A4
:10F9700060E08FE090E00C9404680895809162103C
:10F98000811127C06330A1F028F4613049F0623062
:10F9900059F008956530A1F078F06630A9F0089527
:10F9A00060E089E090E013C060E08AE090E00FC082
:10F9B00060E08BE090E00BC060E08CE090E007C07E
:10F9C00060E08DE090E003C060E08EE090E00C9499
:10F9D0000468089580916210811127C06330A1F0FE
:10F9E00028F4613049F0623059F008956530A1F093
:10F9F00078F06630A9F0089561E089E090E013C0E6
:10FA000061E08AE090E00FC061E08BE090E00BC025
:10FA100061E08CE090E007C061E08DE090E003C021
:10FA200061E08EE090E00C940468089520916210EB
:10FA3000211109C0FC018281882329F061E088E05E
:10FA400090E00C940468089520916210211109C07F
:10FA5000FC018481882329F061E082E090E00C942D
:10FA60000468089520916210211109C0FC0183816E
:10FA7000882329F061E081E090E00C940468089507
:10FA800080916210811105C061E086E090E00C94E5
:10FA90000468089580916210811105C060E08BE0D8
:10FAA00090E00C940468089580916210811105C063
:10FAB00061E087E090E00C94046808958091621002
:10FAC000811105C061E085E090E00C940468089520
:10FAD00080916210811105C061E08AE090E00C9491
:10FAE00004680895CF93DF93FC0125812223A1F1BF
:10FAF000EC018091621081112EC060914B107091C9
:10FB00004C1080915B1090915C100E94973F109276
:10FB100051108091621081110CC06091521070914F
:10FB2000531080915B1090915C100E94973F10924F
:10FB300058108091621081110CC060915910709121
:10FB40005A1080915B1090915C100E94973F109228
:10FB50006110109243101D82DF91CF910895CF93D1
:10FB6000DF93FC01258121111EC0EC018091621000
:10FB7000811117C080914310811113C021E539E62E
:10FB800048EB5BE060E070E080915B1090915C106E
:10FB90000E94E63F90934C1080934B1081E080933D
:10FBA000431081E08D83DF91CF910895862F90914E
:10FBB0006210911102C00C94E4670895CF93C1E0E4
:10FBC00080916210811103C08C2F0E94E467CF5F87
:10FBD000C730B1F7CF91089580916210882329F042
:10FBE0006CED75E081E00C94074184E090E00C94AA
:10FBF000A66780916210882329F068EE73E081E0A7
:10FC00000C94074160E084E090E00C9404688091DB
:10FC1000621081111BC0809147108823B9F068EEF3
:10FC200073E081E00E9407411092471020E836E619
:10FC300048E95AE360E070E080915B1090915C10BD
:10FC40000E94E63F909346108093451008956CED16
:10FC500075E080E00C94074124EF31E0DB010E9465
:10FC6000AECB2FEF30E040E050E00E9484C9CA01E3
:10FC7000B90164527A4F8F4F9F4F80E00C94074137
:10FC800080916210882339F060ED77E081E00E9476
:10FC900007410C94826961E083E090E00C94046871
:10FCA00020916210211109C020914410222329F0D3
:10FCB00002960E9495691092441008952091621056
:10FCC000222389F06FE676E080E00E94074127E872
:10FCD00036E642E350E060E070E080915B10909186
:10FCE0005C100C94E63F20914410211106C002964E
:10FCF0000E94956981E080934410089580E00E94FD
:10FD00002E4181E00E942E4180916210811103C03A
:10FD100082E00E942E416CED75E080E00E94074178
:10FD20006CED75E081E00E940741809162108111C5
:10FD30000DC082E297EBA1E0BB27ABBFFC0167914E
:10FD4000769182E00E9407410C9469660895FC0157
:10FD50008485958597838683868597859187808717
:10FD60008089918993878287808D918D938B828BF7
:10FD7000828D938D958B848B848D958D978B868BBF
:10FD80000895FC018089918993878287828993896C
:10FD9000958784878489958997878687089526E043
:10FDA0000C94F092CF93DF93EC010E94245B688364
:10FDB00079838A839B83CE01DF91CF910895EF925F
:10FDC000FF921F93CF93DF93CDB7DEB765970FB642
:10FDD000F894DEBF0FBECDBF182F7B0188E09BE0FB
:10FDE0000E9467A781E08093360B84E690E09093B1
:10FDF000190B8093180B84E6E816F10418F484E6D6
:10FE0000E82EF12CC70164E670E00E9479CB709374
:10FE1000380B6093370B70931B0B60931A0B109386
:10FE2000150B8FEF810F823010F41230D1F088E083
:10FE30009BE00E948AA78091130B882329F083EC12
:10FE400095EFA8ECBFE304C084EB98ECA6E9B0E41E
:10FE50008093320B9093330BA093340BB093350BFC
:10FE600055C08091130B882329F084EB98ECA6E908
:10FE7000B0E404C083EC95EFA8ECBFE38093320BB1
:10FE80009093330BA093340BB093350B88E09BE039
:10FE90000E9494A78091360B8823C1F11092150B14
:10FEA0008EE690E09A83898388E290E09C838B833E
:10FEB0008CE390E09E838D831D8A83E08F938DB7C2
:10FEC0009EB745970FB6F8949EBF0FBE8DBFADB7D6
:10FED000BEB7119685E1FE01319601900D928A958B
:10FEE000E1F788E09BE00E949EA70FB6F894DEBF82
:10FEF0000FBECDBF65960FB6F894DEBF0FBECDBF67
:10FF0000DF91CF911F91FF90EF90089588E09BE0E3
:10FF100065960FB6F894DEBF0FBECDBFDF91CF91CF
:10FF20001F91FF90EF903ECF0F931F93CF93DF93DE
:10FF3000EC01AB0160E070E02AE00E9412908C01BD
:10FF4000CE010E945A90800F911FDF91CF911F9197
:10FF50000F9108958F929F92AF92BF92CF92DF92AE
:10FF6000EF92FF920F931F93CF93DF931F921F92F5
:10FF7000CDB7DEB7082E000C990BAA0BBB0BFC010A
:10FF80003197EF30F10508F066C28827E056FE4F42
:10FF90008F4F0C94A0CB84E08093F70A8AE0809383
:10FFA000F80A86E28093FA0A81E08093FD0A809342
:10FFB000FE0A8093FC0A4CEE5AE120E030E080918A
:10FFC000F70A90E0281739070CF08CC1FA018591E7
:10FFD0009491A0E0B0E0880F991FAA1FBB1FF90100
:10FFE000EE0FFF1FEE0FFF1FE257F54F8083918347
:10FFF000A283B3832F5F3F4F4E5F5F4FE0CF84E01C
:020000021000EC
:100000008093F70A8AE08093F80A86E28093FA0ADE
:1000100081E08093FD0A8093FE0A82E08093FC0ACF
:1000200044EE5AE120E030E08091F70A90E0281792
:1000300039070CF057C1FA0185919491A0E0B0E026
:10004000880F991FAA1FBB1FF901EE0FFF1FEE0FAC
:10005000FF1FE257F54F80839183A283B3832F5F05
:100060003F4F4E5F5F4FE0CF84E08093F80A85E218
:100070008093FA0A81E08093FD0A88E08093FE0A6B
:1000800083E08093FC0A80E090E0FC01E452F54EAE
:10009000E491DC01A150B54FEC93019688309105B5
:1000A000A1F70E94DF621EC188E08093F70A86E014
:1000B0008093F80A86E28093FA0A81E08093FD0A31
:1000C0008093FE0A84E08093FC0A4CEC5AE120E025
:1000D00030E08091F70A90E0281739070CF002C150
:1000E000FA0185919491A0E0B0E0880F991FAA1FB2
:1000F000BB1FF901EE0FFF1FEE0FFF1FE257F54F79
:1001000080839183A283B3832F5F3F4F4E5F5F4F06
:10011000E0CF88E08093F70A81E08093F80A97E2C5
:100120009093FA0A8093FD0A8093FE0A85E08093FB
:10013000FC0A4CEB5AE120E030E08091F70A90E0B5
:10014000281739070CF0CEC0FA0185919491A0E0F0
:10015000B0E0880F991FAA1FBB1FF901EE0FFF1F08
:10016000EE0FFF1FE257F54F80839183A283B38385
:100170002F5F3F4F4E5F5F4FE0CF82E18093F70AE2
:1001800081E08093F80A97E29093FA0A8093FD0A3F
:100190008093FE0A8FE08093FC0A48E95AE120E050
:1001A00030E08091F70A90E0281739070CF09AC0E8
:1001B000FA0185919491A0E0B0E0880F991FAA1FE1
:1001C000BB1FF901EE0FFF1FEE0FFF1FE257F54FA8
:1001D00080839183A283B3832F5F3F4F4E5F5F4F36
:1001E000E0CFE091620BF091630B74978081918175
:1001F00040E550E060E070E08E59944F0E94366414
:100200002AC182E18093F70A85E08093F80A82E2AE
:100210008093FA0A81E08093FD0A8093FE0A87E0CA
:100220008093FC0A80E993E3A0E0B0E080938E0A1B
:1002300090938F0AA093900AB093910AF2E08F2EC8
:10024000912C01E010E080E090E0A0E0BBE54CE400
:1002500054E060E070E024EEC22E2CE0D22EE12CBF
:10026000F12C9801220F331F220F331F5401AA0CC7
:10027000BB1CAA0CBB1C2257354FF901B7FF0DC0A0
:10028000C082D182E282F38295012257354FF90173
:1002900040835183628373830CC0408351836283A4
:1002A000738395012257354FF901C082D182E282D2
:1002B000F382880F991FAA1FBB1F0E5F1F4FF2E02A
:1002C0008F0E911C22E18216910459F688E79FEF68
:1002D000A0E0B0E08093D20A9093D30AA093D40A0E
:1002E000B093D50A0E944E63B6C0CE0101960E941B
:1002F000CB6223E040E150E060E070E072C084E057
:100300008093F70A82E38093F80A86E28093FA0AE0
:1003100081E08093FD0A8093FE0A8AE08093FC0AC4
:1003200040E95AE120E030E08091F70A90E0281798
:100330003907C4F6FA0185919491A0E0B0E0880FE6
:10034000991FAA1FBB1FF901EE0FFF1FEE0FFF1F22
:10035000E257F54F80839183A283B3832F5F3F4F92
:100360004E5F5F4FE1CF84E08093F70A80E2809395
:10037000F80A86E28093FA0A81E08093FD0A80936E
:10038000FE0A8BE08093FC0A48E85AE120E030E066
:100390008091F70A90E0281739070CF0A3CFFA01F3
:1003A00085919491A0E0B0E0880F991FAA1FBB1F10
:1003B000F901EE0FFF1FEE0FFF1FE257F54F80838D
:1003C0009183A283B3832F5F3F4F4E5F5F4FE0CF98
:1003D000CE0101960E94CB6221E040E154E060E052
:1003E00070E0CE0101960E94AA6335C084E080933C
:1003F000F70A83E08093F80A86E28093FA0A81E0A4
:100400008093FD0A8093FE0A8DE08093FC0A40E809
:100410005AE120E030E08091F70A90E02817390790
:100420000CF060CFFA0185919491A0E0B0E0880FC4
:10043000991FAA1FBB1FF901EE0FFF1FEE0FFF1F31
:10044000E257F54F80839183A283B3832F5F3F4FA1
:100450004E5F5F4FE0CF0F900F90DF91CF911F91D4
:100460000F91FF90EF90DF90CF90BF90AF909F9053
:100470008F9008950F931F93CF93DF93EC01462F36
:1004800050E060E070E02AE00E9412908C01CE0102
:100490000E945A90800F911FDF91CF911F910F9171
:1004A0000895462F50E060E070E02AE00C9412902E
:1004B00080914C0C811180C00E948578809114023B
:1004C000882321F080919214811105C080919114AC
:1004D000882309F471C01092921481E08093140271
:1004E0000E94AC78809190148823D1F065EA76E080
:1004F00080918E1490918F140E945191809191144B
:10050000882341F065EB76E080918E1490918F14F2
:100510000E94519180918E1490918F140E945A9054
:1005200080919114882369F060918C1470918D14DE
:100530001616170624F489ED9CE00E94973F10924E
:10054000911480918A1490918B14806290938B14F3
:1005500080938A1480918914882311F081E001C06E
:1005600080E00E9431A081E0809388140E949C77F3
:100570008091251481110FC08091A612882359F013
:100580002DEC36E744E650E060E070E089ED9CE059
:100590000E94E63F02C00E94CD760E94514E0E940A
:1005A00026780E94245B6093A2127093A31280931A
:1005B000A4129093A512089508952FB7F894882354
:1005C00081F0809127129091281290933612809397
:1005D0003512809137129091381218161906ACF026
:1005E0000FC08091291290912A1290933612809315
:1005F00035128091371290913812181619062CF482
:10060000809137129091381207C0809137129091E3
:1006100038129195819591099093381280933712F1
:100620002FBF0895AF92BF92CF92DF92EF92FF92C9
:100630000F931F93CF93DF931F921F92CDB7DEB717
:100640008C017A836983CE0101966C01580192E096
:10065000A90EB11CE12CF12CC8010E9464C9F6015D
:1006600061916F01861731F0C8010E9476C9FFEFD2
:10067000EF1AFF0A0F5F1F4F0A151B0569F781E08C
:10068000EF2809F480E00F900F90DF91CF911F9138
:100690000F91FF90EF90DF90CF90BF90AF900895B3
:1006A000EF92FF920F931F93CF93DF931F921F92AE
:1006B000CDB7DEB78C017B018AEA8A8341E050E046
:1006C000BE016E5F7F4FC8010E94CBA1D701ED91A3
:1006D000FC910680F781E02DC701199582E8898396
:1006E00041E050E0BE016F5F7F4FC8010E94CBA187
:1006F0000F900F90DF91CF911F910F91FF90EF908E
:100700000895CF92DF92EF92FF920F931F930E9472
:10071000245B6B017C016093941470939514809317
:100720009614909397148091630C0E945593809334
:1007300093149091650C992329F091E0811190E038
:100740009093931480916D0C90916E0CA0916F0C0E
:10075000B091700C97018601081B190B2A0B3B0BFB
:100760004091710C5091720C6091730C7091740CEB
:100770009091660C041715072607370760F4C0929E
:10078000690CD0926A0CE0926B0CF0926C0C109297
:10079000680C892F1EC09093670C809193148093EE
:1007A000660CC092690CD0926A0CE0926B0CF092CD
:1007B0006C0C891761F0C0926D0CD0926E0CE092B7
:1007C0006F0CF092700C91E09093680C02C0109244
:1007D000680C1F910F91FF90EF90DF90CF900895DC
:1007E0000F931F93CF93DF93EC012AE00E941290A6
:1007F0008C01CE010E945A90800F911FDF91CF9102
:100800001F910F910895CF92DF92EF92FF920F9375
:100810001F93CF93DF936B01770FEE08FF08F7FE6E
:100820001BC0EC016DE20E946D908C01442755279E
:10083000BA014C195D096E097F092AE0CE010E94B8
:100840001290800F911FDF91CF911F910F91FF9018
:10085000EF90DF90CF9008952AE0B701A601DF91D5
:10086000CF911F910F91FF90EF90DF90CF900C945C
:100870001290CF92DF92EF92FF920F931F93CF933C
:10088000DF938C016B01770FEE08FF08F7FE12C0B3
:100890006DE20E946D90EC0144275527BA014C1976
:1008A0005D096E097F092AE0C8010E941290C80FF5
:1008B000D91F06C02AE0B701A6010E941290EC01E0
:1008C000C8010E945A908C0F9D1FDF91CF911F91FC
:1008D0000F91FF90EF90DF90CF9008950F931F93AB
:1008E000CF93DF931F92CDB7DEB78C0169830E944F
:1008F00064C96981861729F0C8010E9476C981E020
:1009000001C080E00F90DF91CF911F910F9108956A
:100910008091660C811105C081E09091680C911165
:1009200001C080E00895CF930E947D5084E090E064
:100930009093600C80935F0C1092BD111092C711C0
:100940001092D1111092DB11E9E6F1E1DF011C9266
:10095000179681E1AD3BB807D1F788EA92E1909311
:10096000C6118093C5111092C01180915E0C9091B8
:10097000A812891718F091E09093BD1121EB32E194
:100980003093D0112093CF111092CA119091B112CF
:10099000891718F091E09093C7112AEB32E1309358
:1009A000DA112093D9111092D4119091BA128917AB
:1009B00018F091E09093D11123EC32E13093E411DF
:1009C0002093E3111092DE119091C312891718F051
:1009D00091E09093DB1110925D0C20E030E0D901A2
:1009E000A45BBC4E4D915C9141505109443251057C
:1009F00020F491E090935D0C05C02D5F3F4F2837A8
:100A0000310569F790915D0C992341F12091BB125A
:100A10003091BC122D5D3F4F3093BC122093BB121E
:100A20002091BD123091BE12235231093093BE1273
:100A30002093BD122091C4123091C5122D5D3F4FFD
:100A40003093C5122093C4122091C6123091C71260
:100A5000235231093093C7122093C6129091C513C7
:100A60009F3049F49091C6139F3029F41092681179
:100A70001092671108C020912314309124143093F0
:100A800068112093671122E130E0309365112093C3
:100A9000641120915F0C3091600CACECB2E141E04C
:100AA000B683A5839C91992329F0891718F0408378
:100AB0002F5F3F4F1A96379691E1ED3BF90781F78B
:100AC0003093600C20935F0C2131310534F080E1CC
:100AD00090E09093600C80935F0C0E94B64481EC90
:100AE00091E19093C7108093C6108091C5119091A9
:100AF000C6119093C5108093C4108EEB91E1909332
:100B0000C9108093C8108FEB91E19093CB10809324
:100B1000CA108DEB91E19093CD108093CC108BECAB
:100B200091E19093D1108093D0108091CF1190914A
:100B3000D0119093CF108093CE1088EC91E19093D8
:100B4000D3108093D21089EC91E19093D5108093CB
:100B5000D41087EC91E19093D7108093D61085ED57
:100B600091E19093DB108093DA108091D9119091EC
:100B7000DA119093D9108093D81082ED91E190937F
:100B8000DD108093DC1083ED91E19093DF10809372
:100B9000DE1081ED91E19093E1108093E0108FEDF4
:100BA00091E19093E5108093E4108091E31190918E
:100BB000E4119093E3108093E2108CED91E1909317
:100BC000E7108093E6108DED91E19093E91080930A
:100BD000E8108BED91E19093EB108093EA10209157
:100BE0005F0C3091600C2450310960E07AE0C7E07E
:100BF000462F50E04217530724F5CA010496789F08
:100C0000F001799FF00D1124EC53FF4EC49FC001F9
:100C1000C59F900D1124AC0145595E4E538342830C
:100C2000DC01A759BE4E15964D915C9116975183E4
:100C3000408386599E4E95838483B187A0876F5FDA
:100C4000D7CF81E08093610CCF9108950F931F93CC
:100C5000CF93DF93FC01248135812115310519F4EF
:100C6000FB01108211C0EA0121972C173D0708F4FF
:100C7000E9018B01FC0160817181AE01C8010E9414
:100C8000E4CDC00FD11F1882DF91CF911F910F913A
:100C900008950895089508950F931F93CF93DF93B8
:100CA0008C01FC01178A168AEC01699640E068E025
:100CB000CE010E94A7A24FE766E0CE010E94A7A244
:100CC00040E06CE0CE010E94A7A24FE767E0CE01B2
:100CD0000E94A7A20E94245BF801648F758F868F03
:100CE000978FDF91CF911F910F910895EF92FF920F
:100CF0000F931F93CF93DF938C01FC01778B668B4F
:100D00000E945262EC01F801828193818830910542
:100D100031F57801F9E1EF0EF11CD7FF06C06AE06A
:100D2000C1388FEFD80754F001C068E02C2F9D2FF9
:100D3000C038D1052CF02FE790E002C021E89FEFEA
:100D4000422F592F57FF03C0519541955109C701B3
:100D50000E94A7A2CD2B69F54FE766E027C009974F
:100D600041F57801E9E1EE0EF11CD7FF06C06EE017
:100D7000C138FFEFDF0754F001C06CE02C2F9D2F2E
:100D8000C038D1052CF02FE790E002C021E89FEF9A
:100D9000422F592F57FF03C0519541955109C70163
:100DA0000E94A7A2CD2B29F44FE767E0C7010E945C
:100DB000A7A20E94245BF801648F758F868F978F9E
:100DC000DF91CF911F910F91FF90EF900895CF93F6
:100DD000DF93EC0180919914811108C06A8D7B8D9D
:100DE000CE0149965DDC81E08093991421E83FEFC4
:100DF0003B872A878FE790E09D878C871F861E861A
:100E0000398B288B9B8B8A8B1D8A1C8ADF91CF9113
:100E100008950F931F93CF93DF93EC011F8A1E8ACF
:100E20008C01075E1F4F40E060E0C8010E945C43F8
:100E300040E064E0C8010E945C430E94245B6C8F28
:100E40007D8F8E8F9F8FDF91CF911F910F9108958E
:100E5000CF93DF93EC017F8B6E8B0E9452629C01DB
:100E60008A819B8188309105C1F437FF06C061E01B
:100E700021388FEF38074CF001C060E0A90120381D
:100E800031052CF04FE750E002C041E85FEF57FF1B
:100E90001FC05195419551091BC00997E9F4922F44
:100EA000832F2038310514F09FE780E0492F582F19
:100EB00041388FEF580714F441E85FEF57FF03C044
:100EC000519541955109632F661F6627661F6C5F18
:100ED000CE0149960E945C430E94245B6C8F7D8FFB
:100EE0008E8F9F8FDF91CF9108950F931F93CF9394
:100EF000DF93EC010E94245B0C8D1D8D2E8D3F8DA8
:100F0000DC01CB01801B910BA20BB30B853F914001
:100F1000A105B10540F06E897F89CE01DF91CF91A7
:100F20001F910F9195CFDF91CF911F910F91089550
:100F30000F931F93CF93DF93EC018091981481114D
:100F400012C00A8D1B8D6AEA70E0C8010E941C98CD
:100F5000D801ED91FC910680F781E02DC80119952B
:100F600081E0809398144AE06EE0CE0149960E9499
:100F70005C4321E83FEF3B872A878FE790E09D871E
:100F80008C871F861E86398B288B9B8B8A8B1D8AAC
:100F90001C8ADF91CF911F910F9108950F931F939A
:100FA000CF93DF93EC011F8A1E8A8C01075E1F4FCF
:100FB00040E060E0C8010E941F4340E064E0C801D7
:100FC0000E941F430E94245B6C8F7D8F8E8F9F8FAA
:100FD000DF91CF911F910F910895CF93DF93EC0193
:100FE0007F8B6E8B0E9452629C018A819B8188302C
:100FF0009105C1F437FF06C061E021388FEF380753
:101000004CF001C060E0A901203831052CF04FE719
:1010100050E002C041E85FEF57FF1FC05195419576
:1010200051091BC00997E9F4922F832F203831050D
:1010300014F09FE780E0492F582F41388FEF580771
:1010400014F441E85FEF57FF03C0519541955109F2
:10105000632F661F6627661F6C5FCE0149960E944C
:101060001F430E94245B6C8F7D8F8E8F9F8FDF913B
:10107000CF9108950F931F93CF93DF93EC010E94BC
:10108000245B0C8D1D8D2E8D3F8DDC01CB01801BD3
:10109000910BA20BB30B853F9140A105B10540F028
:1010A0006E897F89CE01DF91CF911F910F9195CFEE
:1010B000DF91CF911F910F9108950F931F93CF93BD
:1010C000DF93EC01E8A1F9A180819181A281B38134
:1010D0008E01075E1F4F81159649A105B10509F4E0
:1010E00051C040E056E960E070E087EB98E00E9474
:1010F000CF7E64E170E080E090E00E94EC5AE8A1CD
:10110000F9A180819181A281B38181152BE492079D
:10111000A105B105E9F068F4803629E09207A10540
:10112000B105A1F080389542A105B105C1F442E0B6
:1011300012C0811521EE9207A105B10559F0811564
:10114000924CA140B10559F445E005C041E003C00F
:1011500043E001C046E06FE0C8010E941F4387EBF7
:1011600098E091D5E8A1F9A1408151816281738114
:1011700087EB98E00E94CF7E64E170E080E090E031
:101180000E94EC5A4AE06EE0C8010E941F4341E011
:1011900067E1C8010E941F434AA168E1C8010E949B
:1011A0001F434BA18FEF840F8E3108F04CE066E1B6
:1011B000C8010E941F4321E83FEF3B872A878FE742
:1011C00090E09D878C871F861E86398B288B9B8B92
:1011D0008A8B1D8A1C8ADF91CF911F910F910895F0
:1011E000EF92FF920F931F93CF93DF93EC0166234F
:1011F000E1F0262F653608F024E60A891B89E88885
:10120000F988D801AE19BF0930E00E94AECB28ECB6
:1012100030E040E050E00E94B0C9E20EF31EFB86D1
:10122000EA86021B130B1D870C87DF91CF911F915C
:101230000F91FF90EF900895CF93DF93CDB7DEB776
:10124000A4970FB6F894DEBF0FBECDBF81310CF06E
:1012500081E12FEC3BE13A83298327EC3BE13C839E
:101260002B832FEB3BE13E832D8327EB3BE138873C
:101270002F832FEA3BE13A87298727EA3BE13C8726
:101280002B872FE93BE13E872D8727E93BE1388B10
:101290002F8729E83BE13A8B298B27E73BE13C8B01
:1012A0002B8B2AE53BE13E8B2D8B25E43BE1388FF0
:1012B0002F8B2BE33BE13A8F298F21E33BE13C8FDE
:1012C0002B8F24E23BE13E8F2D8F28E13BE138A3B9
:1012D0002F8F2CEF3AE13AA329A324EF3AE13CA364
:1012E0002BA3E82FEE0FFF0BEC0FFD1F81819281E6
:1012F000A4960FB6F894DEBF0FBECDBFDF91CF919D
:10130000089580914110909142108068909342100E
:101310008093411008958091411090914210806116
:1013200090934210809341100895FC01828188239C
:1013300071F08381882359F013828091411090913C
:10134000421024E082279093421080934110089528
:10135000FC018281882371F0838181110BC081E0BF
:101360008383809141109091421084609093421049
:10137000809341100895FC018481882371F0858158
:10138000882359F01582809141109091421028E0F5
:10139000822790934210809341100895FC0184812C
:1013A000882371F0858181110BC081E08583809154
:1013B00041109091421088609093421080934110A8
:1013C0000895809141109091421020E282279093DD
:1013D00042108093411008958091411090914210E5
:1013E000806290934210809341100895DC01ED914A
:1013F000FC910680F781E02D60E070E0199477FFA2
:1014000003C07195619571096F3F710519F014F072
:101410006FEF70E080914110909142108C7B917041
:10142000909342108093411080914110909142100E
:101430006F30710514F480641FC06733710514F4B4
:1014400081641AC06F3571051CF48164906114C009
:10145000673871051CF4816490630EC06F3A7105A2
:101460001CF48164906408C0673D71051CF48164BC
:10147000906502C081649066909342108093411001
:10148000089580E094E09093421080934110089575
:1014900080914110909142109260909342108093FD
:1014A00041100895089508950895089508950895A0
:1014B000089508950895089580E008950895089581
:1014C0000895089508950895089508950895089534
:1014D0000895089508950895089508950895089524
:1014E0000895089580E00895089508950895FC01F1
:1014F00064830895FC0162830895FC0113821482C1
:10150000158216821782108611860895089508950F
:101510000895FC0183810895FC0165830895FC0111
:1015200064830895FC0160870895FC016683089533
:10153000FC01128213821482158261E086E10E940E
:10154000675861E086E10E94EF56E2E7F0E08081B3
:1015500081608083109242101092411008951F9272
:101560000F920FB60F9211240BB60F920F931F9389
:101570002F933F934F935F936F937F938F939F939B
:10158000AF93BF93EF93FF938091A2148F5F8093EB
:10159000A2149091A114891708F42FC11092A214DB
:1015A0008091A01490E08730910508F026C1FC01DD
:1015B0008827E155FE4F8F4F0C94A0CB60E086E169
:1015C0000E94EF5680E48093A11481E048C061E05E
:1015D00086E10E94EF5688E08093A11436C060E057
:1015E00086E10E94EF5680919E1490919F1497FF80
:1015F00005C088E18093A11484E031C088E0809325
:10160000A11483E02CC061E086E10E94EF5688E1DE
:101610008093A11480919D148F5F80939D148031DD
:1016200050F010929D1485E01AC061E086E10E949E
:10163000EF5688E0EDCF80919E1490919F14880F13
:10164000991F90939F1480939E1482E008C060E0DD
:1016500086E10E94EF5688E08093A11486E0809393
:10166000A014CBC061E086E10E94EF5680EC80932D
:10167000A114809141109091421090939F148093F7
:101680009E14809141109091421091FF1CC0809156
:101690009C14882369F0809141109091421022E0BF
:1016A0009227909342108093411010929C140BC08B
:1016B00081E080939C1480939B1480939A1482E819
:1016C0009BE00E94D27E80919A148823D1F0809171
:1016D0009B148823B1F00E94245B0091820B10912F
:1016E000830B2091840B3091850BDC01CB01801B97
:1016F000910BA20BB30B8D369042A105B10508F0FA
:1017000070C0809141109091421092FF12C0809160
:101710009C14882339F010924210109241101092BC
:101720009C1407C081E080939C1410929B1410922B
:101730009A14809141109091421084FF14C08091BE
:101740009C14882369F0809141109091421020E10F
:101750008227909342108093411010929C1403C0F2
:1017600081E080939C14809141109091421087FFFA
:1017700013C080919C14882361F080914110909156
:1017800042108058909342108093411010929C1404
:1017900003C081E080939C1480914110909142108D
:1017A00090FF14C080919C14882369F080914110AF
:1017B0009091421021E09227909342108093411023
:1017C00010929C1403C081E080939C14809141107E
:1017D0009091421090939F1480939E141092A014A5
:1017E0000CC010929A148091411090914210806424
:1017F000909342108093411084CFFF91EF91BF915D
:10180000AF919F918F917F916F915F914F913F9198
:101810002F911F910F910F900BBE0F900FBE0F9045
:101820001F901895FF920F931F93CF93DF938C0116
:10183000C62FF42ED22F6AED70E0DC011A968D913E
:101840009C911B970E941C98F80182859385DC016E
:10185000ED91FC910190F081E02D6C2F1995F8012C
:1018600082859385DC01ED91FC910190F081E02D62
:101870006F2D1995F80182859385DC01ED91FC911E
:101880000190F081E02D6D2F1995EC2FF0E0BF0154
:1018900066527F4F6F0D711D6D0F711D6F7777272A
:1018A000F80182859385DF91CF911F910F91FF9071
:1018B0000C941C9820E040E0B5CF65E4FBCF68E4D1
:1018C000F9CFCF93DF93FC012381222321F0EC0198
:1018D00061E4F0DF1B82DF91CF910895CF93DF9316
:1018E000FC012381211105C0EC0160E4E3DF81E00C
:1018F0008B83DF91CF91089563E5DCCFFC012581D7
:10190000222311F060E5D6CF0895FC012481222323
:1019100011F06CE3CFCF0895FC012085222331F034
:101920002185222319F011866BE3C4CF0895FC01B1
:101930002085222339F02185211104C021E021874F
:101940006AE3B8CF0895FC012681222331F0278174
:10195000222319F0178269E3ADCF0895FC01268197
:10196000222339F02781211104C021E0278368E375
:10197000A1CF089567E39ECF6AE49CCF69E49ACF34
:1019800066E398CF65E396CF6EE494CF64E392CF9D
:10199000242F462F6CE446CF462F20E067E442CF49
:1019A000462F20E066E43ECF262F64E43BCFCF9263
:1019B000DF92FF920F931F93CF93DF938C01F62E4C
:1019C000443F81E0580738F0413187E2580728F05A
:1019D00040E157E202C044EF51E0243F81E0380784
:1019E00038F0E9012131374228F0C0E1D7E202C0E6
:1019F000C4EFD1E0CA01845F914022E3C22ED12C12
:101A0000B6010E9479CB462F2F2D62E4C8010ADF70
:101A1000CE01845F9140B6010E9479CB462F2F2DD5
:101A200063E4C801DF91CF911F910F91FF90DF9088
:101A3000CF90F8CE242F462F62E5F4CE242F462FE8
:101A400061E5F0CE262F40E06FE3ECCE262F40E09C
:101A50006EE3E8CE262F40E06DE3E4CE462F20E093
:101A60006FE4E0CE0895CF92DF92EF92FF920F9352
:101A70001F93CF93DF936C017A018B01C0E0D0E01C
:101A8000CE15DF0589F0D8016D918D01D601ED915C
:101A9000FC910190F081E02DC6011995892B11F47C
:101AA0007E0102C02196ECCFC701DF91CF911F913B
:101AB0000F91FF90EF90DF90CF900895FC01A089E7
:101AC000B1898C91A689B78982FD0FC09C91818DC7
:101AD0008F5F8F73228D821749F0218DDF01A20F56
:101AE000B11D5D969C93818F08958C910895089502
:101AF00080E090E00895FC01538D448D252F30E067
:101B0000842F90E0821B930B541710F0CF9608950A
:101B100001970895FC01918D828D981761F0828D57
:101B2000DF01A80FB11D5D968C91928D9F5F9F7311
:101B3000928F90E008958FEF9FEF0895FC01918DB3
:101B4000828D981731F0828DE80FF11D858D90E020
:101B500008958FEF9FEF0895FC01918D228D892FBD
:101B600090E0805C9F4F821B91098F7399270895A5
:101B70008AE198E0F1DF21E0892B09F420E0822F4F
:101B8000089587EB98E0E8DF21E0892B09F420E055
:101B9000822F089584E599E0DFDF21E0892B09F4A5
:101BA00020E0822F089581EF99E0D6DF21E0892B94
:101BB00009F420E0822F0895FC01848DDF01A80F35
:101BC000B11DA35ABF4F2C91848D90E001968F7365
:101BD0009927848FA689B7892C93A089B1898C9184
:101BE00080648C93938D848D981306C00288F3894A
:101BF000E02D80818F7D80830895EF92FF920F9377
:101C00001F93CF93DF93EC0181E0888F9B8D8C8DA8
